:100000000C9463280C9494280C9494280C949428B1
:100010000C9494280C9494280C9494280C94942870
:100020000C9494280C9494280C9494280C94942860
:100030000C9494280C94934E0C9494280C9494282B
:100040000C9494280C94EC5D0C9494280C949428B3
:100050000C9494280C9494280C94AFCB0C94F350EB
:100060000C9494280C9410900C9494280C9494283C
:100070000C9494280C9494280C9494280C94942810
:100080000C9494280C9494280C9494280C94942800
:100090000C9494280C9494280C9494280C949428F0
:1000A0000C9494280C9494280C9494280C949428E0
:1000B0000C9494280C9494280C9494280C949428D0
:1000C0000C9494280C9494280C9494280C949428C0
:1000D0000C9494280C9494280C9494280C949428B0
:1000E0000C949428714F744F634F674F6D4FAB4F13
:1000F000784F7C4F824F864F8A4F904F944F984F46
:10010000AB4F9E4FA24FA64F0F5014501950235083
:100110002D50A65037503F50475051505B506550BE
:1001200074507E50A650885092509C50084AD73B3D
:100130003BCE016E84BCBFFDC12F3D6C74319ABDB6
:1001400056833DDA3D00C77F11BED9E4BB4C3E91DA
:100150006BAAAABE000000803F05A84CCDB2D44EC9
:10016000B93836A9020C50B9918688083CA6AAAACB
:100170002ABE000000803F004E414E494E4954596E
:10018000494E46CDCCCC3D0AD7233C17B7D1387762
:10019000CC2B329595E6241FB14F0A000020410078
:1001A00000C84200401C4620BCBE4CCA1B0E5AAEC2
:1001B000C59D74434F4D4D554E49434154494F4E93
:1001C0000044525952554E004552524F5253004925
:1001D0004E464F004543484F0047322F4733206279
:1001E000616420706172616D65746572730A005399
:1001F0006C6565702E2E2E00205A3A200020593A48
:10020000200042656420583A2000436865617033DD
:100210004420563330302072656164792E00526577
:1002200073756D696E67207072696E7400436C69D6
:10023000636B20746F20726573756D652E2E2E00B2
:10024000456E642066696C65206C6973740A0042AF
:100250006567696E2066696C65206C6973740A0055
:100260005344207072696E74696E67206279746598
:1002700020004E6F74205344207072696E74696E52
:10028000670A0046696C652064656C657465643A4C
:100290000044656C6574696F6E206661696C6564A5
:1002A0002C2046696C653A20006F70656E2066618F
:1002B000696C65642C2046696C653A200025697379
:1002C0000025696D20256973002569682025696D01
:1002D0002025697300256964202569682025696DDA
:1002E00020256973002569792025696420256968BE
:1002F0002025696D20256973005072696E74207421
:10030000696D653A200050726F746563746564208E
:1003100050696E0A004525692025730043686561B0
:1003200070334420563330302072656164792E007A
:10033000D401CF01C801C101B3016F666600444515
:100340004255473A004B494C4C45442E20004D3114
:1003500031332053006F6B0048656174696E67200C
:10036000646F6E652E003F0A0020573A00452569EC
:100370002025730043686561703344205633303064
:100380002072656164792E0042656420646F6E6539
:100390002E003F0A0020573A0042656420486561FC
:1003A00074696E672E00436865617033442056336C
:1003B0003030204F66662E0056333030204C3120CE
:1003C000423A312054303A352054313A30204649AF
:1003D000524D574152455F4E414D453A4D61726C09
:1003E000696E20312E312E3020284769746875627D
:1003F0002920534F555243455F434F44455F555263
:100400004C3A68747470733A2F2F67697468756218
:100410002E636F6D2F4D61726C696E4669726D77D8
:100420006172652F4D61726C696E2050524F544F4E
:10043000434F4C5F56455253494F4E3A312E302070
:100440004D414348494E455F545950453A436865CC
:10045000617033442056333030204558545255444F
:1004600045525F434F554E543A3120555549443A11
:1004700063656465326132662D343161322D343703
:1004800034382D396231322D633535633632663377
:10049000363766660A0053657474696E6720547255
:1004A0006176656C20416363656C65726174696F28
:1004B0006E3A200053657474696E672052657472D9
:1004C00061637420416363656C65726174696F6E0A
:1004D0003A200053657474696E67205072696E74B7
:1004E00020416363656C65726174696F6E3A2000C8
:1004F00053657474696E67205072696E7420616E02
:10050000642054726176656C20416363656C65722A
:100510006174696F6E3A2000205A0020590058001B
:1005200020204D61783A2000205A002059005800C0
:1005300020204D696E3A20004F6E20004F66660005
:10054000536F667420656E6473746F70733A200025
:1005500020643A0020693A0020703A0043290A00DA
:1005600061626C656420286D696E2074656D702011
:1005700000436F6C642065787472756465732061E4
:100580007265200023646566696E652020444546D7
:1005900041554C545F4B64200023646566696E6569
:1005A000202044454641554C545F4B69200023644C
:1005B0006566696E65202044454641554C545F4B45
:1005C000702000504944204175746F74756E652029
:1005D00066696E697368656421205075742074685B
:1005E00065206C617374204B702C204B6920616E08
:1005F00064204B6420636F6E7374616E7473206645
:10060000726F6D2062656C6F7720696E746F204326
:100610006F6E66696775726174696F6E2E680A0025
:10062000504944204175746F74756E652066616928
:100630006C6564212074696D656F75740A0050499A
:1006400044204175746F74756E65206661696C65D0
:1006500064212054656D70657261747572652074D3
:100660006F6F20686967680A00204B643A20002099
:100670004B693A2000204B703A20000A20436C61FD
:100680007373696320504944200A002054753A204E
:1006900000204B753A2000206D61783A2000206DD3
:1006A000696E3A200020643A200020626961733A42
:1006B00020004F666673657473206170706C6965A5
:1006C00064004572723A20546F6F20666172210097
:1006D000546F6F206661722066726F6D207265665E
:1006E0006572656E636520706F696E740A004545BA
:1006F00050524F4D2064697361626C65640A003A20
:1007000020007A5F6D696E3A20202D3230207A5FAA
:100710006D61783A20203230005A204F666673654A
:100720007420004E6F2063617365206C6967687484
:100730000A00416374697665204578747275646552
:10074000723A2000556E6B6E6F776E20636F6D6D21
:10075000616E643A20220025753A253032750025F5
:100760003032753A253032750025756420253032D7
:10077000753A25303275005A00590058000920009A
:100780000000000000000000000000007FFFE0000B
:1007900000000000000000000000007000E0000009
:1007A0000000000000000000000061F86000000090
:1007B00000000000000000000041F82000000000E0
:1007C000000000000000000040F0200000000000D9
:1007D0000000000000000040602000000000000059
:1007E0000000000000005801A07F80000000000011
:1007F00000004104005C63A0FFC000000000000096
:10080000002082005EF7A0FFC00000000000000092
:100810002082005EF7A0FFC0000000000000004141
:1008200004005C63A07F80000000000000008208DC
:10083000005801A07F8000000000000001041000AB
:10084000406020FFC00000000000000104100040D4
:10085000F020FFC00000000000000082080041F806
:1008600020FFC00000000000000041040061F860AB
:100870003F00000000000000000000007000E01ECB
:100880000000000000000001FFFF807FFFE00C007F
:1008900000000000000001FFFF80000000000000D9
:1008A0000000000000000000007FFFE000000000EA
:1008B00000000000000000007000E00000000000E8
:1008C00000000000000000630C6000000000000059
:1008D000000000000000470E2000000000000000A3
:1008E00000000000004F0F2000000000000000008A
:1008F000000000005F0FA0000000000000000000EA
:100900000000005E07A07F800000000000000041A2
:100910000400406020FFC0000000000000002082B2
:100920000040F020FFC00000000000000020820016
:1009300040F020FFC0000000000000004104004023
:1009400060207F80000000000000008208005E0739
:10095000A07F80000000000000010410005F0FA0D5
:10096000FFC0000000000000010410004F0F20FF36
:10097000C000000000000000820800470E20FFC0F9
:1009800000000000000000410400630C603F000014
:100990000000000000000000007000E01E000000E9
:1009A0000000000001FFFF807FFFE00C000000005E
:1009B00000000001FFFF800000005072696E74208B
:1009C00061626F72746564004E6F205344206361EE
:1009D0007264005072696E742066726F6D205344A9
:1009E0000053746F70207072696E74005265737575
:1009F0006D65207072696E7400506175736520704A
:100A000072696E7400436F6E74726F6C0050726521
:100A1000706172650054756E6500496E666F207373
:100A2000637265656E0000060900FE0000000000AC
:100A300001090008FE000005080806000040F0C893
:100A40008888987810050808060000C0F88888880B
:100A50008888F80505050600012030F830200508D3
:100A6000080600002070F820202020E00509090673
:100A700000FF2070A8A8B888887020050909060022
:100A8000FFE080C0B0A8283028280509090600FF2B
:100A9000F8A88888888888A8F8050A0A0600FE2031
:100AA0005050505088A8A8887003030306000340E4
:100AB000A04000002200250028002B002E0031005D
:100AC000340002010000050108010B0100002000B4
:100AD0002300260029002C002F0032000001000016
:100AE00003010601090105050505070508080808B1
:100AF000020202020A0A08080404040401010101B6
:100B000001010101030303030303030304070707B0
:100B10000C0C0C0C0C0C0C0C020202020606060655
:100B2000060606060B0B0B0B0B0B0B0B0102102022
:100B30002008081020401020408002010201080413
:100B400002010102040810204080804020100804A7
:100B50000201800402018040201008040201080400
:100B60000201010204081020408001020408102044
:100B7000408000000A0B02090C0D0E080703040157
:100B80000000000000000000000000000000000065
:100B90000000000000000000000000000000121132
:100BA0001000000000000000000000000000000035
:100BB00000000000000000004B494C4C45442E2032
:100BC00000202D20496E76616C696420657874720E
:100BD00075646572206E756D62657220210A002051
:100BE00020506C616E6E6572427566666572427900
:100BF0007465733A20002046726565204D656D6FFF
:100C000072793A2000436F6D70696C65643A204DCB
:100C1000617920323320323031370A00207C204184
:100C20007574686F723A20286E6F6E652C2064654B
:100C30006661756C7420636F6E666967290A00329D
:100C40003031372D30352D30342031323A303000CC
:100C5000204C61737420557064617465643A20009F
:100C6000312E312E300A004D61726C696E002053B6
:100C70006F6674776172652052657365740A00202F
:100C80005761746368646F672052657365740A0006
:100C90002042726F776E206F757420526573657491
:100CA0000A002045787465726E616C205265736528
:100CB000740A00506F77657255700A007374617220
:100CC000740A006572726F722077726974696E6758
:100CD00020746F2066696C650A00456E6473746FDA
:100CE0007073202563202563202563202563002061
:100CF0005A3A0020593A0020583A00656E647374DD
:100D00006F7073206869743A2000446F6E652073B9
:100D10006176696E672066696C652E0A004D32390E
:100D20000002436172642072656D6F7665640043F2
:100D300061726420696E73657274656400000021DD
:100D400000240027002A002D00300033000101009C
:100D500000040107010A0100060900FE07019203D1
:100D60002120FFFF08FF07FF000000060000010729
:100D70000706020080808080800080030202060156
:100D800005A0A00507070600005050F850F8505085
:100D90000507070600002078A07028F02005070747
:100DA000060000C0C810204098180507070600007C
:100DB0006090A040A89068020303060104C0408030
:100DC00003070706010020408080804020030707BA
:100DD0000601008040202020408005050506000116
:100DE00020A870A8200505050600012020F8202075
:100DF0000203030602FFC04080050101060003F85C
:100E0000020202060200C0C0050505060001081026
:100E10002040800507070600007088888888887051
:100E200003070706010040C040404040E0050707B7
:100E3000060000708808708080F80507070600002B
:100E4000F81020100808F0050707060000103050C1
:100E500090F81010050707060000F880F0080888D1
:100E600070050707060000708080F088887005070D
:100E700007060000F80810202020200507070600BC
:100E800000708888708888700507070600007088E1
:100E90008878080870020505060200C0C000C0C0BE
:100EA0000206060602FFC0C000C040800407070615
:100EB000000010204080402010050303060002F8C7
:100EC00000F804070706010080402010204080053C
:100ED0000707060000708808102000200507070695
:100EE000000070880868A8A8700507070600007051
:100EF0008888F8888888050707060000F08888F049
:100F00008888F00507070600007088808080887058
:100F1000050707060000F08888888888F00507071D
:100F2000060000F88080F08080F8050707060000C2
:100F3000F88080F0808080050707060000708880B8
:100F4000B8888870050707060000888888F88888B0
:100F50008801070706020080808080808080050766
:100F600007060000381010101090600507070600F3
:100F7000008890A0C0A09088050707060000808028
:100F800080808080F805070706000088D8A8888838
:100F900088880507070600008888C8A898888805FB
:100FA000070706000070888888888870050707068C
:100FB0000000F08888F08080800507070600007038
:100FC000888888A89068050707060000F08888F0E0
:100FD000A09088050707060000788080700808F058
:100FE000050707060000F82020202020200507071D
:100FF0000600008888888888887005070706000032
:101000008888888888502005070706000088888817
:101010008888A85005070706000088885020508857
:1010200088050707060000888888502020200507CB
:1010300007060000F80810204080F80307070601A3
:1010400000E08080808080E005050506000180408A
:10105000201008030707060100E02020202020E0E0
:10106000050303060004205088050101060000F86E
:101070000202020602058040050505060000700810
:101080007888780507070600008080B0C88888F057
:1010900005050506000070808088700507070600BA
:1010A000000808689888887805050506000070889B
:1010B000F880700507070600003048E040404040D7
:1010C0000506060600FF7088887808700507070681
:1010D00000008080B0C88888880107070602008069
:1010E0000080808080800308080601FF2000202007
:1010F0002020A040040707060000808090A0C0A028
:1011000090030707060100C04040404040E005054D
:1011100005060000D0A8A8A8A8050505060000B08F
:10112000C8888888050505060000708888887005CD
:1011300006060600FFF08888F08080050606060097
:10114000FF788888780808050505060000B0C88083
:10115000808005050506000070807008F004070710
:101160000600004040E04040403005050506000014
:1011700088888898680505050600008888885020BA
:101180000505050600008888A8A850050505060085
:101190000088502050880506060600FF8888887859
:1011A0000870050505060000F8102040F803070741
:1011B0000601002040408040402001070706020051
:1011C0008080808080808003070706010080404087
:1011D00020404080050202060002689000000006E0
:1011E00000000000000600000000000600000000F3
:1011F00000060000000000060000000000060000DD
:1012000000000006000000000006000000000006CC
:1012100000000000000600000000000600000000C2
:1012200000060000000000060000000000060000AC
:10123000000000060000000000060000000000069C
:101240000000000000060000000000060000000092
:10125000000600000000000600000000000600007C
:10126000000000060000000000060000000000066C
:101270000000000000060000000000060000000062
:10128000000600000000000600000000000600004C
:10129000000000060000000000060000000000063C
:1012A00000000000000600000107070602008000A1
:1012B00080808080800507070600002070A8A0A815
:1012C0007020050707060000304040E04050A805A8
:1012D00005050600008870507088050707060000A5
:1012E000885020F820F8200107070602008080803F
:1012F00000808080050808060000304820505020FB
:101300009060030101060107A0050707060000F829
:1013100088B8B8B888F8050707060001700878880B
:101320007800F80505050600012850A0502805039F
:1013300003060001F80808020202060206408005C2
:101340000707060000F888A88898A8F80501010694
:101350000006F80404040600036090906005070787
:101360000600002020F8202000F8040505060003F0
:1013700060902040F0030505060003E020E020E037
:1013800002020206020640800508080600FF88885F
:10139000888898E880800507070600007898987884
:1013A000181818020202060202C0C0020202060257
:1013B000FF408003050506000340C04040E00507EC
:1013C00007060001708888887000F805050506008A
:1013D00001A0502850A00507070600008890A858D3
:1013E000B808080507070600008890B84898203814
:1013F000050808060000C040C048D838080805079E
:1014000007060000200020408088700508080600BC
:10141000004020007088F888880508080600001041
:1014200020007088F8888805080806000020500011
:101430007088F888880508080600006890007088A1
:10144000F888880508080600005000708888F88829
:10145000880508080600002050207088F888880554
:1014600007070600003860A0B8E0A0B80508080625
:1014700000FF7088808088702060050808060000E2
:10148000402000F880F080F80508080600000810E9
:1014900000F880F080F8050808060000205000F8E9
:1014A00080F080F80507070600005000F880F08003
:1014B000F8030808060100804000E0404040E003D7
:1014C0000808060100204000E0404040E003080812
:1014D00006010040A000E0404040E003070706018D
:1014E00000A000E0404040E005070706000070480B
:1014F00048E848487005080806000068900088C859
:10150000A898880508080600004020708888888808
:10151000700508080600001020708888888870050B
:1015200008080600002050007088888870050808A8
:10153000060000689000708888887005080806001A
:1015400000500070888888887005050506000188AD
:10155000502050880508080600FF1070A8A8A8A809
:101560007040050808060000402088888888887038
:1015700005080806000010208888888888700508FB
:101580000806000020500088888888700508080632
:1015900000005000888888888870050808060000C8
:1015A00010208850202020200509090600FFC04097
:1015B000704848704040E00408080601FF609090C1
:1015C000A09090E080050808060000402000700808
:1015D00078887805080806000010200070087888D0
:1015E0007805080806000020500070087888780503
:1015F00008080600006890007008788878050707DA
:101600000600005000700878887805080806000079
:101610002050207008788878050606060000D0283B
:1016200078A0A8500506060600FF7080887020602C
:101630000508080600004020007088F88070050842
:10164000080600001020007088F880700508080661
:1016500000002050007088F8807005070706000021
:1016600050007088F8807003080806010080400070
:1016700040C04040E003080806010020400040C090
:101680004040E003080806010040A00040C0404080
:10169000E0030707060100A00040C04040E0050746
:1016A00007060000A040A010788870050808060012
:1016B00000689000B0C888888805080806000040C7
:1016C0002000708888887005080806000010200037
:1016D000708888887005080806000020500070880F
:1016E000888870050808060000689000708888885F
:1016F000700507070600005000708888887005058F
:10170000050600012000F800200507070600FF106D
:1017100070A8A8A8704005080806000040200088AE
:1017200088889868050808060000102000888888C6
:101730009868050808060000205000888888986886
:101740000507070600005000888888986805090981
:101750000600FF102000888888F808700407070634
:1017600001FFC04060506040E00508080600FF50DF
:101770000088888878087024F4D43050C38E20C242
:10178000A24017828B7011127A910D816CD90AA830
:1017900061E108C7586607615143061E4B5D05C1EC
:1017A00045A7041A411104093D98037139310340DA
:1017B00036DB0265339102D4305402802E1D026361
:1017C0002CEE01752AC501B028A001102781018FD8
:1017D0002564012B244B01E0223401AC211F018D33
:1017E000200D01801FFC00841EED00971DDF00B856
:1017F0001CD200E61BC600201BBC00641AB200B25B
:1018000019A8000A19A0006A189900D11791004080
:10181000178B00B516840031167E00B31579003A97
:10182000157300C7146F0058146A00EE1366008821
:1018300013630025135E00C7125B006C125700157E
:10184000125400C111510070114F0021114B00D6EC
:101850001049008D1047004610440002104200C09D
:101860000F4000800F3E00420F3C00060F3B00CBB4
:101870000E3800930E37005C0E3500270E3400F34F
:101880000D3200C10D3100900D3000600D2E003280
:101890000D2D00050D2C00D90C2B00AE0C29008558
:1018A0000C29005C0C2700350C27000E0C2600E8E4
:1018B0000B2400C40B2400A00B23007D0B23005A33
:1018C0000B2100390B2100180B2000F80A1F00D94A
:1018D0000A1E00BB0A1E009D0A1D00800A1D00632F
:1018E0000A1C00470A1B002C0A1B00110A1A00F7E9
:1018F000091A00DD091900C4091900AB0919009281
:101900000917007B091800630917004C09160036F7
:10191000091600200916000A091500F5081500E04F
:10192000081400CC081400B8081400A4081400908F
:101930000813007D0812006B0813005808120046B7
:1019400008120034081100230811001208110001C8
:10195000081100F0071000E0071000D0071000C0C9
:10196000071000B0070F00A107100091070E0083B9
:10197000070F0074070F0065070E0057070E004998
:10198000070E003B070D002E070E0020070D001369
:10199000070D0006070D00F9060C00ED060D00E02E
:1019A000060C00D4060C00C8060C00BC060C00B0E7
:1019B000060C00A4060B0099060C008D060B008295
:1019C000060B0077060B006C060B0061060A005739
:1019D000060B004C060A0042060A0038060A002ED2
:1019E000060A0024060A001A060A00100609000763
:1019F000060A00FD050900F4050900EB050900E2EF
:101A0000050900D9050900D0050900C7050900BE70
:101A1000050900B5050800AD050800A50509009CED
:101A2000050800940508008C050800840508007C62
:101A3000050800740508006C050700650508005DD1
:101A4000050700560508004E05070047050700403A
:101A500005080038050700310507002A050700239F
:101A60000507001C050600160507000F05070008FE
:101A700005060002050700FB040600F5040700EE5A
:101A8000040600E8040600E2040700DB040600D5B3
:101A9000040600CF040600C9040600C3040600BD06
:101AA000040600B7040600B1040500AC040600A655
:101AB000040600A00405009B0406009504050090A0
:101AC0000406008A04050085040500800406007AE7
:101AD00004050075040500700405006B040500662C
:101AE000040500610405005C04050057040500526C
:101AF0000405004D04050048040500430405003EAC
:101B00000404003A04050035040500300404002CE8
:101B100004050027040400230405001E0404001A21
:101B200004040016040500110404000D0404000957
:101B30000405000404040000040400FC030400F88D
:101B4000030400F4030400F0030400EC030400E8C1
:101B5000030400E4030400E0030400DC030400D8F1
:101B6000030400D4030400D0030400CC030400C821
:101B7000030300C503030024F404D9201BC40C5C38
:101B80000E9804C4095F0265077101F405F900FBB2
:101B900004B30048048700C10369005803550003DB
:101BA000034500BE023A008402310053022A002994
:101BB00002250004022000E4011C00C8011900AF46
:101BC00001170098011400840113007101100061D5
:101BD00001100051010E0043010D0036010B002BD6
:101BE000010B0020010B00150109000C0109000385
:101BF000010800FB000800F3000800EB000700E408
:101C0000000600DE000600D8000600D2000600CC68
:101C1000000500C7000500C2000500BD000400B9B2
:101C2000000400B5000400B1000400AD000400A9E8
:101C3000000400A5000300A20003009F0004009B15
:101C40000003009800030095000200930003009039
:101C50000003008D0002008B000300880002008654
:101C600000020084000300810002007F0002007D6A
:101C70000002007B0002007900020077000100767C
:101C80000002007400020072000100710002006F87
:101C90000002006D0001006C0002006A0001006992
:101CA0000002006700010066000100650001006499
:101CB0000002006200010061000100600001005F9D
:101CC0000002005D0001005C0001005B0001005AA1
:101CD00000010059000100580001005700010056A2
:101CE00000010055000100540001005300000053A2
:101CF0000001005200010051000100500001004F9E
:101D00000001004E0000004E0001004D0001004C9B
:101D10000001004B0000004B0001004A0001004997
:101D20000001004800000048000100470001004693
:101D3000000000460001004500000045000100448D
:101D40000001004300000043000100420000004287
:101D50000001004100000041000100400001003F7F
:101D60000000003F0001003E0000003E0001003D79
:101D70000000003D0001003C0000003C0000003C71
:101D80000001003B0000003B0001003A0000003A67
:101D9000000100390000003900010038000000385F
:101DA0000000003800010037000000370001003655
:101DB000000000360000003600010035000000354C
:101DC0000000003500010034000000340000003441
:101DD0000001003300000033000000330001003236
:101DE000000000320000003200010031000000312C
:101DF0000000003100010030000000300000003021
:101E00000001002F0000002F0000002F0000002F15
:101E10000001002E0000002E0000002E0001002D09
:101E20000000002D0000002D0000002D0001002CFE
:101E30000000002C0000002C0000002C0001002BF2
:101E40000000002B0000002B0000002B0001002AE6
:101E50000000002A0000002A0000002A00010029DA
:101E600000000029000000290000002900000029CE
:101E700000010028000000280000002800000028C1
:101E800000000028000100270000002700000027B4
:101E900000000027000000270001002600000026A7
:101EA000000000260000002600000026000100259A
:101EB000000000250000002500000025000000258E
:101EC0000000002500010024000000240000002480
:101ED0000000002400000024000100230000002373
:101EE0000000002300000023000000230000002366
:101EF0000000002300010022000000220000002258
:101F00000000002200000022000000220001002149
:101F1000000000210000002100000021000000213D
:101F2000000000210000002100010020000000202E
:101F30000000002000000020000000200000002021
:101F400000000020000000200001001F0000001F12
:101F50000000001F0000001F0000001F0000001F05
:101F60000000001F0001001E0000001E0000001EF7
:101F70000000001E0000004D383420582059205A1F
:101F80002045006265640A002C2073797374656DC6
:101F90002073746F70706564212048656174657288
:101FA0005F49443A200048656174696E6720666144
:101FB000696C65640048656174696E672066616973
:101FC0006C65640048656174696E67206661696C60
:101FD00065640048656174696E67206661696C6557
:101FE000640070012C0190012701B0012201C001A1
:101FF0001D01F00118011002130130020E016002F0
:10200000090190020401C002FF000003FA0040032E
:10201000F5008003F000D003EB002004E60070041C
:10202000E100E004DC004005D700C005D200400616
:10203000CD00D006C8008007C3003008BE00F008FD
:10204000B900C009B400B00AAF00B00BAA00D00CB0
:10205000A500000EA000500F9B00C010960050126B
:10206000910000148C00C0158700B0178200B019D1
:102070007D00D01B7800001E730040206E0090226F
:102080006900F024640040275F0090295A00E02B8B
:102090005500102E500020304B0010324600E03327
:1020A000410090353C001037370070383200A039BD
:1020B0002D00B03A2800A03B2300603C1E00103DDC
:1020C0001900903D1400103E0F00703E0A00C03E03
:1020D0000500003F0000403FFBFF803FF6FFC03F90
:1020E000F1FF466C6F7700466C6F770046616E209B
:1020F00073706565640046616E2073706565640089
:1021000042656400426564004E6F7A7A6C65004EE9
:102110006F7A7A6C6500537065656400537065650D
:1021200064004D61696E005072656865617420508D
:102130004C412042656400507265686561742050AE
:102140004C4120456E640050726568656174205092
:102150004C4100507265706172650050726568652F
:102160006174204142532042656400507265686585
:1021700061742041425320456E6400507265686569
:102180006174204142530050726570617265004D68
:1021900034323800507265686561742041425300E2
:1021A0005072656865617420504C4100436F6F6CDC
:1021B000646F776E004D38340044697361626C65FA
:1021C0002073746570706572730053657420686F56
:1021D0006D65206F66667365747300473238004121
:1021E00075746F20686F6D65004D6F76652061783E
:1021F0006973004D61696E004D6F76652058004D22
:102200006F76652059004D6F7665205A00457874C9
:102210007275646572004D6F766520302E316D6D7C
:10222000004D6F766520316D6D004D6F7665203104
:10223000306D6D004D6F766520617869730045786B
:10224000747275646572004D6F7665205A004D6F2B
:1022500076652059004D6F766520580020204D3856
:102260003531205A005A2D50726F6265204F6666D4
:1022700073657420286D6D293A0A002044002049B6
:102280000020204D333031205000504944207365E8
:102290007474696E67733A0A002046002042002079
:1022A000480020204D3134352053004D6174657253
:1022B00069616C2068656174757020706172616D10
:1022C00065746572733A0A00205A00205900202074
:1022D0004D323036205800486F6D65206F6666734A
:1022E00065743A0A00204500205A00205900205801
:1022F0000020420020540020204D32303520530071
:10230000416476616E6365643A20533C6D696E5F2B
:1023100066656564726174653E20543C6D696E5FEC
:1023200074726176656C5F66656564726174653E42
:1023300020423C6D696E5F7365676D656E745F7496
:10234000696D655F6D733E20583C6D61785F78798B
:102350005F6A65726B3E205A3C6D61785F7A5F6A96
:1023600065726B3E20453C6D61785F655F6A6572A2
:102370006B3E0A0020540020520020204D323034A1
:10238000205000416363656C65726174696F6E20F3
:1023900028756E6974732F7332293A20503C70721D
:1023A000696E745F616363656C3E20523C72657454
:1023B000726163745F616363656C3E20543C747248
:1023C0006176656C5F616363656C3E0A0020450061
:1023D000205A0020590020204D3230312058004D25
:1023E0006178696D756D20416363656C65726174B8
:1023F000696F6E2028756E6974732F7332293A0ADB
:1024000000204500205A0020590020204D32303352
:102410002058004D6178696D756D20666565647240
:10242000617465732028756E6974732F73293A0A75
:1024300000204500205A0020590020204D3932202C
:10244000580053746570732070657220756E6974DE
:102450003A0A0020204D3230302044300A0020203B
:102460004D3230302044002044697361626C6564F1
:102470000A0046696C616D656E74207365747469D9
:102480006E67733A002020473231203B20556E6939
:10249000747320696E206D6D0A0A007A5F6D696E33
:1024A0003A2000795F6D696E3A2000785F6D696E41
:1024B0003A20005265706F7274696E6720656E64B1
:1024C00073746F70207374617475730A007C3C3E82
:1024D0005E2B3D3F2F5B5D3B2C2A225C00457874D0
:1024E0007275646572004D6F7665205A004D6F7687
:1024F000652059004D6F76652058005072657061F7
:10250000726500526573746F7265206661696C73E1
:102510006166650046696C616D656E74004D6F742F
:10252000696F6E0054656D706572617475726500D7
:102530004D61696E00507265686561742041425357
:1025400020636F6E66005072656865617420504C40
:102550004120636F6E66005049442D440050494449
:102560002D44005049442D49005049442D49005004
:1025700049442D50005049442D5000200820466108
:1025800063740020082046616374002008204D61B8
:1025900078002008204D6178002008204D617800E7
:1025A0002008204D696E002008204D696E0020082B
:1025B000204D696E004F6666004F6E2000417574B5
:1025C0006F74656D700046616E20737065656400A0
:1025D00046616E2073706565640042656400426503
:1025E00064004E6F7A7A6C65004E6F7A7A6C650083
:1025F000436F6E74726F6C004265640042656400E4
:102600004E6F7A7A6C65004E6F7A7A6C650046611F
:102610006E2073706565640046616E207370656539
:10262000640054656D706572617475726500534421
:102630002063617264206F6B0A006F70656E526F69
:102640006F74206661696C65640A00766F6C756DE5
:10265000652E696E6974206661696C65640A005351
:102660004420696E6974206661696C0A0061757442
:102670006F25692E67004D3234004D3233202573AB
:102680000057726974696E6720746F2066696C65A3
:102690003A20006F70656E206661696C65642C205D
:1026A00046696C653A20006F70656E206661696CE2
:1026B00065642C2046696C653A200046696C65208B
:1026C00073656C65637465640A002053697A653AC2
:1026D000200046696C65206F70656E65643A200065
:1026E0006F70656E206661696C65642C2046696C4C
:1026F000653A20002066696C653A20004E6F7720AD
:10270000002220706F73002220706172656E743A2F
:102710002200535542524F5554494E452043414C97
:102720004C207461726765743A22004B494C4C45E9
:10273000442E2000747279696E6720746F20636183
:102740006C6C207375622D67636F64652066696CBD
:102750006573207769746820746F6F206D616E797E
:10276000206C6576656C732E204D4158206C657623
:10277000656C2069733A004572726F723A006F6B34
:1027800000627573793A2070617573656420666FB5
:102790007220696E7075740A00627573793A2070E0
:1027A000617573656420666F7220757365720A00C7
:1027B000627573793A2070726F63657373696E67BF
:1027C0000A004B494C4C45442E20004B494C4C20B0
:1027D000636175736564206279204B494C4C2062BB
:1027E0007574746F6E2F70696E0A004B494C4C45BE
:1027F000442E20004B494C4C206361757365642066
:10280000627920746F6F206D75636820696E6163F3
:10281000746976652074696D65202D206375727208
:10282000656E7420636F6D6D616E643A2000506C4C
:1028300065617365207265736574005052494E542A
:1028400045522048414C544544005072696E7465AD
:10285000722068616C7465642E206B696C6C282929
:102860002063616C6C6564210A00656E7175657525
:1028700065696E6720220000000000000000000073
:102880000000005761726E696E673A20486F6D698B
:102890006E672042756D702044697669736F72208F
:1028A0003C20310A000000A0400000A040000000D1
:1028B00040000096430000964300009643FFFFFF50
:1028C0004E6F204C696E65204E756D626572207783
:1028D00069746820636865636B73756D2C204C6147
:1028E0007374204C696E653A20004B494C4C45444A
:1028F0002E200053544F505045442E2000507269F2
:102900006E7465722073746F707065642064756591
:1029100020746F206572726F72732E204669782062
:10292000746865206572726F7220616E64207573C1
:1029300065204D39393920746F2072657374617266
:10294000742E202854656D706572617475726520EF
:1029500069732072657365742E20536574206974E1
:102960002061667465722072657374617274696E39
:1029700067290A004E6F20436865636B73756D208D
:1029800077697468206C696E65206E756D6265721A
:102990002C204C617374204C696E653A200063688A
:1029A00065636B73756D206D69736D617463682CFD
:1029B000204C617374204C696E653A20004C696E3E
:1029C00065204E756D626572206973206E6F74208C
:1029D0004C617374204C696E65204E756D62657232
:1029E0002B312C204C617374204C696E653A2000A9
:1029F0004D313130004D3331004D3834205820599D
:102A0000205A20450053442072656164206572722B
:102A10006F720A00446F6E65207072696E74696E21
:102A2000672066696C650A0020496E76616C69648E
:102A3000206578747275646572200000009643000A
:102A400000964300009643000000000000000000D4
:102A5000000000205A3A200020593A2000426564C4
:102A600020583A200020746F6F206C6F6E672065CD
:102A70007874727573696F6E2070726576656E74A6
:102A800065640A0020636F6C6420657874727573E6
:102A9000696F6E2070726576656E7465640A0020D9
:102AA000706F736974696F6E206F7574206F662024
:102AB00072616E67652E0A003F50726F626520007A
:102AC0004E6F206D6F76652E00486F6D6520257303
:102AD00025732573206669727374002066697273AA
:102AE000740A005A0059005800486F6D6520005361
:102AF00074616E6461726420446576696174696FA3
:102B00006E3A20002052616E67653A2000204D61C8
:102B1000783A2000204D696E3A20004D65616E3A8A
:102B2000200046696E697368656421002072616ED9
:102B300067653A2000206D61783A2000206D696E4B
:102B40003A2000207369676D613A2000206D65614D
:102B50006E3A20003A207A3A2000206F662000204A
:102B60005A00205900205800476F696E6720746F23
:102B70003A00436C6F636B776973650A00436F7546
:102B80006E7465722D0020446972656374696F6E9E
:102B90003A2000202020616E676C653A2000537453
:102BA000617274696E67207261646975733A20009E
:102BB000506F736974696F6E696E67207468652001
:102BC00070726F62652E2E2E0A003F4E756D626523
:102BD00072206F66206C65677320696E206D6F765A
:102BE000656D656E74206E6F7420706C61757369AD
:102BF000626C652028302D3135292E0A0059005885
:102C0000003F53616D706C652073697A65206E6F4B
:102C10007420706C61757369626C652028342D3581
:102C200030292E0A004D3438205A2D50726F6265BB
:102C3000205265706561746162696C6974792054B1
:102C40006573740A003F566572626F7365204C6548
:102C500076656C206E6F7420706C61757369626C40
:102C6000652028302D34292E0A0043616E6E6F7462
:102C7000206F70656E2073756264697220006563F1
:102C8000686F3A0046696C2E204469612E004669DF
:102C90006C2E204469612E004F6666004F6E200046
:102CA0004520696E206D6D3300436F6E74726F6CDA
:102CB0000043616E6E6F7420656E7465722073756B
:102CC000626469723A2000022E2E004D61696E0026
:102CD00048617264636F6465642044656661756C05
:102CE000742053657474696E6773204C6F616465FA
:102CF000640A004573746570732F6D6D00457374BD
:102D00006570732F6D6D005A73746570732F6D6DE0
:102D1000005A73746570732F6D6D0059737465700C
:102D2000732F6D6D005973746570732F6D6D00583E
:102D300073746570732F6D6D005873746570732FA5
:102D40006D6D00412D74726176656C00412D747259
:102D50006176656C00412D72657472616374004127
:102D60002D7265747261637400416D617820450055
:102D7000416D6178204500416D6178205A00416DB8
:102D80006178205A00416D6178205900416D617869
:102D9000205900416D6178205800416D61782058BC
:102DA000005654726176206D696E005654726176D9
:102DB000206D696E005654726176206D696E005602
:102DC0006D696E00566D696E00566D696E00566DC8
:102DD0006178204500566D6178204500566D617818
:102DE000204500566D6178205A00566D6178205A52
:102DF00000566D6178205A00566D61782059005652
:102E00006D6178205900566D6178205900566D61CA
:102E100078205800566D6178205800566D617820F2
:102E2000580056652D6A65726B0056652D6A65728D
:102E30006B0056652D6A65726B00567A2D6A657255
:102E40006B00567A2D6A65726B0056792D6A657231
:102E50006B0056792D6A65726B0056792D6A657222
:102E60006B0056782D6A65726B0056782D6A657214
:102E70006B0056782D6A65726B00416363656C0068
:102E8000416363656C005A204F6666736574005A2F
:102E9000204F666673657400436F6E74726F6C00CA
:102EA00020746F6F206C6F6E672065787472757315
:102EB000696F6E2070726576656E7465640A0020B5
:102EC000636F6C6420657874727573696F6E2070BF
:102ED000726576656E7465640A001000C90210019F
:102EE0002C014001220170011801B0010E01F00116
:102EF00004015002FA00B002F0003003E600D003F3
:102F0000DC009004D2007005C800A006BE000008D6
:102F1000B400B009AA00D00BA000600E96006011AA
:102F20008C000015820020197800C01D6E00A022C0
:102F30006400B0275A00902C500000314600E03465
:102F40003C0010383200903A2800603C1E00A03D42
:102F50001400803E0A00203F0000544845524D4175
:102F60004C2052554E4157415900546865726D616D
:102F70006C2052756E61776179004572723A204D0E
:102F8000494E54454D5020424544004572723A2006
:102F90004D494E54454D50004D494E54454D5020DD
:102FA000747269676765726564004572723A204D94
:102FB000415854454D5020424544004572723A20D4
:102FC0004D415854454D50004D415854454D5020A9
:102FD000747269676765726564001FFFFFFFFFFF1A
:102FE000FF600000000001FF400000000000FF80C3
:102FF00000000000007F83CF00000C303F87FF807F
:10300000000C301F867980000C000F8C30C7838C39
:1030100030E78C30CFC7CC31F38C30DCECEC33B9FB
:103020008C30D86C6C33198C30D06C0C33198C30DC
:10303000D86C0C33198C30DC6C0E3B198C30CF7C87
:10304000079F198C30C77C038F19400000000000D7
:1030500002600000000000061FFFFFFFFFFFF800F6
:10306000600000000000600000E00000E0000001DF
:10307000F80000000001F80003F80003F800000762
:10308000FE0000000007FE000FFE000F1E00001FE4
:103090000F81C000381F0F803F0F803E0F80007CE3
:1030A00003E1C000387C03E0FC03E0F803E000F03B
:1030B00000F1C00038F000F1F000F1E000F000C0D5
:1030C0000071C00038C00071C00071C0007000C045
:1030D0000001C00038C003E1C00031C0003000C0B2
:1030E0000001C00038C00F81C00031C0003000C0F6
:1030F0000001FFFFF8C07E01FFFC31C0003000C0BE
:103100000001FFFFF8C1F001FFFC31C0003000C03A
:103110000001FFFFF8C7C001FFFC31C0003000C054
:103120000001C00038FF0001C00031C0003000C005
:103130000001C00038FC0001C00031C0003000C0F8
:103140000031C00038E00031C00031C0003000E084
:1031500000F1C00038E000F1C00031C00070007C18
:1031600003E1C000387C03E1C00031F001E0001F42
:103170000F81C000381F0F81C00031FC07C000075D
:10318000FE0000000007FE00000001CF0F0000015C
:10319000F80000000001F800000001C3FC0000007E
:1031A0006000000000006000000001C0F0000000AE
:1031B00000000000000000000000000060000000AF
:1031C00000000000000000000000000000000000FF
:1031D00000000000000000000000000000000000EF
:1031E000000000000000000000000E00001F0300AF
:1031F000000000000000000000003F80007FC300CE
:1032000000000000000000000000FFE001FBF300F0
:1032100000000000000000000003E0F807E0FF00ED
:103220000000000000000000000F803E1F8E3F00E5
:103230000000000000000000000E001F9E3F8F00F5
:1032400000000000000000000000001F98FFE300E5
:1032500000000000000000000000007E19FFF300E5
:103260000000000000000000000001F819FFF3005A
:10327000000000000000000000000FE019FFF30054
:10328000000000000000000000001F8019FFF30094
:103290000000000000000000000007E019FFF3003C
:1032A0000000000000000000000001FC19FFF30016
:1032B00000000000000000000000003F19FFF300C4
:1032C0000000000000000000000C000F9C7FC70001
:1032D0000000000000000000000F001F9F1F1F00E3
:1032E0000000000000000000000FC07E0FC07E0044
:1032F00000000000000000000003F1F803F1F800F6
:1033000000000000000000000000FFE000FFE000FF
:10331000000000000000000000003F80003F80002F
:10332000000000000000000000000E00000E000081
:10333000000000000000000000000000000000008D
:10334000000000000000000000000000000000007D
:10335000000000000000000000000000000000006D
:10336000000000000000000000000000000000005D
:105050000000000000000000000000000000002030
:1050600042403A0020403A00202F0020423A0020DF
:105070002F0020543A004D31343520533C696E6482
:1050800065783E206F7574206F662072616E67656B
:105090002028302D31290A00205A3A0020593A00A0
:1050A00020436F756E7420583A0020453A00205A0C
:1050B0003A0020593A00583A00526573656E643AD6
:1050C00020009DDE66DE11241FBECFEFD1E2DEBFE1
:1050D000CDBF00E00CBF14E0A0E0B2E0E8ECFBEDD7
:1050E00001E00BBF02C007900D92A235B107D9F7BE
:1050F00024E1A2E5B4E001C01D92AB36B207E1F7AE
:1051000018E2C2E6D8E200E006C021970109802F2C
:10511000FE010E944DEDC136D10780E00807A9F7D6
:105120000E9404DA0C94D3ED0C9400002F923F926D
:105130004F925F926F927F928F929F92AF92BF92A7
:10514000CF92DF92EF92FF920F931F93CF93DF9353
:10515000CDB7DEB7CF58D1090FB6F894DEBF0FBE7A
:10516000CDBF80916D0620E6829FC001112483513E
:105170009B4F9093620C8093610C80911B1380FF76
:105180001BC0EEE7FCE284918F010F5F1F4F882365
:1051900021F00E94008FF801F6CF0091610C109170
:1051A000620CD8018D918D01882319F00E94008F27
:1051B000F8CF8AE00E94008FE091610CF091620CC0
:1051C0008081803231F43196F093620CE093610C6F
:1051D000F3CF8E3469F01091610C0091620C6AE299
:1051E00070E0812F902F0E949BED009721F52AC03F
:1051F000818190ED980F9A3010F08D3261F73296E0
:10520000F093620CE093610CE091610CF091620C00
:10521000808180538A3010F43196F2CFE091610C96
:10522000F091620C80818032B1F63196F093620C7D
:10523000E093610CF3CFFC0131968291803231F022
:105240008A3221F0A12FB02F9D9102C01082F5CF9C
:10525000FD01808111968032D9F380538A3020F08D
:10526000EEE7FCE20C94A141E12CF12C2AE02E9D0A
:10527000B0012F9D700D11247B01B0E3EB1AF108F2
:105280008191E80EF11C87FDFA94808180538A3069
:1052900070F38F013196D8018C918032D1F3109345
:1052A0005D0400935C0421E030E03093600C2093B7
:1052B0005F0C9D3409F4DAC7943511F40C9437412E
:1052C000973411F00C944F41B4E0EB16F10409F45B
:1052D00087C540F4F2E0EF16F10410F50E94F2A346
:1052E0000C9498412AE5E216F10409F4FDC660F435
:1052F0004CE1E416F10409F4B1C55EE1E516F104F0
:1053000009F42DC60C9498418BE5E816F10409F4D4
:10531000EFC69CE5E916F10409F4EFC60C94984138
:1053200080911602882311F40C94984111E0A2E0B8
:10533000EA16F10409F010E00E94919A82E50E94B9
:10534000A699882309F452C10E94689A6B017C01D6
:105350004090BC045090BD046090BE047090BF04A7
:105360002091C0043091C1044091C2045091C30403
:105370002BAF3CAF4DAF5EAF8091830C9091840C0E
:10538000A091850CB091860C23968CAF9DAFAEAFEB
:10539000BFAF23972091870C3091880C4091890CE6
:1053A00050918A0C2B962CAF3DAF4EAF5FAF2B9731
:1053B00020E030E0A901C701B6010E943FE6882342
:1053C00009F4F4C4A301920123966CAD7DAD8EADBA
:1053D0009FAD23970E943FE681110FC02BAD3CADDE
:1053E0004DAD5EAD2B966CAD7DAD8EAD9FAD2B976B
:1053F0000E943FE6882309F4D9C420E030E0A901E7
:10540000C701B6010E943FE6881F8827881F18132E
:105410000BC080E090E0A0E8BFE367968CAF9DAF43
:10542000AEAFBFAF67970AC020E030E040E85FEB67
:1054300067962CAF3DAF4EAF5FAF6797A301920168
:1054400023966CAD7DAD8EAD9FAD23970E9461EA32
:105450002F966CAF7DAF8EAF9FAF2F972BAD3CAD2E
:105460004DAD5EAD2B966CAD7DAD8EAD9FAD2B97EA
:105470000E9461EA63966CAF7DAF8EAF9FAF63977A
:105480002F962CAD3DAD4EAD5FAD2F97CA01B90142
:105490000E94A4E64B015C0163962CAD3DAD4EAD80
:1054A0005FAD6397CA01B9010E94A4E69B01AC01FC
:1054B000C501B4010E9462EA0E94CDEC27966CAF50
:1054C0007DAF8EAF9FAF279720E030E040E05FE3F5
:1054D0000E94A4E64B015C01A7019601C701B60139
:1054E0000E94A4E66B017C01A5019401C501B401F1
:1054F0000E94A4E69B01AC01C701B6010E9461EACB
:105500000E94CDEC9B01AC0167966CAD7DAD8EAD7C
:105510009FAD67970E94A4E64B015C0123962CADDA
:105520003DAD4EAD5FAD2397C301B2010E9462EA6B
:1055300020E030E040E05FE30E94A4E66B017C01E4
:1055400063966CAD7DAD8EAD9FAD639790582796F9
:105550002CAD3DAD4EAD5FAD27970E943EEB9B015C
:10556000AC01C501B4010E94A4E69B01AC01C701D6
:10557000B6010E9462EAA30192010E9461EA6B01F6
:105580007C012B962CAD3DAD4EAD5FAD2B976BAD39
:105590007CAD8DAD9EAD0E9462EA20E030E040E03F
:1055A0005FE30E94A4E62B013C0127962CAD3DADA4
:1055B0004EAD5FAD27972F966CAD7DAD8EAD9FAD97
:1055C0002F970E943EEB9B01AC01C501B4010E94E4
:1055D000A4E69B01AC01C301B2010E9462EA2BADBB
:1055E0003CAD4DAD5EAD0E9461EA14C089E40E94FD
:1055F000A699882329F00E94689A6B017C0103C058
:10560000C12CD12C76018AE40E94A6998823F9F056
:105610000E94689A2B966CAF7DAF8EAF9FAF2B9791
:1056200020E030E0A901C701B6010E943FE68111E8
:105630001EC020E030E0A9012B966CAD7DAD8EAD93
:105640009FAD2B970E943FE6811111C0AFC320E0B0
:1056500030E0A901C701B6010E943FE6882309F4A2
:10566000A5C32B961CAE1DAE1EAE1FAE2B97D70149
:10567000C601B0588BAF9CAFADAFBEAF2B962CAD73
:105680003DAD4EAD5FAD2B97505823962CAF3DAF3F
:105690004EAF5FAF23979C01AD01BC01CD010E94CD
:1056A000A4E64B015C0123962CAD3DAD4EAD5FAD44
:1056B0002397CA01B9010E94A4E69B01AC01C50170
:1056C000B4010E9462EA0E94CDECA7966CAF7DAF58
:1056D0008EAF9FAFA7978091BC049091BD04A0911D
:1056E000BE04B091BF0427968CAF9DAFAEAFBFAFE5
:1056F0002797A7019601BC01CD010E9462EA679637
:105700006CAF7DAF8EAF9FAF67972091C004309193
:10571000C1044091C2045091C3042F962CAF3DAFF9
:105720004EAF5FAF2F972B962CAD3DAD4EAD5FAD1D
:105730002B972F966CAD7DAD8EAD9FAD2F970E94B0
:1057400062EA6B966CAF7DAF8EAF9FAF6B97809127
:10575000830C9091840CA091850CB091860C6F966F
:105760008CAF9DAFAEAFBFAF6F9767962CAD3DAD21
:105770004EAD5FAD6797BC01CD010E9461EA6B0140
:105780007C012091870C3091880C4091890C5091BC
:105790008A0CA3962CAF3DAF4EAF5FAFA3976B962D
:1057A0002CAD3DAD4EAD5FAD6B97A3966CAD7DADB1
:1057B0008EAD9FADA3970E9461EA4B015C01809181
:1057C000C4049091C504A091C604B091C704AF96DB
:1057D0008CAF9DAFAEAFBFAFAF979C01AD016091F5
:1057E0008B0C70918C0C80918D0C90918E0C0E9482
:1057F00061EA63966CAF7DAF8EAF9FAF63972091E8
:105800008F0C3091900C4091910C5091920CAB9672
:105810002CAF3DAF4EAF5FAFAB978091C804909176
:10582000C904A091CA04B091CB04E3968CAF9DAF9C
:10583000AEAFBFAFE397A70196016BAD7CAD8DAD69
:105840009EAD0E94A4E62B013C01A5019401239684
:105850006CAD7DAD8EAD9FAD23970E94A4E69B01FC
:10586000AC01C301B2010E9462EA2B013C01A50117
:1058700094016BAD7CAD8DAD9EAD0E94A4E64B0155
:105880005C01A701960123966CAD7DAD8EAD9FADF9
:1058900023970E94A4E69B01AC01C501B4010E94BC
:1058A00061EAA30192010E94D5EA6B017C0120E02C
:1058B00030E0A9010E943FE687FF0AC02BED3FE0E0
:1058C00049EC50E4C701B6010E9462EA6B017C0119
:1058D000112351F02BED3FE049EC50E4C701B60134
:1058E0000E9461EA6B017C0120E030E0A901C70160
:1058F000B6010E943FE681112AC06F962CAD3DADE6
:105900004EAD5FAD6F9727966CAD7DAD8EAD9FAD03
:1059100027970E943FE681111AC0A3962CAD3DAD9A
:105920004EAD5FADA3972F966CAD7DAD8EAD9FADA7
:105930002F970E943FE681110AC02BED3FE049EC12
:1059400050E4C701B6010E9462EA6B017C01A79690
:105950002CAD3DAD4EAD5FADA797C701B6010E941E
:10596000A4E69B01AC010E94A4E64B015C01639696
:105970002CAD3DAD4EAD5FAD6397CA01B9010E943C
:10598000A4E69B01AC01C501B4010E9462EA0E9439
:10599000CDEC4B015C012FE632E143E85AE30E9473
:1059A0003FE687FDFFC1C501B4010E94D7EB0E940D
:1059B000ABEB2D967FAF6EAF2D97DB01AB2B31F4A8
:1059C000E1E0F0E02D96FFAFEEAF2D972D962EADD6
:1059D0003FAD2D97B90180E090E00E9443E64B0176
:1059E0005C019B01AC01C701B6010E943EEB27960A
:1059F0006CAF7DAF8EAF9FAF2797A50194016396E3
:105A00006CAD7DAD8EAD9FAD63970E943EEBA796CA
:105A10006CAF7DAF8EAF9FAFA797E3962CAD3DAD3A
:105A20004EAD5FADE397AB966CAD7DAD8EAD9FADEA
:105A3000AB970E9461EAA50194010E943EEBAB96F0
:105A40006CAF7DAF8EAF9FAFAB9727962CAD3DADC2
:105A50004EAD5FAD2797CA01B9010E94A4E620E0D0
:105A600030E040E05FE30E94A4E69B01AC0160E00F
:105A700070E080E89FE30E9461EA63966CAF7DAFBF
:105A80008EAF9FAF6397AF968CAD9DADAEADBFAD02
:105A9000AF9789879A87AB87BC87E3962CAD3DADDE
:105AA0004EAD5FADE3972D873E874F87588B609152
:105AB000190270911A02072E000C880B990B0E9494
:105AC00045E620910002309101024091020250917E
:105AD00003020E94A4E62AE037ED43E25CE30E9461
:105AE000A4E66F966CAF7DAF8EAF9FAF6F970E94AD
:105AF000E7509B01AC0128533F4F4F4F5F4FA39698
:105B00002CAF3DAF4EAF5FAFA3974BAC5CAC6DAC71
:105B10007EAC22242394312CD12C2D968EAD9FADBA
:105B20002D972816390609F429C10E94065C0E94A7
:105B3000E750DC01CB01A3962CAD3DAD4EAD5FAD82
:105B4000A397821B930BA40BB50BB7FD10C00E944B
:105B5000E7509B01AC0128533F4F4F4F5F4FA39637
:105B60002CAF3DAF4EAF5FAFA3970E94BD92D394D1
:105B700038E13D150CF44BC063962CAD3DAD4EADF8
:105B80005FAD639723966CAD7DAD8EAD9FAD2397D2
:105B90000E94A4E64B015C0127962CAD3DAD4EADB5
:105BA0005FAD2797B201C3010E94A4E6A50194014D
:105BB0000E9462EA7B018C0163962CAD3DAD4EAD37
:105BC0005FAD6397B201C3010E94A4E64B015C0183
:105BD00027962CAD3DAD4EAD5FAD279723966CADAE
:105BE0007DAD8EAD9FAD23970E94A4E69B01AC01D5
:105BF000C501B4010E9461EA2B013C01C701D80133
:105C000023968CAF9DAFAEAFBFAF239756C0B10107
:105C100080E090E00E9443E627962CAD3DAD4EAD6E
:105C20005FAD27970E94A4E64B015C010E943BEB0D
:105C30006B017C01C501B4010E94C3EC4B015C0106
:105C4000A70196016BAD7CAD8DAD9EAD0E94A4E623
:105C50002B013C01A50194012B966CAD7DAD8EAD61
:105C60009FAD2B970E94A4E69B01AC01C301B2013A
:105C70000E9462EA2B013C01A50194016BAD7CAD51
:105C80008DAD9EAD0E94A4E64B015C01A70196017B
:105C90002B966CAD7DAD8EAD9FAD2B970E94A4E68B
:105CA0009B01AC01C501B4010E9461EA23966CAF6F
:105CB0007DAF8EAF9FAF2397D12C9201A301679642
:105CC0006CAD7DAD8EAD9FAD67970E9462EA698332
:105CD0007A838B839C8323962CAD3DAD4EAD5FAD17
:105CE00023976B966CAD7DAD8EAD9FAD6B970E948B
:105CF00062EA6D837E838F839887A7962CAD3DAD36
:105D00004EAD5FADA79769857A858B859C850E948E
:105D100062EA69877A878B879C87AB962CAD3DAD0D
:105D20004EAD5FADAB976D857E858F8598890E945E
:105D300062EA6D877E878F87988B80912702882300
:105D400021F0CE0101960E943E90C09056046F96BD
:105D5000ECACFDAC0EAD1FAD6F979E01235F3F4FC6
:105D6000AE01475F5F4FBE016B5F7F4FCE01019673
:105D70000E943BBD4FEF241A340ACFCEC090560488
:105D80006F96ECACFDAC0EAD1FAD6F972FE83CE00D
:105D90004BE85CE067E87CE083E89CE00E943BBD68
:105DA0000E942F990E94AB710C949841E7E7F7E2AB
:105DB00084918F010F5F1F4F882321F00E94008F75
:105DC000F801F6CFE9EDF1E084918F010F5F1F4FED
:105DD000882311F40C9498410E94008FF801F4CFAD
:105DE00080E50E94A699882329F00E945D9A6B01A4
:105DF0007C0103C0C12CD12C760183E50E94A699B9
:105E0000882321F00E94009B6B017C010E949B5D16
:105E10000E94AB718091630C9091640CA091650C11
:105E2000B091660CC80ED91EEA1EFB1E8091460278
:105E3000811105C060E08FEE91E00E9488560E94BB
:105E4000E750DC01CB018C199D09AE09BF09B7FDF4
:105E500002C00C9498410E94BD92F1CF0E949B5DBC
:105E60000E94FB9581E080930B0288E50E94A69931
:105E7000E82E89E50E94A699082F8AE50E94A69936
:105E8000F82EE11005C0011105C011E0182705C06A
:105E9000011102C010E001C0182F80E1ECEBF4E02A
:105EA000A3E8BCE001900D928A95E1F7111105C0BD
:105EB000E11003C0002309F440C020E030E040EAD4
:105EC00050E46091730C7091740C8091750C9091FA
:105ED000760C0E9462EA60938B0C70938C0C80931A
:105EE0008D0C90938E0C2091C4043091C504409188
:105EF000C6045091C7040E9488EC18165CF41982FD
:105F00001A821B821C82BE016F5F7F4F8BE89CE070
:105F10000E94FC96111105C0E11003C0011107C0D9
:105F20000CC080E090E00E94D0901123B9F381E092
:105F300090E00E94D090111102C0FF2021F082E079
:105F400090E00E94D0900E949B71809154048093B5
:105F50000B020E94E1950E9408D60C94984188E5B6
:105F60000E94A699882319F00E94689A0EC020E02A
:105F700030E040E251E46091BC047091BD04809136
:105F8000BE049091BF040E9462EA4B015C0189E566
:105F90000E94A699882319F00E94689A0EC020E0FA
:105FA00030E040E251E46091C0047091C1048091FE
:105FB000C2049091C3040E9462EA2B013C0120912B
:105FC000730C3091740C4091750C5091760C2BAF82
:105FD0003CAF4DAF5EAF20916B0C30916C0C40919B
:105FE0006D0C50916E0CC501B4010E9461EA2091C4
:105FF0006F0C3091700C4091710C5091720C239683
:106000002CAF3DAF4EAF5FAF239720E030E040E2D2
:1060100051E40E9461EA6B017C0127E137EB41ED1D
:1060200058EB0E9488EC87FF02C00C94984123E053
:1060300030E046E953E4C701B6010E943FE6181676
:1060400014F40C94984123962CAD3DAD4EAD5FAD4C
:106050002397C301B2010E9461EA20E030E040E2F0
:1060600051E40E9461EA6B017C0127E137EB41EDCD
:1060700058EB0E9488EC87FF02C00C94984123E003
:1060800030E046E953E4C701B6010E943FE6181626
:1060900014F40C94984120E030E0A9016BAD7CAD84
:1060A0008DAD9EAD0E9462EA2BAD3CAD4DAD5EADB7
:1060B0000E9461EA6B017C0127E137EB41ED58EB6F
:1060C0000E9488EC87FF02C00C94984123E030E0E6
:1060D00046E953E4C701B6010E943FE6181614F4DE
:1060E0000C9498410C94514110925B040C9498418B
:1060F00081E080935B040C94994185E40E94A69909
:10610000B82E811102C00E949B5D00EB802E02E040
:10611000902E8CEBC82E84E0D82E97E7E92E9CE0D9
:10612000F92E00E010E0A12CD4018D914D010E94C8
:10613000A699882309F44EC0F6012081318142815D
:106140005381C457DF4F2883CC58D040C357DF4F0B
:106150003883CD58D040C257DF4F4883CE58D04007
:10616000C157DF4F5883CF58D0400E94689AD6015C
:106170006D937D938D939C931397C457DF4F288124
:10618000CC58D040C357DF4F3881CD58D040C2578C
:10619000DF4F4881CE58D040C157DF4F5881CF588C
:1061A000D04003301105B1F00E9461EA9B01AC01BF
:1061B000F70160817181828193810E9462EAD70137
:1061C0006D937D938D939C931397C8010E94529970
:1061D000AA24A3940F5F1F4FB4E0CB0ED11CE4E0C0
:1061E000EE0EF11C0430110509F09ECFAA2019F023
:1061F0000E949B7137C0BB20A9F1C090C804D09009
:10620000C904E090CA04F090CB042091C9123091E7
:10621000CA124091CB125091CC12C701B6010E9414
:10622000A4E60E9493EC6093F90F7093FA0F8093A9
:10623000FB0F9093FC0FC701B6010E94A6EB2FB78E
:10624000F89460939D0B70939E0B80939F0B90939B
:10625000A00B2FBF1092E90F1092EA0F1092EB0FD4
:106260001092EC0F0E9408D60C949841F1E7EF16BB
:10627000F10409F450C608F0D7C030E3E316F10486
:1062800009F433C508F068C058E1E516F10409F4D3
:1062900095C2B0F592E1E916F10409F42EC778F43D
:1062A000B2E0EB16F10408F4C2C1E1E1EE16F1042C
:1062B00011F00C9498410E94E1A30C949841F5E1EF
:1062C000EF16F10409F470C248F434E1E316F10466
:1062D00011F00C949841EFE4F2E023C246E1E41699
:1062E000F10409F465C257E1E516F10411F00C94CC
:1062F000984140E061E0C8010E9426870C949841D3
:106300008CE1E816F10409F4AEC268F4AAE1EA16D9
:10631000F10409F45EC208F06AC210922D100E94C6
:106320000C8C0C949841EFE1EE16F10409F4EFC3E4
:1063300038F42EE1E216F10409F49CC20C94984161
:1063400030E2E316F10409F498C34AE2E416F104DA
:1063500009F483C40C9498415CE5E516F10409F452
:106360000EC768F591E5E916F10409F4A6C6A0F494
:10637000BCE4EB16F10409F4BCC4EDE4EE16F10440
:1063800009F4BBC4FBE4EF16F10411F00C9498413E
:106390000E94CC8B0C94984123E5E216F10409F499
:1063A000A7C608F4A1C644E5E416F10409F4A5C69D
:1063B00055E5E516F10409F4CFC60C9498418CE636
:1063C000E816F10409F4A3C5C8F4A9E6EA16F10435
:1063D00009F4E4C538F4E8E6EE16F10409F491C4D2
:1063E0000C949841FAE6EF16F10409F42EC62BE658
:1063F000E216F10409F44FC60C9498413EE6E31608
:10640000F10409F4CFC408F4E6C55FE6E516F1042B
:1064100009F4DBC480E7E816F10411F00C9498410C
:1064200085E493E00E9455929DEDE916F10411F484
:106430000C946D3B08F065C0BEEBEB16F10409F45B
:10644000E8C578F5F7E7EF16F10409F435C798F4D5
:1064500033E7E316F10409F421C708F419C755E737
:10646000E516F10411F00C94984160E0C8010E9417
:106470009D560C94984189E7E816F10409F427C762
:1064800008F41EC7ACE8EA16F10409F470C5B1E9D6
:10649000EB16F10411F00C9498410E94C7D60C94AD
:1064A0009841ECECEE16F10409F456C7A0F429EC7F
:1064B000E216F10409F411C73BECE316F10409F408
:1064C0002EC748ECE416F10411F00C9498410E9498
:1064D000BBD50C9498415EECE516F10411F40C94D4
:1064E000813A08F4A3C793EDE916F10411F40C9472
:1064F000C83AACEDEA16F10411F40C94603B0C942C
:106500009841B2E9EB16B1E0FB0611F40C94A53FFB
:10651000F0F5FEE2EF16F1E0FF0611F40C94773C83
:1065200090F43CE2E31631E0F30611F40C94B23B34
:1065300010F00C94D83B52EEE516F10411F40C94D3
:10654000863B0C94984183E6E81681E0F80611F446
:106550000C940E4148F4AFE2EA16A1E0FA0611F4F9
:106560000C94EE3C0C949841B0E9EB16B1E0FB06BC
:1065700011F40C94A23FE1E9EE16E1E0FE0611F001
:106580000C94984181E00E946B970C949841F6EF2F
:10659000EF16F1E0FF0611F40C94C94040F53CEA17
:1065A000E31631E0F30611F40C94A93F58F45AE9CC
:1065B000E51651E0F50611F00C9498410E9484D53F
:1065C0000C94984184EFE81681E0F80611F40C94DD
:1065D000B04095EFE91691E0F90611F00C9498415E
:1065E0000E9482B280E00E94C7720C949841A3E599
:1065F000EA16A3E0FA0611F40C94D84048F4E7EF49
:10660000EE16E1E0FE0611F40C94CC400C94984197
:10661000F0EAEF16F3E0FF0609F475C227EEE21682
:1066200023E0F20611F40C9427410C94984180E584
:106630000E94A699882361F00E945D9A6B017C01FB
:10664000BB24B394672B682B692B31F4B12C04C0A5
:10665000B12CC12CD12C760183E50E94A699882308
:1066600099F00E94009B6B017C01B1100FC0672B59
:10667000682B692B59F4D8018C91882339F061E09B
:10668000C8010E949D5607C0BB20A9F360E08DE2BF
:1066900092E00E94885683E090E09093600C809393
:1066A0005F0C81E080939E060E949B5D0E94AB710F
:1066B000C114D104E104F104E9F08091630C9091DC
:1066C000640CA091650CB091660CC80ED91EEA1E30
:1066D000FB1E0E94E750DC01CB018C199D09AE091D
:1066E000BF09B7FF1AC080919E068823B1F00E94AF
:1066F000BD92EFCF80919E06882319F00E94BD9233
:10670000F9CF80912D1060E0882319F08EE192E09E
:1067100002C08AE092E00E94885610929E060C9475
:10672000984184918F010F5F1F4F882321F00E94B1
:10673000008FF801F6CF1092B3121092B21240E01F
:1067400050E0BA018EE590E10E94CE788BE1EEE553
:10675000F0E1DE01159601900D928A95E1F78091A6
:106760005C1090915D109C838B838EE293E09A8302
:10677000898340E050E0BE016F5F7F4F8FEE93E072
:106780000E9420A9CE0101960E9423B4E0E4F2E029
:1067900084918F010F5F1F4F882311F40C9498414F
:1067A0000E94008FF801F4CF0E943B8A0C9498411C
:1067B00010922D1010922E100C94984180912E1052
:1067C000882319F081E080932D100E94CC8B0C94CB
:1067D000984180912E10882311F40C94984183E500
:1067E0000E94A69981110C94BE410C94984180910D
:1067F0002E10882351F1E0E6F2E084918F010F5FC3
:106800001F4F882321F00E94008FF801F6CF60917E
:10681000A9127091AA128091AB129091AC124AE029
:106820000E94078F8FE20E94008F6091A5127091E5
:10683000A6128091A7129091A8124AE00E94078F99
:106840008AE00E94008F0C949841E2E7F2E0849184
:106850008F010F5F1F4F882311F40C9498410E9401
:10686000008FF801F4CF40E060E0C8010E94268765
:106870000C94984180912E10882311F40C94984127
:1068800088EF91E10E949C7888EF91E10E94E57E7B
:1068900010922C1010922B10E0905C04F0905D048C
:1068A00080912E10882311F40C9498410E94DC866C
:1068B000FE0131966F01CF010E9413B48AE590E189
:1068C00090937A1080937910D7018C918F3209F0D0
:1068D00060C06FE270E0C7010E949BED8C010F5F0A
:1068E0001F4F09F45CC06FE270E0C8010E949BED8D
:1068F0005C01009709F454C00817190708F050C04C
:106900004C01801A910AA401B801CE0180960E9420
:10691000C4EDE0E2F0E0EC0FFD1FE80DF91D108280
:106920008E01005E1F4FF80181918F01882319F0BD
:106930000E94008FF8CF8AE00E94008F609179104A
:1069400070917A106115710511F06C5F7F4F21E035
:10695000AE01405E5F4FCE0105960E94ED7E811133
:1069600012C0BE01605E7F4F89EA92E00E94847689
:106970008EE20E94008F8AE00E94008FC6010E9472
:1069800023B40C949841D0927A10C092791085016A
:10699000A6CF8BE790E190937A10809379108701CE
:1069A0006091791070917A106115710511F06C5F2A
:1069B0007F4F18A21BA222E0A801CE0180960E9460
:1069C000ED7E811102C0F12C14C0CE0180960E9490
:1069D0008EA88823C1F361E0CE0180960E94B5D1D4
:1069E000009789F325EEDC012C931BA20E94AC7664
:1069F000F82ECE0180960E941DB4FF2009F1E3E835
:106A0000F2E084917F01BFEFEB1AFB0A882321F0AB
:106A10000E94008FF701F5CFF80181918F01882343
:106A200019F00E94008FF8CF8AE00E94008F109228
:106A3000A9121092AA121092AB121092AC1218C0A6
:106A4000E1E9F2E084917F012FEFE21AF20A882354
:106A500021F00E94008FF701F5CFD8018D918D01B3
:106A6000882319F00E94008FF8CF8EE20E94008FD9
:106A7000C6010E9423B40C94984180912D1081117D
:106A80000E949B5D00915C0410915D0461E270E0E6
:106A9000C8010E949BED009719F08C010F5F1F4FFA
:106AA00080E50E94A699882349F0FF24F394809101
:106AB0005204909153048017910708F0F12C8091B3
:106AC0002E10882311F40C9498414F2D61E0C801D9
:106AD0000E94268783E50E94A699882349F0809129
:106AE0005204909153048017910710F40C94CF41F5
:106AF00080912E10882319F081E080932D10F110E1
:106B00000C94984162CE0E94D6A30C9498410E94A6
:106B100039A81CE3C12ED12CE12CF12CA701960140
:106B20000E9404EA762E672ECA01B901A7019601D8
:106B30000E9404EA6B017C01CA01B90128E130E03E
:106B400040E050E00E9404EA4B015C01C9016DE69F
:106B500071E00E9426ED8E010F5F1F4F61157105D8
:106B600099F06F927F92DF92CF929F928F929F9334
:106B70008F937F936F9385EE92E09F938F931F93F4
:106B80000F930E94D8E512C00097B1F06F927F92E8
:106B9000DF92CF929F928F929F938F9385ED92E099
:106BA0009F938F931F930F930E94D8E50FB6F8948D
:106BB000DEBF0FBECDBF36C081149104A104B10465
:106BC00079F06F927F92DF92CF929F928F9289ECB1
:106BD00092E09F938F931F930F930E94D8E5E6CF87
:106BE000C114D104E104F10469F06F927F92DF9245
:106BF000CF9281EC92E09F938F931F930F930E940B
:106C0000D8E5D4CF6F927F928DEB92E09F938F93D4
:106C10001F930F930E94D8E50F900F900F900F9045
:106C20000F900F9060E0C8010E949D56EEE7FCE2D5
:106C300084917F019FEFE91AF90A882321F00E94CD
:106C4000008FF701F5CFB80189EF92E00E948476BA
:106C50008AE00E94008F0C94984183E50E94A699D7
:106C6000882311F40C9498410E94509A7C018F3F24
:106C7000910519F010F00C94984180E50E94A699B6
:106C8000882339F00E94509A8C0197FF04C00C941D
:106C900098410DE010E0D02EE4EBF2E0C801992716
:106CA000219131912817390731F0B3E0E430FB0727
:106CB000B9F70C94E141E7E7F7E284918F010F5FA8
:106CC0001F4F882321F00E94008FF801F6CFE6E0E5
:106CD000F3E084918F010F5F1F4F882311F40C9410
:106CE00098410E94008FF801F4CF0E94EF9D0C9410
:106CF00098410E940C8C0C9498410E9420A80C94FE
:106D0000984188E690E00E94E89981110C9498419E
:106D100080911B1383FF02C00C94984183E50E946D
:106D2000A6998823D9F10E94509A9093890680935E
:106D3000880680E00E9453CE0E94509A86359105C5
:106D40003CF40E9420A860E08CE193E00E94885609
:106D50000E94509A8C0160915F0470916004809150
:106D60006104909162040E94A6EB60177107B4F46D
:106D700084E893E09F938F938091550490E001966F
:106D80009F938F9385E193E09F938F931F920E942F
:106D9000B18B0FB6F894DEBF0FBECDBF0E9436E1B7
:106DA0000C9498418EE40E94A699882311F40C94C7
:106DB00098410E9493DE60936114709362148093F3
:106DC0006314909364140C94984183E50E94A699EF
:106DD000882319F00E94B99901C080E080931B13A9
:106DE000EEE7FCE284918F010F5F1F4F882321F0B3
:106DF0000E94008FF801F6CFEEE3F3E084918F015B
:106E00000F5F1F4F882321F00E94008FF801F6CFFB
:106E100080911B138823A1F1B0E3CB2EB3E0DB2ECE
:106E2000E12CF12C20E080911B1390E00E2C02C08D
:106E3000959587950A94E2F780FF17C0BB24B39419
:106E4000B20E222319F08CE20E94008FF6012591E8
:106E50003491F901849189010F5F1F4F882321F03C
:106E60000E94008F9801F5CF2B2DFFEFEF1AFF0A3C
:106E700032E0C30ED11C45E0E416F104A1F642C095
:106E8000EAE3F3E084918F010F5F1F4F8823D1F174
:106E90000E94008FF801F6CF8AE50E94A699882308
:106EA00011F40C9400410E94689A6B017C0120E06F
:106EB00030E040EA51EC0E9488EC87FF02C00C945D
:106EC000F24020E030E040EA51E4C701B6010E9400
:106ED0003FE6181614F40C94F240C0921113D092AD
:106EE0001213E0921313F0921413C0928D02D092F9
:106EF0008E02E0928F02F092900242E0C701B6014A
:106F00000E94878F8AE00E94008F0C949841109213
:106F100004020C94984183E50E94A699882369F0A5
:106F20000E94B999809341028D3310F40C949841DA
:106F30008CE3809341020C949841EEE7FCE284914B
:106F40008F010F5F1F4F882321F00E94008FF801EF
:106F5000F6CF4091410250E060E070E08EE493E0B3
:106F60000E94BE648AE00E94008F0C949841809138
:106F70001B1383FF02C00C94984183E50E94A699DD
:106F8000882311F40C9498410E94509A90938D0696
:106F900080938C060E9420CE0C94984189E690E064
:106FA0000E94E899811111C0E5E5F3E084918F0119
:106FB0000F5F1F4F882321F00E94008FF801F6CF4A
:106FC0000E943CD78AE00E94008F1092600C1092C1
:106FD0005F0C0C94EA468DE690E00E94E8998111DE
:106FE0000C94984180911B1383FF02C00C9498412C
:106FF00083E50E94A69928968FAF289781110C945B
:10700000F64182E50E94A69981110C94F6410C94F8
:10701000984180911B1383FF02C00C94984160E05B
:1070200089E993E00E94885683E50E94A6992896F4
:107030008FAF289781110C94994382E50E94A699FD
:1070400081110C9499430C94984183E50E94A69970
:10705000882321F00E9487DE8C0102C00FEF10E030
:1070600080E50E94A699882319F00E9487DE02C05D
:1070700080E090E098010F3F110519F010F02FEF1C
:1070800030E0892B11F00C94984130938B062093BB
:107090008A060C94984180E50E94A699811106C049
:1070A00010928B0610928A060C9498410E9487DEFB
:1070B000892B11F00C949841F3CF0E9486CE0E9448
:1070C0009B5D0E94449210928B0610928A0668EE95
:1070D00073E080E090E00E94CE5560E086EA93E0A5
:1070E0000E9488560C94984110925A040C9498412E
:1070F00081E080935A040C94994183E50E94A699FB
:10710000882361F00E94009B6093420270934302C7
:1071100080934402909345020C94984188E50E9424
:10712000A69981110C940A4589E50E94A6998111BE
:107130000C940A458AE50E94A69981110C940A458F
:1071400085E40E94A69981110C940A450E949B5DDA
:107150000E9444920C94984183E50E94A69988234A
:1071600011F40C9498410E94009B6093670C7093FB
:10717000680C8093690C90936A0C0C94984150EBC6
:10718000C52E52E0D52E6DEBE62E62E1F62E10E014
:10719000D6018D916D010E94A699882309F46DC0D6
:1071A000133009F063C00E94689A4B015C0120E033
:1071B00030E040EA51E40E943FE687FF4EC0A5015F
:1071C00094016091C9127091CA128091CB12909172
:1071D000CC120E943EEB2B013C019B01AC01609163
:1071E000091370910A1380910B1390910C130E9454
:1071F000A4E66093091370930A1380930B13909382
:107200000C13A30192016091F9127091FA1280910E
:10721000FB129091FC120E94A4E66093F912709305
:10722000FA128093FB129093FC1260915D1470919E
:107230005E1480915F14909160140E9443E6A30154
:1072400092010E94A4E60E94ABEB60935D147093E0
:107250005E1480935F14909360148092C912909290
:10726000CA12A092CB12B092CC1207C00E94689AA8
:10727000F70160837183828393831F5FF4E0EF0ED5
:10728000F11C143009F084CF0E945AD50C94984117
:107290000E949B5D0E9408D60C949841E8EBF3E0B5
:1072A00084918F010F5F1F4F882311F40C94984134
:1072B0000E94008FF801F4CF0E9465720C949841EF
:1072C00081E080930B02809354040C9499411092B6
:1072D0000B02109254040C94984135EDE32E32E1E8
:1072E000F32E00EB12E044E0D42ED00ED8018D91A5
:1072F0008D010E94A699882349F00E94689A0E94F5
:10730000ABEBF7016083718382839383F4E0EF0E2C
:10731000F11CD012EBCF0E942DD40C9498419DEE1D
:10732000E92E92E1F92E00EB12E024E0D22ED00EED
:10733000D8018D918D010E94A699882339F00E9471
:10734000689AF7016083718382839383F4E0EF0E80
:10735000F11CD012EDCFECC783E50E94A6998823DB
:10736000D9F00E94689AAB01BC0140930D13509371
:107370000E1360930F13709310134093CD1250931C
:10738000CE126093CF127093D01280EF94E00E94DF
:10739000F8648AE00E94008F80E50E94A699882305
:1073A00099F00E94689AAB01BC0140930D13509371
:1073B0000E1360930F137093101383ED94E00E94EB
:1073C000F8648AE00E94008F82E50E94A6998823D3
:1073D00099F00E94689AAB01BC014093D11250937E
:1073E000D2126093D3127093D41284EB94E00E9473
:1073F000F8648AE00E94008F84E50E94A6998823A1
:1074000009F496C70E94689AAB01BC014093CD1263
:107410005093CE126093CF127093D01286E994E00D
:107420000E94F8648AE00E94008F82C783E50E9470
:10743000A699882351F00E94689A6093E91270938C
:10744000EA128093EB129093EC1284E50E94A699C5
:10745000882351F00E94689A6093E5127093E612B7
:107460008093E7129093E81282E40E94A699882301
:1074700051F00E945D9A60931713709318138093D4
:10748000191390931A1388E50E94A699882351F046
:107490000E94689A6093FD127093FE128093FF120F
:1074A0009093001389E50E94A699882351F00E94C9
:1074B000689A60930113709302138093031390935F
:1074C00004138AE50E94A699882351F00E94689AC5
:1074D000609305137093061380930713909308131A
:1074E00085E40E94A699882309F422C70E94689A1D
:1074F0006093091370930A1380930B1390930C13EA
:1075000017C710EBA12E12E0B12E0CEBC02E04E039
:10751000D02E80EBE82E84E0F82E00E010E0D501BC
:107520008D915D010E94A699882311F10E94689AAD
:107530002B013C01F70120813181428153810E945E
:1075400061EA9B01AC01D6016D917D918D919C9179
:107550000E9462EAF6016083718382839383D7017C
:107560004D925D926D927C921397C8010E94529940
:107570000F5F1F4FB4E0CB0ED11CE4E0EE0EF11C08
:107580000330110561F60E949B710E9408D6D0C697
:10759000EEE7FCE284918F010F5F1F4F882321F0FB
:1075A0000E94008FF801F6CF83E50E94A6998823F8
:1075B00021F00E94259A80932702E0E4F5E084916F
:1075C0008F010F5F1F4F882321F00E94008FF80169
:1075D000F6CF80912702811103C0ECE3F5E002C0F1
:1075E000E8E3F5E084918F010F5F1F4F882321F0BE
:1075F0000E94008FF801F6CFE0E3F5E084918F015F
:107600000F5F1F4F882321F00E94008FF801F6CFF3
:107610004091F10B5091F20B6091F30B7091F40BD0
:107620008EE295E00E94F8644091F50B5091F60BC4
:107630006091F70B7091F80B8BE295E00E94F86473
:107640004091F90B5091FA0B6091FB0B7091FC0B80
:1076500088E295E00E94F864E0E2F5E084918F0111
:107660000F5F1F4F882321F00E94008FF801F6CF93
:1076700040911B0250911C0260911D0270911E02EC
:107680008EE195E00E94F86440911F025091200223
:1076900060912102709122028BE195E00E94F864D2
:1076A000409123025091240260912502709126029C
:1076B00088E195E00E94F8648AE00E94008F38C655
:1076C00083E50E94A699882309F432C60E94509A45
:1076D00090931A02809319022BC68DED90E00E94C0
:1076E000E899811125C683E50E94A699882309F4AB
:1076F0001FC60091550410E00E94509A000F111F00
:10770000F801E95EFD4F9183808312C680E50E94F7
:10771000A699882309F40CC60E94509A8C0183E52F
:107720000E94A699882321F00E94509A7C0103C0F0
:10773000EE24EA94FE2CC7010196039708F0F8C5E1
:1077400017FDF6C5E4EBF2E0C801992721913191CC
:107750002817390709F4ECC523E0E430F207B1F744
:107760000C94C24683E50E94A699882319F00E94D2
:1077700087DE02C084E091E099A388A380E50E949F
:10778000A699882349F00E9487DE893833E1930760
:1077900028F088E893E102C088EE93E09A83898319
:1077A000BE01605E7F4FCE0101960E947D8BC0C5F9
:1077B00085E40E94A699811110C080E50E94A699D7
:1077C000882399F00E94689A609328027093290296
:1077D00080932A0290932B0208C00E94509A181698
:1077E00019065CF7E7E7F7E271C089E40E94A69901
:1077F000882381F00E94689A2CEA35EC47E25EE328
:107800000E94A4E6609330027093310280933202AA
:107810009093330284E40E94A699882381F00E9409
:10782000689A2CEA35EC47E25EE30E943EEB6093F7
:107830002C0270932D0280932E0290932F02EEE77C
:10784000FCE284918F010F5F1F4F882321F00E947B
:10785000008FF801F6CF40912802509129026091E3
:107860002A0270912B0288E595E00E94F8642CEAC8
:1078700035EC47E25EE36091300270913102809115
:107880003202909133020E943EEBAB01BC0184E5D1
:1078900095E00E94DB642CEA35EC47E25EE3609100
:1078A0002C0270912D0280912E0290912F020E9445
:1078B000A4E6AB01BC0180E595E00E94DB648AE0B0
:1078C0000E94008F35C50E94008FF80184918F01BE
:1078D0000F5F1F4F8111F7CF0FE813E0D8018D9193
:1078E0008D01882309F40ECB0E94008FF7CF83E52A
:1078F0000E94A699082F8823D1F00E94509ABC01BB
:10790000990F880B990B0E9445E660939102709342
:107910009202809393029093940211E020E030E071
:10792000A9010E943FE6811110E01093161380E533
:107930000E94A699182F8823A9F020E030E0A90121
:1079400060919102709192028091930290919402C1
:107950000E943FE6882319F00E94259A182F109361
:107960001613E6C40111E4C4EEE7FCE284918F0132
:107970000F5F1F4F882321F00E94008FF801F6CF80
:1079800080911613811103C060E873E002C062EFBA
:1079900073E081E795E00E94847620E030E040E0EB
:1079A0005FE36091910270919202809193029091B5
:1079B00094020E9462EA0E94A6EB80E695E00E9493
:1079C0006B76ECE5F5E084918F010F5F1F4F882304
:1079D00009F4AEC40E94008FF801F5CF85E40E943F
:1079E000A699882321F00E94509A8C0102C000E0E1
:1079F00010E083E40E94A699882349F00E94509ADF
:107A0000CA57DF4F99838883C658D04008C0E5E045
:107A1000F0E0CA57DF4FF983E883C658D04085E5C8
:107A20000E94A699ED968FAFED97882329F00E94CA
:107A3000259AED968FAFED9783E50E94A69988234E
:107A400019F00E94509A04C017FD08C086E990E022
:107A50000115110529F41092550402C086E490E046
:107A60001092600C10925F0CBC01990F880B990B5F
:107A70000E9445E624966FAF24972C967FAF2C97F3
:107A800060968FAF609764969FAF64970E94E750AF
:107A90004B015C01012B19F400EA13E00EC003EB6B
:107AA00013E0D8018D918D01882319F00E94008F79
:107AB000F8CF8AE00E94008F3BC4F80181918F01CA
:107AC000882319F00E94008FF8CF8AE00E94008F6F
:107AD0000E9486CE8FE780932F1381E0809304026B
:107AE000C258DF4F88829982AA82BB82CE57D0408B
:107AF000C857DF4F88829982AA82BB82C858D0407B
:107B000068961FAE6897F0E46C96FFAF6C972CE117
:107B1000A0962FAFA09736E4AC963FAFAC97E09617
:107B20001FAEE097A4961FAEA497A8961FAEA89785
:107B3000E4961FAEE497EC961CAE1DAE1EAE1FAED3
:107B4000EC97E8961CAE1DAE1EAE1FAEE897C12C9A
:107B5000D12C7601FFE74F2E512C612C712C8FE731
:107B600090E0A0E0B0E023968CAF9DAFAEAFBFAF8A
:107B70002397CE57DF4F188219821A821B82C25870
:107B8000D04091E0EE969FAFEE9729961FAE1EAEC5
:107B90002997212C312C00E010E0809104028823E9
:107BA00009F4C9C10E94E7506BAF7CAF8DAF9EAFA7
:107BB00080912D13882309F4CBC00E94ADCE209074
:107BC0005F0430906004009161041091620491019F
:107BD000A801E0966FADE097A4967FADA497A89614
:107BE0008FADA897E4969FADE4970E943FE687FF8C
:107BF0000CC0E0962FAEE097A4963FAEA497A8964F
:107C00000FAFA897E4961FAFE4979101A80168967B
:107C10006FAD68976C967FAD6C97A0968FADA0976F
:107C2000AC969FADAC970E9488EC181664F46896E9
:107C30002FAE68976C963FAE6C97A0960FAFA0974B
:107C4000AC961FAFAC97EE96AFADEE9724962FADE6
:107C500024972C963FAD2C9760964FAD6097649615
:107C60005FAD6497B101C801AA2309F455C00E9411
:107C700088EC18160CF06CC04BAD5CAD6DAD7EADF4
:107C8000481959096A097B09DB01CA0188589341DF
:107C9000A109B109B7FD5CC023968CAD9DADAEAD19
:107CA000BFAD239784199509A609B709B595A7957E
:107CB0009795879580932F13CE57DF4F488359832D
:107CC0006A837B83C258D0402496BFAD2497E09648
:107CD000BFAFE0972C96EFAD2C97A496EFAFA4978B
:107CE0006096FFAD6097A896FFAFA89764962FADFA
:107CF0006497E4962FAFE4978BAD9CADADADBEAD70
:107D0000C258DF4F88839983AA83BB83CE57D04064
:107D1000EE961FAEEE971CC00E943FE687FF18C08C
:107D20008BAD9CADADADBEADC258DF4F2881398162
:107D30004A815B81CE57D040821B930BA40BB50BBD
:107D4000AC01BD01485853416109710977FF8BC6E9
:107D500020E030E040EA51E424966FAD24972C9661
:107D60007FAD2C9760968FAD609764969FAD6497BA
:107D70000E9462EA9B01AC01B101C8010E9488EC3B
:107D800018166CF4EEE3F6E084918F010F5F1F4F3D
:107D9000882309F4CDC20E94008FF801F5CF80E35B
:107DA00098EFAFEFBFEFC857DF4F288139814A8185
:107DB0005B81C858D040821B930BA40BB50B2BAD35
:107DC0003CAD4DAD5EAD820F931FA41FB51FB7FD37
:107DD00011C00E943CD78AE00E94008F8BAD9CAD01
:107DE000ADADBEADC857DF4F88839983AA83BB83EF
:107DF000C858D0408BAD9CADADADBEAD880F991FBE
:107E0000AA1FBB1FC258DF4F288139814A815B817D
:107E1000CE57D040821B930BA40BB50B8819990940
:107E2000AA09BB0981389F44A241B10568F0E0E28C
:107E3000F6E084918F010F5F1F4F882309F478C209
:107E40000E94008FF801F5CF29964EAD5FAD2997BE
:107E5000CA57DF4F88819981C658D040841795074B
:107E60000CF066C0E3ECF5E084918F010F5F1F4FCB
:107E7000882321F00E94008FF801F6CFB701A601F8
:107E80008EEA95E00E94F8648AE00E94008FE896EE
:107E90004CAD5DAD6EAD7FADE89789E995E00E9490
:107EA000F8648AE00E94008FEC964CAD5DAD6EAD3B
:107EB0007FADEC9784E895E00E94F8648AE00E9428
:107EC000008FED969FADED97992309F431C2C092D2
:107ED0002802D0922902E0922A02F0922B022CEA88
:107EE00035EC47E25EE3E8966CAD7DAD8EAD9FADBF
:107EF000E8970E94A4E66093300270933102809369
:107F00003202909333022CEA35EC47E25EE3EC96C2
:107F10006CAD7DAD8EAD9FADEC970E943EEB609356
:107F20002C0270932D0280932E0290932F0200C298
:107F30000E94AE5632CE809104028111F9C10E9496
:107F400086CEF6C10E949B5DF3C180E00E946B97D4
:107F5000EFC1A0EBB4E0BCAFABAF8CEB282E84E05C
:107F6000382EE7E6F4E02196FFAFEEAF219700E070
:107F700010E021962EAD3FAD21972756344029962B
:107F80003FAF2EAF29972196AEADBFAD21978D9112
:107F90002196BFAFAEAF2197882309F4ACC0F8019A
:107FA000E55EFD4F2081318142815381F801EF5020
:107FB000F44F60817181828193810E9462EA20E0A6
:107FC00030E040E05FE30E94A4E69B01AC01F101D8
:107FD00060817181828193810E9488EC181634F44B
:107FE000C8018958974D0E94A57103C060E070E0F8
:107FF000CB01D1018D909D90AD90BC90F801E559D9
:10800000F34F20813181428153810E9462EA9B01BA
:10801000AC01C501B4010E9461EA6B017C0120E062
:1080200030E040EA51EC0E9488EC87FD35C020E04A
:1080300030E040EA51E4C701B6010E943FE618165D
:108040005CF1EBADFCAD4080518062807380A70194
:108050009601C301B2010E9461EA6B017C01A30198
:1080600092010E9461EA9B01AC01C501B4010E942A
:1080700062EAD1016D937D938D939C931397EBAD41
:10808000FCADC082D182E282F38229968EAD9FAD93
:1080900029970E9452992FC0E7E7F7E284918F0158
:1080A0000F5F1F4F882321F00E94008FF801F6CF49
:1080B000E0EDF6E084918F010F5F1F4F882321F0E0
:1080C0000E94008FF801F6CF61E082EC96E00E94FA
:1080D00088560E94644C88E290E09A83898388ECF9
:1080E00090E099A388A3BE016F5F7F4FCE01809679
:1080F0000E947D8B1DC12BAD3CAD2C5F3F4F3CAF33
:108100002BAF0C5F1F4F34E0230E311C0C301105D8
:1081100009F02FCF0E949B710E9408D660E082EB8D
:1081200096E00E94885683E992E099A388A304E62A
:1081300010E01A830983BE01605E7F4FCE01019675
:108140000E947D8B8AEB92E099A388A31A8309830E
:10815000BE01605E7F4FCE0101960E947D8BE8C01C
:10816000E7E7F7E284918F010F5F1F4F882321F02B
:108170000E94008FF801F6CFEEEEF6E084918F01B9
:108180000F5F1F4F882309F4D3C00E94008FF801AE
:10819000F5CF0E9482B2CCC083E50E94A6998823C5
:1081A00021F00E94259A91E089270E94C772C0C0E1
:1081B000EEE7FCE284918F010F5F1F4F882321F0CF
:1081C0000E94008FF801F6CFE9E1F7E084918F017A
:1081D0000F5F1F4F882311F40C944C370E94008FBF
:1081E000F801F4CFE2E0F7E084918F010F5F1F4FB9
:1081F000882311F40C9482370E94008FF801F4CF89
:108200004091111350911213609113137091141334
:108210008FEF96E00E94F8640C948237E7E7F7E26C
:1082200084918F010F5F1F4F882321F00E94008FE0
:10823000F801F6CFE3E2F7E084918F010F5F1F4F63
:10824000882309F475C00E94008FF801F5CF81E002
:10825000809316021092500C83E50E94A699882301
:1082600009F48DC50E94259A811162C088C5E092EB
:108270005604EEE7FCE284918F010F5F1F4F8823C5
:1082800021F00E94008FF801F6CFB701772782E333
:1082900097E00E946B768AE00E94008F49C080E0E0
:1082A00048C00E94FB9583E50E94A699882309F4A3
:1082B00063C00E94259AEE24E394F12C082FA301B9
:1082C0009201C501B4010E94B4976B017C012CEAB4
:1082D00035EC47E257E3C501B4010E9462EAAB0105
:1082E000BC0182E092E00E94DB642CEA35EC47E2BC
:1082F00057E3C301B2010E9462EAAB01BC018DEFFA
:1083000091E00E94DB642CEA35EC47E257E3C701B9
:10831000B6010E9462EAAB01BC0188EF91E00E94C5
:10832000DB648AE00E94008F0E94E1950E9408D6DB
:1083300081E01092600C10925F0C81111AC00C94B5
:10834000302984918F010F5F1F4F882321F00E94F5
:10835000008FF801F6CF6091610C7091620C84E49B
:1083600097E00E94847682E20E94008F8AE00E9459
:10837000008F0E9441952EC581E09DCF0E9493DE23
:10838000AB01BC014093A9125093AA126093AB12A7
:108390007093AC1288EF91E10E94CE78C9CF0E9411
:1083A00093DEAB01BC014093A9125093AA126093D3
:1083B000AB127093AC1288EF91E10E94CE780C94CE
:1083C000783561E08D2D0E94AC4F6E2D8D2D0E9471
:1083D000644EB7018D2D0E94E84F0930110509F058
:1083E000A7CFF0928B06E0928A06A2CF0E94509A05
:1083F000909389068093880680E00E9453CE0E9465
:10840000509A8635910544F40E9420A860E084E7E4
:1084100093E00E94885602C00E94CC8B609188062F
:1084200070918906072E000C880B990B0E9445E677
:1084300020915F0430916004409161045091620486
:108440000E9488EC1816B4F484E893E09F938F930D
:108450008091550490E001969F938F938DE693E071
:108460009F938F931F920E94B18B0FB6F894DEBF3B
:108470000FBECDBF0E9436E181E0809304021092CE
:10848000600C10925F0C23961CAE1DAE1EAE1FAE8C
:10849000239727961CAE1DAE1EAE1FAE27971BAEB0
:1084A0002C961FAE2C979CE360969FAF6097ACE133
:1084B0006496AFAF6497B6E46896BFAF6897C12C77
:1084C000D12CF0E8EF2EAFEBFA2E812C912C540139
:1084D0006091880670918906072E000C880B990B15
:1084E0000E9445E6162F072F782E692E262F372F4C
:1084F000482F592FB601C7010E943FE6882311F18A
:1085000020915F04309160044091610450916204B5
:10851000612F702F872D962D0E943FE6881F882798
:10852000881F8BAF2896EFAD2897EE2379F088232C
:1085300069F080910402882309F4FACE60E088E5AE
:1085400093E06EC11C2D0D2D7E2C6F2C0E94E750E8
:108550006B017C01DC01CB0127962CAD3DAD4EAD0E
:108560005FAD2797821B930BA40BB50BB7FD47C0DC
:10857000D701C60188519C4FAF4FBF4F27968CAF94
:108580009DAFAEAFBFAF27970E943CD7E9E6F3E0BF
:1085900084912F019FEF491A590A882321F00E94E4
:1085A000008FF201F5CF81149104A104B104D1F040
:1085B000D501C401805F984DAF4FBF4FBC01CD01C5
:1085C0006C197D098E099F0928EE33E040E050E0E8
:1085D0000E9404EACA01B9010E946D8F8AE00E94DC
:1085E000008F0DC0E6E6F3E084912F01AFEF4A1A49
:1085F0005A0A882321F00E94008FF201F5CF0E94D1
:10860000BD920E94AB7160915F0470916004809193
:108610006104909162040E94A6EB072E000C880B67
:10862000990B0E9445E61B012C019B01AC01612FB7
:10863000702F872D962D0E9461EA9F7781149104F7
:10864000A104B10449F420E030E040E85FE30E9477
:108650003FE687FF0BC008C020E030E040E450E474
:108660000E9488EC181614F446015701BBADBB23D9
:1086700009F443C023962CAD3DAD4EAD5FAD2397BD
:10868000211531054105510541F0D701C601821B75
:10869000930BA40BB50BB7FD30C09101A2012C9632
:1086A0006FAD2C9760967FAD609764968FAD6497A1
:1086B00068969FAD68970E9461EA20E030E040EC48
:1086C0005FE30E943FE687FD34CFD701C601805AA1
:1086D0009541AF4FBF4F23968CAF9DAFAEAFBFAFAD
:1086E00023972C962FAE2C9760963FAE609764969A
:1086F0004FAE649768965FAE6897809104028823B6
:1087000009F417CF81149104A104B10429F4C12EF6
:10871000D02EE72CF62CDCCE90E1C91A97E2D90ACC
:10872000E108F108C818D908EA08FB08F7FE01CFEC
:10873000EECF0E94509A90938D0680938C060E94F3
:1087400020CE0E94509A069714F00E94CC8B81E0B4
:10875000809304021092600C10925F0C809156047A
:108760008093550423961CAE1DAE1EAE1FAE2397FC
:1087700027961CAE1DAE1EAE1FAE27971BAE2C96C5
:108780001FAE2C97ACE36096AFAF6097BCE16496E8
:10879000BFAF6497E6E46896EFAF6897C12CD12C21
:1087A00070E8E72EEFEBFE2E812C912C54016091A6
:1087B0008C0670918D06072E000C880B990B0E9479
:1087C00045E6162F072F782E692E262F372F482F94
:1087D000592FB601C7010E943FE6882321F120915D
:1087E0006304309164044091650450916604612FE4
:1087F000702F872D962D0E943FE6881F8827881F9F
:108800008BAF2896FFAD2897FF2389F0882379F056
:1088100080910402882309F48BCD60E088E893E01E
:108820000E94885685CD1C2D0D2D7E2C6F2C0E940C
:10883000E7506B017C01DC01CB0127962CAD3DADEF
:108840004EAD5FAD2797821B930BA40BB50BB7FD05
:1088500047C0D701C60188519C4FAF4FBF4F2796E5
:108860008CAF9DAFAEAFBFAF27970E943CD7E5E975
:10887000F3E084912F019FEF491A590A882321F0D0
:108880000E94008FF201F5CF81149104A104B1047C
:10889000D1F0D501C401805F984DAF4FBF4FBC01EF
:1088A000CD016C197D098E099F0928EE33E040E067
:1088B00050E00E9404EACA01B9010E946D8F8AE06B
:1088C0000E94008F0DC0E2E9F3E084912F01AFEF29
:1088D0004A1A5A0A882321F00E94008FF201F5CF2C
:1088E0000E94BD920E94AB71609163047091640418
:1088F00080916504909166040E94A6EB072E000CFF
:10890000880B990B0E9445E61B012C019B01AC01D1
:10891000612F702F872D962D0E9461EA9F77811419
:108920009104A104B10449F420E030E040E85FE3A1
:108930000E943FE687FF0BC008C020E030E040E423
:1089400050E40E9488EC181614F446015701BBADA0
:10895000BB2309F443C023962CAD3DAD4EAD5FADB6
:108960002397211531054105510541F0D701C60175
:10897000821B930BA40BB50BB7FD30C09101A20174
:108980002C966FAD2C9760967FAD609764968FADF7
:10899000649768969FAD68970E9461EA20E030E096
:1089A00040EC5FE30E943FE687FD32CFD701C6016E
:1089B000805A9541AF4FBF4F23968CAF9DAFAEAF5E
:1089C000BFAF23972C962FAE2C9760963FAE609743
:1089D00064964FAE649768965FAE68978091040284
:1089E000882309F415CF81149104A104B10429F45A
:1089F000C12ED02EE72CF62CDACE90E1C91A97E2E0
:108A0000D90AE108F108C818D908EA08FB08F7FEF6
:108A1000FFCEEECF0E949B5D88E50E94A699882339
:108A200019F05F9A1092AC0489E50E94A6998823F8
:108A300019F08A9A1092AD048AE50E94A6998823BB
:108A400051F09FB7F89480910801816080930801EC
:108A50009FBF1092AE0485E40E94A699882309F472
:108A600067CC129A65CC29964EAD5FAD2997141646
:108A700015060CF049C1CE57DF4F88809980AA8037
:108A8000BB80C258D040880E991EAA1EBB1ECE576E
:108A9000DF4F288139814A815B81C258D040281B31
:108AA000390B4A0B5B0BCA01B901A30192010E9469
:108AB000F5E9A50194010E9426EA23964CAC5DAC31
:108AC0006EAC7FAC2397420E531E641E751E34E1BC
:108AD00043165104610471041CF14CEE4416510418
:108AE000610471043CF450E84516510461047104BA
:108AF0003CF105C05BEE452E512C612C712C239668
:108B00004CAE5DAE6EAE7FAE23978EEF90E0A0E0F0
:108B1000B0E084199509A609B7092C013D0116C0DA
:108B200024E130E040E050E023962CAF3DAF4EAF63
:108B30005FAF239744E1442E512C612C712C06C069
:108B400023964CAE5DAE6EAE7FAE239723964CADB2
:108B50005DAD6EAD7FAD23978AEA96E00E943FDE61
:108B6000B301A20185EA96E00E943FDE68964FAD10
:108B700068976C965FAD6C97A0966FADA097AC961A
:108B80007FADAC978EE996E00E94F864E0964FAD19
:108B9000E097A4965FADA497A8966FADA897E496CA
:108BA0007FADE49787E996E00E94F86429964EAD80
:108BB0005FAD2997433051050CF4A6C0C301B20143
:108BC0000E9445E620E030E040E850E40E94A4E640
:108BD0006B017C0168962FAD68976C963FAD6C97E2
:108BE000A0964FADA097AC965FADAC97E0966FADF9
:108BF000E097A4967FADA497A8968FADA897E4962A
:108C00009FADE4970E9461EA2BED3FE049E450E418
:108C10000E94A4E620E030E040E05FE30E94A4E68A
:108C20009B01AC01C701B6010E943EEB6B017C01C8
:108C3000C501B4010E9445E62FE632E143E85AE35C
:108C40000E94A4E64B015C01B701A60181E996E010
:108C50000E94F864B501A4018BE896E00E94F864D4
:108C60002AE939E949E15FE3C701B6010E94A4E6B8
:108C70006B017C019B01AC010E9462EAA501940199
:108C80000E943EEBE8966CAF7DAF8EAF9FAFE8974A
:108C9000A5019401C701B6010E94A4E620E030E0DE
:108CA00040E05EE30E94A4E6EC966CAF7DAF8EAF31
:108CB0009FAFEC97EBE7F6E084915F015FEFA51AB9
:108CC000B50A882321F00E94008FF501F5CFB70186
:108CD000A60185E796E00E94F864E8964CAD5DAD8C
:108CE0006EAD7FADE8978FE696E00E94F864EC9653
:108CF0004CAD5DAD6EAD7FADEC9789E696E00E9420
:108D0000F8648AE00E94008F23968CAD9DADAEADD5
:108D1000BFAD2397840D951DA61DB71DB595A795CD
:108D20009795879580932F1329968EAD9FAD2997A0
:108D3000019629969FAF8EAF299724969FAD2497D1
:108D400068969FAF68972C96AFAD2C976C96AFAF97
:108D50006C976096BFAD6097A096BFAFA0976496E2
:108D6000EFAD6497AC96EFAFAC978BAC9CACADAC71
:108D7000BEACF1E0EE96FFAFEE970C94A83E0E94D9
:108D8000C8D7D6CA0E949B5DD02E60E0802F0E947B
:108D9000AC4F4FEFE416F40659F4802F0E94DBD954
:108DA00031E020E0892B09F030E0032F122F05C0BD
:108DB000EA94EF2861F000E010E08D2D0E94DBD9ED
:108DC0008017910709F4B4CA0E94BD92F6CF01E062
:108DD00010E0F3CFC157DF4F0FB6F894DEBF0FBEE0
:108DE000CDBFDF91CF911F910F91FF90EF90DF905A
:108DF000CF90BF90AF909F908F907F906F905F903B
:108E00004F903F902F9008954F925F926F927F9274
:108E10008F929F92AF92BF92CF92DF92EF92FF928A
:108E20000F931F93CF93DF93CDB7DEB762970FB643
:108E3000F894DEBF0FBECDBF10929B060E94E75094
:108E40000091900410919104209192043091930428
:108E50006B017C01C01AD10AE20AF30AF7FC13C0C5
:108E600020918F04209520938F04DC01CB018A543C
:108E70009C4FAF4FBF4F8093900490939104A09369
:108E80009204B0939304FF24F39480918F04811192
:108E900001C0F12C0E942D568091D30F853198F49A
:108EA000FF2049F080918A0690918B06892B19F05A
:108EB0000DE918E002C000E817E023E14FE061E0AF
:108EC00089E00E945DA58091D30F8D3108F093C198
:108ED0008830D0F56091880670918906072E000CC5
:108EE000880B990B0E9445E620E030E040E05FE30C
:108EF0000E9462EA0E94A6EB7C876B87643671054C
:108F00002CF46A30710524F426E003C022E101C08C
:108F10002CE082E190E0821B910997FD01969595E6
:108F200087959195819591098B5F8093D60F87E006
:108F30008093D70FCE010B960E9495550E9407D1C2
:108F40008DE797E00E94FAD08091D30F8D3108F021
:108F500044C08091D50F853108F43FC060915F0413
:108F60007091600480916104909162040E94A6EB6C
:108F7000072E000C880B990B0E9445E620E030E09C
:108F800040E05FE30E9462EA0E94A6EB9B017E87BD
:108F90006D87643671050CF06BC32A3031050CF017
:108FA00065C326E082E190E0821B910997FD01965E
:108FB000959587959195819591098B5F8093D60FB3
:108FC0008CE18093D70FCE010D960E9495550E949B
:108FD00007D18DE797E00E94FAD08091D30F8531B9
:108FE00040F58091D50F813120F160918806709114
:108FF0008906072E000C880B990B0E9445E62091EC
:109000005F043091600440916104509162040E94B9
:1090100088EC18160CF02EC31092BF0F02E022E06D
:1090200041E16DE08FE99FE00E9408B681E0809306
:10903000BF0F8091D30F8830D0F560918C0670916E
:109040008D06072E000C880B990B0E9445E620E048
:1090500030E040E05FE30E9462EA0E94A6EB788B7A
:109060006F87643671052CF46A30710524F426E0AC
:1090700003C022E101C02CE082E190E0821B910953
:1090800097FD0196959587959195819591098F5AB0
:109090008093D60F87E08093D70FCE010F960E9462
:1090A00095550E9407D18DE797E00E94FAD08091F4
:1090B000D30F8D3108F044C08091D50F853108F46D
:1090C0003FC0609163047091640480916504909145
:1090D00066040E94A6EB072E000C880B990B0E94D9
:1090E00045E620E030E040E05FE30E9462EA0E9453
:1090F000A6EB9B017A8B698B643671050CF0C5C2B7
:109100002A3031050CF0BFC226E082E190E0821BDC
:10911000910997FD0196959587959195819591096E
:109120008F5A8093D60F8CE18093D70FCE01419652
:109130000E9495550E9407D18DE797E00E94FAD0D2
:109140008091D30F853140F58091D50F813120F189
:1091500060918C0670918D06072E000C880B990B80
:109160000E9445E6209163043091640440916504B7
:10917000509166040E9488EC18160CF088C2109278
:10918000BF0F02E022E042E168E58FE99FE00E9424
:1091900008B681E08093BF0F8091D30F8C3158F5D2
:1091A0008091D50F843138F120918A0630918B0659
:1091B0002F5F3F4F44E6429FC001439F900D112413
:1091C00097FF02C081509F4F292F392F330F330B48
:1091D0003A832983232B79F088E68093D60F8BE19D
:1091E0008093D70FCE0101960E9495550E9407D11A
:1091F00085E20E94E6868091D30F843328F4809123
:10920000D50F8A3208F04CC28091D30F853328F4F1
:109210008091D50F813308F06BC280912D10882387
:1092200009F44BC08091D30F843308F046C080917D
:10923000D50F823308F441C02091FB11222319F18C
:109240008091A5129091A612A091A712B091A81298
:109250000097A105B10509F452C2BC01CD016D59B9
:109260007F4F8F4F9F4F24E630E040E050E00E9458
:1092700004EA6091A9127091AA128091AB129091A8
:10928000AC120E9404EA48E4249FB0011124072E86
:10929000000C880B990B0E9445E62AE037ED43E26B
:1092A0005CE30E94A4E60E94ABEB262F02E042E3BF
:1092B00067E38FE99FE00E9408B68091D30F813366
:1092C00008F060C08091D50F893208F45BC00E941D
:1092D00039A82B013C018CE3882E912CA12CB12CB8
:1092E000C301B201A50194010E9404EACA01B901B7
:1092F000A50194010E9404EACA01962E872E590105
:109300008E010F5F1F4F41E8441641E5540641E0CE
:109310006406710408F4F5C1B90128E130E040E0C9
:1093200050E00E9404EA29013A018F929F92C50100
:1093300068E170E00E9426ED9F938F935F924F92B9
:1093400089E697E09F938F931F930F930E94D8E530
:109350000FB6F894DEBF0FBECDBF9AE04916510498
:109360006104710408F0FCC197E0892F880F980F01
:109370009195955A9093D60F80E38093D70FC801AB
:109380000E9407D1E091990FF0919A0F8481811189
:10939000D4C06091BC047091BD048091BE049091D2
:1093A000BF040E94A6EB7A836983CE0101960E94D6
:1093B0002955BC0180EA94E00E94AFED6091C004A1
:1093C0007091C1048091C2049091C3040E94A6EBE5
:1093D0007A836983CE0101960E942955BC018BE9ED
:1093E00094E00E94AFED2CEA35EC47E257E3609140
:1093F000C4047091C5048091C6049091C7040E9472
:1094000062EA20E030E048EC52E40E94A4E60E94C8
:10941000A6EB4B015C0197FD19C090E1891697E21C
:109420009906A104B104E4F0C501B40120E137E2DA
:1094300040E050E00E9426EACA01B9012AE030E08B
:1094400040E050E00E9426EA605D0BC0B094A0941A
:1094500090948094811C911CA11CB11C6DE201C0F0
:1094600060E26093490C28EE821623E09206A10484
:10947000B10494F0C501B40128EE33E040E050E0BF
:109480000E9426EACA01B9012AE030E040E050E03B
:109490000E9426EA605D01C060E260934A0CC5014B
:1094A000B40124E630E040E050E00E9426EA9AE071
:1094B000492E512C612C712CCA01B901A3019201D2
:1094C0000E9426EA605D60934B0CC501B401A301C4
:1094D00092010E9426EA4B015C01672B682B692BE5
:1094E00079F08EE280934C0CCA01B901A30192017C
:1094F0000E9426EA605D60934D0C80E3880D15C0E4
:10950000CA01B901A30192010E9426EA662339F03B
:109510008EE280934C0C605D60934D0C05C080E240
:1095200080934D0C80934C0C80E280934E0C69E448
:109530007CE084E994E00E94AFED8091D30F883203
:1095400098F48091D50F8D3178F02BE040E86DE1F3
:1095500080E00E9488A68091D30F873228F4809102
:10956000D50F8F3108F0FEC08091D30F823328F4DD
:109570008091D50F8B3208F060C18091D30F803479
:1095800028F48091D50F883308F074C180919D062E
:10959000882349F00E9436D040E050E0BA0181E8CB
:1095A0009CE40E94CACF2091190230911A02409186
:1095B0007606509177066091780670917906C90118
:1095C000840F951F2436310524F4853691053CF42B
:1095D00016C02436310531F08436910584F484E6D2
:1095E00090E00DC04B3051056105710514F00A97EC
:1095F00006C0463F5F4F6F4F7F4F6CF40A969093C3
:109600001A02809319021092760610927706109231
:109610007806109279068091190290911A028A3088
:1096200091053CF0883E43E094072CF087EE93E0F0
:1096300002C08AE090E090931A0280931902629629
:109640000FB6F894DEBF0FBECDBFDF91CF911F9153
:109650000F91FF90EF90DF90CF90BF90AF909F90D1
:109660008F907F906F905F904F9008952CE09ACCF0
:1096700022E198CC02E022E041E16DE08FE99FE039
:109680000E9408B6D6CC2CE040CD22E13ECD02E0CF
:1096900022E042E168E58FE99FE00E9408B67CCDB8
:1096A00007E028E04AE26AE28FE99FE00E9408B6FC
:1096B00005E022E04CE262E38FE99FE00E9408B6F9
:1096C00024E04AE061E38AE20E9488A66091A10F4B
:1096D0007091A20F82E38093BB0F8BE28093BC0F4B
:1096E0002BEB3FE042E38FE99FE00E94F0B48CCD8A
:1096F00024E04AE461E386E30E9488A68ECD20E060
:10970000C2CD44E6A416B104C0F48F929F92C50165
:1097100068E170E00E9426ED9F938F938FE597E0BC
:109720009F938F931F930F930E94D8E50FB6F894E1
:10973000DEBF0FBECDBF95E018CE8F929F923F93B4
:109740002F9387E597E09F938F931F930F930E942A
:10975000D8E50FB6F894DEBF0FBECDBF96E005CEBC
:1097600098E003CE83E08093D60F86E28093D70FF4
:10977000FF2029F08BE797E00E94FAD00DC080917E
:109780006704811102C08FE305C08091AC04811190
:10979000F1CF80E20E94E6868BE08093D60F16E23E
:1097A0001093D70F80EA94E00E9407D18BE2809358
:1097B000D60F1093D70FFF2029F089E797E00E947A
:1097C000FAD00DC080916804811102C08FE305C0FA
:1097D0008091AD048111F1CF80E20E94E68683E39F
:1097E0008093D60F16E21093D70F8BE994E00E9476
:1097F00007D183E58093D60F1093D70FFF2029F070
:1098000087E797E00E94FAD00DC08091690481112A
:1098100002C08FE305C08091AE048111F1CF80E2D8
:109820000E94E6868BE58093D60F86E28093D70F61
:1098300084E994E00E9407D197CE84E00E941CD076
:1098400083E08093D60F12E31093D70F86E00E9437
:10985000E6D00E942D568CE08093D60F1093D70F40
:1098600089E192E00E9495550E9407D185E20E940D
:10987000E68683CE1092D60F8FE38093D70F86E4CF
:1098800092E00E9407D182CE80915E048630D8F4A7
:1098900096E0899FF0011124E559FB4F20910D02BC
:1098A00030910E02318320834091760650917706E5
:1098B000609178067091790642835383648375833F
:1098C0008F5F80935E04089540E050E0BA0184E029
:1098D00097E40C94CACFE0915E04EE2389F0E15046
:1098E000E0935E0486E0E89FF0011124E559FB4F08
:1098F0004281538164817581808191810C94CACFAA
:10990000E3CF0F931F93CF93DF9310929B06809129
:10991000760690917706A0917806B091790681300D
:109920009048A105B10540F0109276061092770696
:109930001092780610927906C09176068091A5045F
:109940001816DCF4282F082E000C330B2150310997
:109950004C2F0C2E000C550B4217530774F0CFEF11
:10996000C80F8C2F90E0A0E0B0E080937606909333
:109970007706A0937806B09379061092BA12809178
:10998000B912C81714F4C093B9128091B912082EF5
:10999000000C990B04962C2F0C2E000C330B821705
:1099A000930724F48CEF8C0F8093B9121091B912A5
:1099B000D0E001E0112341F08091FD0F9091FE0F66
:1099C000891B8F70B9F519C080914002882349F036
:1099D00081E0C11180E024E04AE15AE06D2F0E944D
:1099E000EE5580919D06882339F3C111E5CF73DFD1
:1099F0008091BA12882301F30EC180912D1081113C
:109A000019C01130D1F480914002882351F081E0D7
:109A1000C13009F080E023E04DE05AE06D2F0E9454
:109A2000EE5580919D06882331F1C13021F583E008
:109A300097E61BC0113009F4D6C01230E1F48091D2
:109A40004002882351F081E0C23009F080E023E039
:109A500045E05AE06D2F0E94EE5580919D068823C7
:109A600051F0C23041F482E494E80E94825980911E
:109A7000BA128111D0C080912E10882309F48BC0B6
:109A80008091FB11882309F476C080912D108823E2
:109A9000E9F01330D9F580914002882351F081E03C
:109AA000C33009F080E020E249EF59E06D2F0E94B9
:109AB000EE5580919D06882309F48CC0C33009F0CF
:109AC00089C010922D100E940C8C50C01330F1F4FC
:109AD00080914002882351F081E0C33009F080E09A
:109AE00020E24CEE59E06D2F0E94EE5580919D06CC
:109AF000882309F46FC0C33009F06CC080912E1028
:109B0000811100932D100E94CC8B30C0143009F0CD
:109B100061C080914002882351F081E0C43009F097
:109B200080E020E241EE59E06D2F0E94EE558091D9
:109B30009D06882309F44EC0C43009F04BC00E9432
:109B4000DC8680916A0480936D0610926E060E94F6
:109B500084D50E9420A810928B0610928A0610923B
:109B6000040260E08AEB99E00E9488568091BA1264
:109B7000882381F150C0133011F084E02CC0809113
:109B800040028823C1F081E0C33009F080E023E087
:109B900043ED59E00DC0133081F7809140028823D6
:109BA00051F081E0C33009F080E023E048EC59E057
:109BB0006D2F0E94EE5580919D068823F1F2C330EF
:109BC000E1F683EB9EEA0E9482598091BA128823C3
:109BD000A1F221C085E0DF5F1F5FD53009F0EACE3A
:109BE0008093A50418C080914002882349F081E049
:109BF000C13009F080E023E045E15AE06D2FEED757
:109C000080919D06882309F436CFC13009F033CF07
:109C100082E59AE62ACFDF91CF911F910F910895A7
:109C2000CF92DF92EF92FF920F931F93CF93DF9328
:109C30006C017A018B01C0E0D0E0CE15DF0589F020
:109C4000D8016D918D01D601ED91FC910190F081CB
:109C5000E02DC6011995892B11F47E0102C02196D1
:109C6000ECCFC701DF91CF911F910F91FF90EF9043
:109C7000DF90CF9008950E945BED0F931F93CF93D9
:109C8000DF93EB018A01181619066CF4843121E088
:109C9000920714F083E191E09093890680938806FF
:109CA00080E00E9453CED7FD06C0D0938D06C093AE
:109CB0008C060E9420CE10938B0600938A06DF91BB
:109CC000CF911F910F9100CE1F93CF93DF93282F39
:109CD00030E0F901EE58F44F8491F901E45DF44F5E
:109CE000D491F901EA51F54FC491CC23C1F0162F5C
:109CF0008111DCD0EC2FF0E0EE0FFF1FEE54F54F9A
:109D0000A591B4918FB7F894111105C09C91ED2FD6
:109D1000E095E92302C0EC91ED2BEC938FBFDF912E
:109D2000CF911F9108951F920F920FB60F92112499
:109D30000BB60F922F933F934F935F936F937F9345
:109D40008F939F93AF93BF93EF93FF93809172068E
:109D500090917306A0917406B0917506892B8A2B99
:109D60008B2B59F180917106E0916F06F09170068E
:109D70009081892780838091720690917306A091CB
:109D80007406B0917506181619061A061B060CF013
:109D900055C08091720690917306A0917406B0919F
:109DA00075060197A109B109809372069093730615
:109DB000A0937406B093750641C080910C02E1E255
:109DC000FDE0E4919FEF90930C02E230C9F050F473
:109DD000EE2399F0E13081F590916F009D7F909393
:109DE0006F002AC0E43019F1E0F0E53029F59091D8
:109DF00073009D7F909373001FC010926E001CC073
:109E0000909170009D7F9093700091E09093B000CE
:109E10009091B100987F94609093B1001092B3003C
:109E20000BC0909171009D7F9093710005C090913F
:109E300072009D7F9093720060E046DFFF91EF918A
:109E4000BF91AF919F918F917F916F915F914F9152
:109E50003F912F910F900BBE0F900FBE0F901F9050
:109E600018953FB7F8948091B8069091B906A091E3
:109E7000BA06B091BB0626B5A89B05C02F3F19F0C6
:109E80000196A11DB11D3FBFBA2FA92F982F88277A
:109E9000820F911DA11DB11DBC01CD0142E0660FD5
:109EA000771F881F991F4A95D1F7089590E0FC010C
:109EB0003197E231F10508F04EC08827EE58FF4F88
:109EC0008F4F0C944DED809180008F7703C080916F
:109ED00080008F7D80938000089580918000877F2F
:109EE000F9CF84B58F7702C084B58F7D84BD089586
:109EF0008091B0008F7703C08091B0008F7D8093F8
:109F0000B0000895809190008F7707C080919000F5
:109F10008F7D03C080919000877F8093900008958B
:109F20008091A0008F7707C08091A0008F7D03C033
:109F30008091A000877F8093A000089580912001E8
:109F40008F7707C0809120018F7D03C08091200111
:109F5000877F809320010895CF93DF9390E0FC01E9
:109F6000E45DF44F2491FC01EA51F54F849188237C
:109F700061F190E0880F991FFC01E35CF24FC591FD
:109F8000D491FC01EE54F54FA591B491611109C033
:109F90009FB7F8948881209582238883EC912E23A3
:109FA0000BC0623061F49FB7F8943881822F80959E
:109FB00083238883EC912E2B2C939FBF06C08FB7F1
:109FC000F894E8812E2B28838FBFDF91CF910895DD
:109FD0001F93CF93DF93182FEB0161E0BDDF209734
:109FE00011F460E004C0CF3FD10531F461E0812F6E
:109FF000DF91CF911F9168CEE12FF0E0EE58F44F42
:10A00000E4914E2F50E0FA013197E231F10508F06A
:10A010009DC08827EC57FF4F8F4F0C944DED84B5B2
:10A02000806884BDC7BD97C084B5806284BDC8BD4B
:10A0300092C080918000806880938000D0938900D6
:10A04000C093880088C080918000806280938000E7
:10A05000D0938B00C0938A007EC08091800088607E
:10A0600080938000D0938D00C0938C0074C0809149
:10A07000B00080688093B000C093B3006CC0809142
:10A08000B00080628093B000C093B40064C080913F
:10A090009000806880939000D0939900C0939800BE
:10A0A0005AC080919000806280939000D0939B0072
:10A0B000C0939A0050C08091900088608093900077
:10A0C000D0939D00C0939C0046C08091A000806802
:10A0D0008093A0008091A0008F7B8093A000D093FC
:10A0E000A900C093A80037C08091A000806280932F
:10A0F000A000D093AB00C093AA002DC08091A00017
:10A1000088608093A000D093AD00C093AC0023C0C2
:10A1100080912001806880932001D0932901C09311
:10A12000280119C080912001806280932001D09382
:10A130002B01C0932A010FC0809120018860809379
:10A140002001D0932D01C0932C0105C0C038D1054A
:10A150000CF04CCF46CFDF91CF911F9108958F9295
:10A160009F92AF92BF92CF92DF92EF92FF926B01DC
:10A170007C0177DE4B015C01C114D104E104F104E0
:10A18000E9F06FDEDC01CB0188199909AA09BB0946
:10A19000883E9340A105B10578F321E0C21AD108A9
:10A1A000E108F10888EE880E83E0981EA11CB11C1E
:10A1B000C114D104E104F10421F7DECFFF90EF9048
:10A1C000DF90CF90BF90AF909F908F9008952FB762
:10A1D000F8946091B4067091B5068091B60690919E
:10A1E000B7062FBF08951F920F920FB60F9211243A
:10A1F0002F933F938F939F93AF93BF938091B40618
:10A200009091B506A091B606B091B7063091B3060D
:10A2100023E0230F2D3720F40196A11DB11D05C0A9
:10A2200026E8230F0296A11DB11D2093B30680934B
:10A23000B4069093B506A093B606B093B706809186
:10A24000B8069091B906A091BA06B091BB060196E6
:10A25000A11DB11D8093B8069093B906A093BA06CC
:10A26000B093BB06BF91AF919F918F913F912F917A
:10A270000F900FBE0F901F9018958F929F92AF92E4
:10A28000BF92CF92DF92EF92FF92CF93FC01C080FA
:10A29000D180E280F38020E030E0A901C701B6015F
:10A2A0000E943FE687FF08C0C701B601905820E032
:10A2B00030E048EC52E406C020E030E048EC52E4E4
:10A2C000C701B6010E94A4E60E94A6EB6B017C01C7
:10A2D000603AF6E87F07F1E08F07910584F020EA05
:10A2E00036E841E050E00E9426EACA01B9012AE0BE
:10A2F00030E040E050E00E9426EA605D01C060E28C
:10A300006093480C80E1C81687E2D806E104F104A6
:10A3100094F0C701B60120E137E240E050E00E942E
:10A3200026EACA01B9012AE030E040E050E00E948C
:10A3300026EA605D01C060E26093490CE8EECE164B
:10A34000E3E0DE06E104F10494F0C701B60128EE73
:10A3500033E040E050E00E9426EACA01B9012AE059
:10A3600030E040E050E00E9426EA605D01C060E21B
:10A3700060934A0CC701B60124E630E040E050E0AB
:10A380000E9426EA8AE0882E912CA12CB12CCA01C9
:10A39000B901A50194010E9426EA605D60934B0C0F
:10A3A0008EE280934C0CC701B601A50194010E9476
:10A3B00026EAC62FCA01B901A50194010E9426EA26
:10A3C000605D60934D0CC05DC0934E0C88E49CE0D2
:10A3D000CF91FF90EF90DF90CF90BF90AF909F9084
:10A3E0008F9008950F931F93CF93DF9300D01F9208
:10A3F000CDB7DEB78091760690917706A09178066A
:10A40000B0917906B7FF08C01092760610927706D1
:10A41000109278061092790680917A0690917B06C8
:10A42000A0917C06B0917D0640917606509177060A
:10A43000609178067091790684179507A607B7078B
:10A4400044F48093760690937706A0937806B093B1
:10A45000790680914002882371F1409176065091EF
:10A460007706609178067091790680917E069091CA
:10A470007F06A0918006B09181068A019B01080F9A
:10A48000191F2A1F3B1FC901B8010E9445E62AE097
:10A4900037ED43E25CE30E94A4E669837A838B8311
:10A4A0009C83CE010196E9DEBC01809184069091E7
:10A4B00085060E9419D180919D06882381F14091E3
:10A4C00076065091770660917806709179068091B2
:10A4D0007E0690917F06A0918006B09181068A0148
:10A4E0009B01080F191F2A1F3B1FC901B8010E94B9
:10A4F00045E62AE037ED43E25CE30E94A4E6E09102
:10A500008206F0918306309721F060837183828305
:10A510009383E1D9E0918606F091870619950F9013
:10A520000F900F900F90DF91CF911F910F91089591
:10A530008F929F92AF92BF92CF92DF92EF92FF9253
:10A54000CF9320E030E048EC52E4FC01608171815F
:10A55000828193810E94A4E60E94A6EB6B017C019C
:10A5600097FF0AC0F094E094D094C094C11CD11C11
:10A57000E11CF11C8DE201C08BE28093480CC70105
:10A58000B60120E137E240E050E00E9426EA8AE08E
:10A59000882E912CA12CB12CCA01B901A5019401DE
:10A5A0000E9426EA605D6093490CC701B60128EE5F
:10A5B00033E040E050E00E9426EACA01B901A5015B
:10A5C00094010E9426EA605D60934A0CC701B601BF
:10A5D00024E630E040E050E00E9426EACA01B901DA
:10A5E000A50194010E9426EA605D60934B0C8EE207
:10A5F00080934C0CC701B601A50194010E9426EA84
:10A60000C62FCA01B901A50194010E9426EA605D26
:10A6100060934D0CC05DC0934E0C88E49CE0CF91DC
:10A62000FF90EF90DF90CF90BF90AF909F908F9072
:10A6300008958F929F92AF92BF92CF92DF92EF9246
:10A64000FF92FC01C080D180E280F38020E030E006
:10A65000A901C701B6010E943FE687FF04C0C701F8
:10A66000B601905802C0C701B6010E94A6EB6B016B
:10A670007C016031F7E27F078105910584F020E1DC
:10A6800037E240E050E00E9426EACA01B9012AE020
:10A6900030E040E050E00E9426EA605D01C060E2E8
:10A6A00060934A0C88EEC81683E0D806E104F104F2
:10A6B00094F0C701B60128EE33E040E050E00E947C
:10A6C00026EACA01B9012AE030E040E050E00E94E9
:10A6D00026EA605D01C060E260934B0CE4E6CE16B2
:10A6E000D104E104F10494F0C701B60124E630E09E
:10A6F00040E050E00E9426EACA01B9012AE030E0B9
:10A7000040E050E00E9426EA605D01C060E2609394
:10A710004C0CFAE0CF16D104E104F1049CF08AE07D
:10A72000882E912CA12CB12CC701B601A501940152
:10A730000E9426EACA01B901A50194010E9426EAF5
:10A74000605D01C060E260934D0CC701B6012AE074
:10A7500030E040E050E00E9426EA605D60934E0CDD
:10A760008AE49CE0FF90EF90DF90CF90BF90AF9095
:10A770009F908F9008950F931F93CF93DF9300D0F6
:10A780001F92CDB7DEB78091760690917706A091A3
:10A790007806B0917906B7FF08C01092760610923D
:10A7A0007706109278061092790680917A06909139
:10A7B0007B06A0917C06B0917D0640917606509173
:10A7C0007706609178067091790684179507A60739
:10A7D000B70744F48093760690937706A0937806A3
:10A7E000B093790680914002882371F140917606FA
:10A7F00050917706609178067091790680917E0677
:10A8000090917F06A0918006B09181068A019B01FC
:10A81000080F191F2A1F3B1FC901B8010E9443E6F8
:10A8200020E030E048EC52E40E94A4E669837A8399
:10A830008B839C83CE010196FCDEBC018091840653
:10A84000909185060E9419D180919D06882391F1EF
:10A85000409176065091770660917806709179065E
:10A8600080917E0690917F06A0918006B09181062E
:10A870008A019B01080F191F2A1F3B1FC901B8013C
:10A880000E9443E620E030E048EC52E40E94A4E657
:10A890000E94ABEBE0918206F0918306309721F0A5
:10A8A000608371838283938316D8E0918606F0914A
:10A8B000870619950F900F900F900F90DF91CF9111
:10A8C0001F910F91089520E030E040E251E4FC0137
:10A8D00060817181828193810E94A4E60E94A6EB2F
:10A8E0009B0177FF06C022273327261B370B8DE2FB
:10A8F00001C08BE28093490CC90168EE73E00E94AD
:10A900003AEDCB01EAE0F0E0BF010E943AED805D54
:10A9100080934A0CC90164E670E00E943AEDCB01D5
:10A92000BF010E943AED805D80934B0CC901BF01CD
:10A930000E943AED282FCB01BF010E943AED805DC5
:10A9400080934C0C8EE280934D0C205D20934E0C36
:10A9500089E49CE008958F929F92AF92BF92CF922C
:10A96000DF92EF92FF92CF9320E030E048EC52E488
:10A97000FC0160817181828193810E94A4E60E9422
:10A98000A6EB6B017C0197FD10C020E137E240E0AF
:10A9900050E00E9426EACA01B9012AE030E040E016
:10A9A00050E00E9426EA605D09C0F094E094D094E3
:10A9B000C094C11CD11CE11CF11C6DE26093490CD8
:10A9C000C701B60128EE33E040E050E00E9426EADD
:10A9D0008AE0882E912CA12CB12CCA01B901A501C5
:10A9E00094010E9426EA605D60934A0CC701B6019B
:10A9F00024E630E040E050E00E9426EACA01B901B6
:10AA0000A50194010E9426EA605D60934B0C8EE2E2
:10AA100080934C0CC701B601A50194010E9426EA5F
:10AA2000C62FCA01B901A50194010E9426EA605D02
:10AA300060934D0CC05DC0934E0C89E49CE0CF91B7
:10AA4000FF90EF90DF90CF90BF90AF909F908F904E
:10AA50000895FC0140815181852F881F8827881F18
:10AA600029F022273327241B350B01C09A01483EC9
:10AA70005340ACF0C90168EE73E00E943AEDCB019F
:10AA8000EAE0F0E0BF010E943AED805D80934B0C5C
:10AA9000C90164E670E00E943AEDCB0112C0243691
:10AAA0003105B4F0811102C080E201C08DE28093D3
:10AAB0004B0CC90164E670E00E943AEDCB01EAE07C
:10AAC000F0E0BF010E943AED805D80934C0C11C014
:10AAD00090E290934B0C90934C0C2A3031059CF0F3
:10AAE000811102C080E201C08DE280934C0CEAE04B
:10AAF000F0E0C901BF010E943AEDCB01BF010E9405
:10AB00003AED805D05C0811102C080E201C08DE296
:10AB100080934D0CC9016AE070E00E943AED805DBF
:10AB200080934E0C8BE49CE00895FC0120813181E0
:10AB300037FD0FC0243631058CF0C90164E670E0A2
:10AB40000E943AEDCB016AE070E00E943AED805D30
:10AB500006C03195219531098DE201C080E28093D4
:10AB60004C0C2A30310564F0EAE0F0E0C901BF0185
:10AB70000E943AEDCB01BF010E943AED805D01C019
:10AB800080E280934D0CC9016AE070E00E943AEDCA
:10AB9000805D80934E0C8CE49CE00895CF92DF9210
:10ABA000EF92FF926B017C0183E3C816D104E104AC
:10ABB000F10460F082E3C81AD108E108F10862E309
:10ABC00070E080E090E0CBDA21D6EECFC701B6018D
:10ABD000C6DAFF90EF90DF90CF9018C60F931F93C7
:10ABE000CF93DF93982F862F8A01D22F692F0E944F
:10ABF000EDCF9091D30F8091470C891748F1909138
:10AC0000D50F8091460C981718F1C4E1F801849192
:10AC1000882331F00E94CFD0C81B0F5F1F4FF6CFA3
:10AC2000CC2329F080E20E94E686C150F9CF8091C2
:10AC3000470C9AE79093D60F8093D70F8D2F0E94E1
:10AC4000E6D080E2DF91CF911F910F910C94E686C0
:10AC5000DF91CF911F910F91089587E59DE00E94AC
:10AC6000E8A581E080939F0608950F931F93AFDAC4
:10AC70000091AF061091B0062091B1063091B20656
:10AC8000DC01CB01801B910BA20BB30BB7FD0CC0F9
:10AC900086B186FB992790F981E08927349B8260F1
:10ACA000329B84608093AE068091AE068170909155
:10ACB000AE0691FD82609091AD06891731F1813029
:10ACC000A9F028F0823041F0833059F01CC0913057
:10ACD00089F0923099F017C0992361F0933071F0A8
:10ACE00012C0913059F0923071F404C0992331F0C0
:10ACF000933049F49091AC06915003C09091AC060A
:10AD00009F5F9093AC068093AD061F910F910895BD
:10AD10009C018091500C681778F0962FB9019093A0
:10AD2000500C42E450E086E492E00E94AFE50E94BD
:10AD30006FA883E08093400208952091500C211168
:10AD40000CC0BC0142E450E086E492E00E94C4EDF5
:10AD50000E946FA883E08093400208954F925F9213
:10AD60006F927F928F929F92AF92BF92CF92DF921B
:10AD7000EF92FF920F931F93CF93DF9300D01F9218
:10AD8000CDB7DEB710910F021F3FF1F020DAC0906F
:10AD90008E06D0908F06E0909006F0909106DC0130
:10ADA000CB018C199D09AE09BF09B7FD0DC02091DB
:10ADB000FE0F8091FD0F30E090E001968F70992793
:10ADC0002817390709F011C250DF8091AE0682FFC3
:10ADD0003EC08091AB0681113CC081E08093AB0600
:10ADE00090919E06892780939D0610929E0683E08F
:10ADF000809340021092AE06EAD9DC01CB018C5060
:10AE00009E4FAF4FBF4F8093AF069093B006A09375
:10AE1000B106B093B20680ED97E09C838B8382E30A
:10AE200090E09A838983BE016D5F7F4FCE010196CA
:10AE30000E947D8B16E0115061F08FEF9FE00E9421
:10AE4000296D62E070E080E090E089D9F4CF109243
:10AE5000AB0610910901109511708091AA06181780
:10AE6000A1F0112309F4E2C10E943B8A8091AA0655
:10AE7000823021F060E08FE29DE04ADF1093AA0665
:10AE800083E0809340020E9436D0A1D96B017C01FF
:10AE90008091A6069091A706A091A806B091A90658
:10AEA000A7019601281B390B4A0B5B0B57FF05C006
:10AEB00080919C06882309F4F4C1D701C6018C59FE
:10AEC0009F4FAF4FBF4F8093A6069093A706A093C6
:10AED000A806B093A9068091AC0618162CF48091B0
:10AEE000AC06843074F408C08091AC069927819533
:10AEF0000CF4909504972CF480919D0681119FC0CD
:10AF0000AFC080919B06882309F472C08091AC0683
:10AF1000181664F48091AC06082E000C990B97FD6E
:10AF2000039695958795959587950EC08091AC066B
:10AF3000082E000C990B97FD03969595879595958E
:10AF400087959195819591098090970690909806A4
:10AF5000A0909906B0909A0681149104A104B104BE
:10AF6000D1F1BC01990F880B990B0E9445E62B018A
:10AF70003C01C701B601681979098A099B090E9439
:10AF800043E69B01AC01C301B2010E943EEB20E00D
:10AF900030E04AE754E40E94A4E64B015C0120E063
:10AFA00030E040E253E40E9488EC87FF0FC020E0CD
:10AFB00030E046E952E4C501B4010E9488EC87FD07
:10AFC0000AC02AE030E040E050E009C024E630E06A
:10AFD00040E050E004C021E030E040E050E0C092AA
:10AFE0009706D0929806E0929906F0929A0604C0CD
:10AFF00021E030E040E050E0A091AC060A2E000CC9
:10B00000BB0B0E944CEA24E030E040E050E00E949C
:10B0100026EA8091760690917706A0917806B09105
:10B020007906820F931FA41FB51F80937606909315
:10B030007706A0937806B09379061092AC06D701F4
:10B04000C6018856954CAF4FBF4F8093A206909390
:10B05000A306A093A406B093A50682E080934002C5
:10B0600080910D0290910E028450974441F480919A
:10B070001002882309F4E5C08150809310022FB795
:10B08000F8948091920690919306A0919406B091C5
:10B0900095062FBF3AE0B695A795979587953A956F
:10B0A000D1F7009741E0A407B10520F08FEF9FEFA3
:10B0B000A0E0B0E09695879520914002211105C04F
:10B0C00030919C063111E9C053C0009741F0409186
:10B0D000A0065091A1064817590708F049C0809171
:10B0E0009C06811111C0223050F0243028F0243009
:10B0F00031F41092400203C081E0809340020E942C
:10B10000F18681E080939C0684E00E941CD081E05F
:10B110008093BF0FE0910D02F0910E0219951092ED
:10B120009D0680919C06882351F00E9435A691E0EF
:10B13000811101C090E090939C06911192C0809083
:10B14000A0069090A106A12CB12C41D8DC01CB0126
:10B150008C199D09AE09BF0988169906AA06BB0677
:10B1600038F435D86C197D097093A1066093A00658
:10B1700080910D0290910E028450974421F08091AD
:10B180009606882379F088E9C80E8AE3D81EE11C68
:10B19000F11CC092A206D092A306E092A406F092FF
:10B1A000A5060FC08091A2069091A306A091A406C7
:10B1B000B091A506C81AD90AEA0AFB0AF7FE0E944E
:10B1C000644C80919C0681116CC08091400281305A
:10B1D00049F008F466C0843008F063C081E08093D1
:10B1E00040025FC0109240025CC024E01202F001F5
:10B1F0001124EC5FFC4F20E030E040E752E4608136
:10B200007181828193810E943EEBC12C7B018C0174
:10B2100028EC34E044EC54E060EC74E08CEB94E017
:10B220000E943BBD8FEF80930F02CECD10922D1068
:10B2300010922E10823009F421CE60E082E29DE06F
:10B240001CCE8CE0809310028091A0069091A10604
:10B2500001979093A1068093A00681E0809340021D
:10B260000ECF8090A0069090A106A12CB12C0E9438
:10B27000E750DC01CB018C199D09AE09BF09881686
:10B280009906AA06BB0668F40E94E7506C197D096E
:10B290007093A1066093A00604C0009709F434CF10
:10B2A00016CF0F900F900F900F90DF91CF911F91BD
:10B2B0000F91FF90EF90DF90CF90BF90AF909F9055
:10B2C0008F907F906F905F904F9008950E9436D03E
:10B2D0003E98469A3C98449A3A98429AEAE0F1E0BD
:10B2E00080818E7F80839FB7F894EBE0F1E08081CE
:10B2F000816080839FBF82E08093AA06B6DC1092B3
:10B30000AC060895CF93DF931F921F92CDB7DEB79F
:10B3100089839A830E94444C40E050E0BA018981BD
:10B320009A810F900F90DF91CF910C94CACF2F92FA
:10B330003F924F925F926F927F928F929F92AF92C5
:10B34000BF92CF92DF92EF92FF92CF93DF9300D024
:10B350001F92CDB7DEB76090880670908906809006
:10B360005F0490906004A0906104B0906204B30107
:10B37000072C000C880B990B0E9445E6A50194014F
:10B380000E9461EA6B017C016093DD0B7093DE0B20
:10B390008093DF0B9093E00B20ED3CEC4CE45DE3FD
:10B3A00060912C0270912D0280912E0290912F02BB
:10B3B0000E94A4E61B012C012091D90B3091DA0BDD
:10B3C0004091DB0B5091DC0BC501B4010E9461EA96
:10B3D0009B01AC01C201B1010E94A4E61B012C013A
:10B3E00023E333E343E75FE36091D50B7091D60B22
:10B3F0008091D70B9091D80B0E94A4E69B01AC01E1
:10B40000C201B1010E9462EA69837A838B839C83C3
:10B410006093D50B7093D60B8093D70B9093D80B7A
:10B420008092D90B9092DA0BA092DB0BB092DC0BDE
:10B4300020E030E040E251E4C701B6010E9488EC10
:10B44000181624F481E08093D40B89C020E030E00A
:10B4500040E251ECC701B6010E943FE687FD02C001
:10B46000672821F481E08093D40B9DC08091D40B98
:10B47000882351F01092D00B1092D10B1092D20B66
:10B480001092D30B1092D40B2091280230912902F4
:10B4900040912A0250912B02C701B6010E94A4E6F6
:10B4A0002B013C016093CC0B7093CD0B8093CE0BA2
:10B4B0009093CF0B2091D00B3091D10B4091D20BB8
:10B4C0005091D30BC701B6010E9462EA4B015C01A7
:10B4D0006093D00B7093D10B8093D20B9093D30BCE
:10B4E000209130023091310240913202509133026A
:10B4F0000E94A4E69B01AC016093C80B7093C90B3A
:10B500008093CA0B9093CB0BC301B2010E9462EAF5
:10B5100029813A814B815C810E9461EA2B013C01C7
:10B5200020E030E04FE753E40E9488EC20E030E078
:10B53000A9011816DCF4C701B6010E9488EC1816A0
:10B5400074F4A7019601C501B4010E9461EA6093F9
:10B55000D00B7093D10B8093D20B9093D30B412CD3
:10B56000512C8FE7682E83E4782E20C0C301B201EE
:10B570000E943FE687FF1AC020E030E0A901C70122
:10B58000B6010E943FE687FF0EC0A7019601C501E4
:10B59000B4010E9461EA6093D00B7093D10B809349
:10B5A000D20B9093D30B412C512C3201C301B20129
:10B5B0000F900F900F900F90DF91CF91FF90EF9031
:10B5C000DF90CF90BF90AF909F908F907F906F90C3
:10B5D0005F904F903F902F90089560916304709119
:10B5E000640480916504909166040E94A6EBCB01EF
:10B5F00008952F923F924F925F926F927F928F9217
:10B600009F92AF92BF92CF92DF92EF92FF920F93F1
:10B610001F93CF93DF93EC0146EE5FE181E090E072
:10B62000FA0125913491C217D3070CF05DC09C013B
:10B6300021503109220F331F220F331FD901AC5182
:10B64000B04EFD01659174912E51304EF901A590D7
:10B65000B490FC01EE0FFF1FEE0FFF1FEC51F04EF8
:10B66000E590F490FD01C590D490FA0105911491F4
:10B67000F90125903490072E000C880B990B0E943D
:10B6800045E62B013C01CA19DB09BE01DD0F880B21
:10B69000990B0E9445E64B015C01B7016C197D09CD
:10B6A000072E000C880B990B0E9445E69B01AC010C
:10B6B000C501B4010E94A4E66B017C01B8016219C6
:10B6C0007309072E000C880B990B0E9445E69B011D
:10B6D000AC01C701B6010E943EEB9B01AC01C30166
:10B6E000B2010E9462EA11C001964C5F5F4F803444
:10B6F000910509F095CFE0EEF0E265917491072E87
:10B70000000C880B990B0E9445E6DF91CF911F91A9
:10B710000F91FF90EF90DF90CF90BF90AF909F90F0
:10B720008F907F906F905F904F903F902F900895F3
:10B73000CF92DF92EF92FF920F931F93CF93DF93FD
:10B740001F921F92CDB7DEB77C018A01809116024D
:10B75000882309F443C0E7E7F7E284916F019FEF84
:10B76000C91AD90A882341F069837A830E94008F1D
:10B77000F60169817A81F1CFFB0184916F019FEF1E
:10B78000C91AD90A882321F00E94008FF601F5CF4B
:10B79000E8E8FFE184916F019FEFC91AD90A882375
:10B7A00021F00E94008FF601F5CFF7FC0AC0B70127
:10B7B000FF0C880B990B0E946D8F8AE00E94008F0E
:10B7C0000DC0E3E8FFE184917F019FEFE91AF90AD8
:10B7D000882321F00E94008FF701F5CF8091C70BDD
:10B7E000811108C01092160281E08093C70BC80136
:10B7F0000E9455920F900F90DF91CF911F910F9162
:10B80000FF90EF90DF90CF900C9486CE4F925F9296
:10B810006F927F928F929F92AF92BF92CF92DF9260
:10B82000EF92FF920F931F9380912D1381110FC000
:10B830001F910F91FF90EF90DF90CF90BF90AF904E
:10B840009F908F907F906F905F904F9008950E948F
:10B85000ADCE0E94E7502B013C01609188067091AB
:10B860008906072E000C880B990B0E9445E6209153
:10B870005F0430916004409161045091620412E1D0
:10B88000812E912C08E2A02EB12CC12CD12C7B0151
:10B890008C016DEE7BE08BEE9BE00E9433CD80E06F
:10B8A00090E045DD4B015C01C0905F04D0906004E6
:10B8B000E0906104F09062046091AA047091AB047E
:10B8C000072E000C880B990B0E9445E69B01AC01EA
:10B8D000C701B6010E9488EC1816CCF460910902E9
:10B8E00070910A02072E000C880B990B0E9445E606
:10B8F0009B01AC01C701B6010E943FE687FF07C06C
:10B90000C501B4010E94A6EB7595679501C060E082
:10B9100060932F138091211390912213A0912313F0
:10B92000B09124130097A105B105A9F0A3019201DC
:10B93000281B390B4A0B5B0B57FD0DC00E94A3CB94
:10B940002091251330912613821793070CF4A8C079
:10B9500080E00E9453CE8091271390912813A091EC
:10B960002913B0912A130097A105B10599F0A301FD
:10B970009201281B390B4A0B5B0B57FD0BC02DDEC8
:10B9800020912B1330912C13821793070CF480C055
:10B990000E9420CE8091E70B9091E80BA091E90BDB
:10B9A000B091EA0BA3019201281B390B4A0B5B0BE8
:10B9B00057FD3ECF38E8430E33E1531E611C711C26
:10B9C0004092E70B5092E80B6092E90B7092EA0B01
:10B9D00060918C0670918D06072E000C880B990BD8
:10B9E0000E9445E62091630430916404409165040F
:10B9F00050916604EFE08E2E912CFCE3AF2EB12C1B
:10BA0000CC24CA94DC2C7B018C0161EE7BE085EEBA
:10BA10009BE00E9433CDC0906304D0906404E0901A
:10BA20006504F090660420E030E040EA50E4C7018D
:10BA3000B6010E9488EC87FD20C020E030E046E19E
:10BA400053E4C701B6010E943FE61816B4F06091B6
:10BA50008C0670918D06072E000C880B990B0E94A6
:10BA600045E69B01AC01C701B6010E943FE687FD98
:10BA70001FC080E080932E13DBCE10922E139FB751
:10BA8000F894809102018F7D809302019FBFD0CEF8
:10BA900046EA5FE165EB7FE18FEF9FEF49DE7ACF0A
:10BAA00044EC5FE163ED7FE180E090E041DE53CF65
:10BAB0008FE7E0CF880F991F880F991FFC01EF5681
:10BAC000F44F4081518162817381FC01E052FB4F50
:10BAD0004083518362837383E0918F0BF091900BCD
:10BAE00082899389A489B5898093C30B9093C40BF1
:10BAF000A093C50BB093C60B0895CF93DF932FB7D8
:10BB0000F894EC01CC0FDD1FCC0FDD1FFE01EF56CA
:10BB1000F44F60817181828193812FBF0E9445E63D
:10BB2000C053DB4F288139814A815B810E94A4E6A2
:10BB3000DF91CF9108959091FD0F8091FE0F98179E
:10BB400019F00E94BD92F7CF089580918C0B80FF71
:10BB500003C0899A8FEF02C0899881E08093110217
:10BB600080918C0B81FF03C08F988FEF02C08F9A5A
:10BB700081E08093120280918C0B9FB782FF09C0F5
:10BB8000F89480910B01826080930B019FBF8FEF2F
:10BB900008C0F89480910B018D7F80930B019FBFAB
:10BBA00081E08093130280918C0B83FF03C0169871
:10BBB0008FEF02C0169A81E080931402089590914D
:10BBC000FD0F8091FE0F981731F08091FE0F8F5F6F
:10BBD0008F708093FE0F08951F920F920FB60F92F1
:10BBE00011240BB60F92BF92CF92DF92EF92FF9289
:10BBF0000F931F932F933F934F935F936F937F9375
:10BC00008F939F93AF93BF93EF93FF93CF93DF9364
:10BC100000D01F92CDB7DEB780916E008B7F8093EE
:10BC20006E0080916F008D7F80936F007894C0903C
:10BC3000BF0BD090C00BE090C10BF090C20BC114B1
:10BC4000D104E104F10409F442C080910B02811196
:10BC500004C08091AF048823D1F10E94B671F9EB42
:10BC6000CF16FBE0DF06E104F10488F008EBC01A10
:10BC70000BE0D00AE108F108C092BF0BD092C00BD4
:10BC8000E092C10BF092C20B88EB9BE009C0C601A9
:10BC90001092BF0B1092C00B1092C10B1092C20BEE
:10BCA00090938900809388002091880030918900CA
:10BCB000809184009091850040962817390708F0FC
:10BCC0006EC0809184009091850040961FC0809145
:10BCD0008D0B90918E0B009709F494C08C0101504C
:10BCE000110910938E0B00938D0B1092900B1092F4
:10BCF0008F0B65DF012B41F487E79FE19093520C96
:10BD00008093510C0E943C7188EC90E090938900E4
:10BD10008093880044C0C8010E94268C24E630E04D
:10BD200080910B02882309F4B6C4C901293BBBE00A
:10BD30003B0708F0EAC590938900809388008091C2
:10BD4000B10B9091B20BA091B30BB091B40B820FD9
:10BD5000931FA11DB11D8093B10B9093B20BA093C3
:10BD6000B30BB093B40B209188003091890080917F
:10BD700084009091850040962817390748F48091F7
:10BD8000840090918500409690938900809388006C
:10BD9000BB2029F01092900B10928F0B10DFF894BB
:10BDA00080913013882321F080916E008B7F03C037
:10BDB00080916E00846080936E0080916F0082603D
:10BDC00080936F000F900F900F900F90DF91CF91A5
:10BDD000FF91EF91BF91AF919F918F917F916F9163
:10BDE0005F914F913F912F911F910F91FF90EF9095
:10BDF000DF90CF90BF900F900BBE0F900FBE0F90B3
:10BE00001F901895C0908F0BD090900BC114D10447
:10BE100009F0ADC19091FD0F8091FE0F981749F187
:10BE20009091FE0F1DE4919F900111242454394FED
:10BE30008091920690919306A0919406B0919506F8
:10BE4000F901E75BFF4F4081518162817381841B5F
:10BE5000950BA60BB70B8093920690939306A09335
:10BE60009406B0939506D9018C9188608C936901F2
:10BE70000BC08FB7F894109292061092930610920E
:10BE80009406109295068FBFD092900BC0928F0BA4
:10BE9000C114D10409F468C1F60152A180918C0B40
:10BEA000418158130AC0242F30E080911502082EDA
:10BEB000000C990B2817390729F050938C0B4093ED
:10BEC000150243DE1092BB0B1092BC0B1092BD0BFF
:10BED0001092BE0BD601D7968D919C91D897813444
:10BEE000BCE99B0728F48132EEE49E0748F002C0CB
:10BEF00080E49CE9969587959695879524E007C000
:10BF00008131F7E29F0730F09695879522E02093E4
:10BF1000BA0B08C021E02093BA0B8032910510F4CF
:10BF200080E290E08C0100521109011528E012070F
:10BF3000D8F0E12FFF27EE0FFF1FEE0FFF1FCF01FD
:10BF40008958944EFC01329645915491AA27059F39
:10BF50009001049F210D3A1F06942A1F3A1F1124B5
:10BF6000FC01859194911CC09801369527952C7FF2
:10BF70002958384EF90185919491F90132966591CD
:10BF80007491A80147705527649F9001659F300DFB
:10BF9000749F300D112443E0369527954A95E1F7BB
:10BFA000821B930B8436910588F48CEDE82E83E098
:10BFB000F82ED7018D917D01882319F00E94008F02
:10BFC000F8CFC8010E94268C84E690E09093B90BCC
:10BFD0008093B80B8091BA0B8093B70BF60183ADB9
:10BFE00094AD9093B60B8093B50B8134FCE99F0719
:10BFF00028F481320EE4900748F002C080E49CE906
:10C00000969587959695879524E007C0813117E22C
:10C01000910730F09695879522E02093BA0B08C0DF
:10C0200021E02093BA0B8032910510F480E290E079
:10C030008C0100521109011528E01207D8F0E12FF8
:10C04000FF27EE0FFF1FEE0FFF1FCF018958944E01
:10C05000FC01329645915491AA27059F9001049FB7
:10C06000210D3A1F06942A1F3A1F1124FC018591C5
:10C0700094911CC09801369527952C7F2958384EED
:10C08000F90185919491F901329665917491A80115
:10C0900047705527649F9001659F300D749F300D48
:10C0A000112473E0369527957A95E1F7821B930B5F
:10C0B0008436910588F45CEDE52E53E0F52ED7012A
:10C0C0008D917D01882319F00E94008FF8CFC8015F
:10C0D0000E94268C84E690E0AC0160E070E0409322
:10C0E000B10B5093B20B6093B30B7093B40B90935E
:10C0F000890080938800F60182899389A489B58993
:10C10000B695A79597958795B095A09590958195AB
:10C110009F4FAF4FBF4F8093AD0B9093AE0BA0934B
:10C12000AF0BB093B00B8093A90B9093AA0BA09385
:10C13000AB0BB093AC0B8093A50B9093A60BA09385
:10C14000A70BB093A80B8093A10B9093A20BA09385
:10C15000A30BB093A40B1092C30B1092C40B1092BC
:10C16000C50B1092C60B03C080ED97E0CFCD809138
:10C170000B028111C7C38091AF048111C3C3209109
:10C18000BA0B222309F4AFC1E0918F0BF091900B11
:10C190004091A10B5091A20B6091A30B7091A40B45
:10C1A00082819381A481B581840F951FA61FB71F3B
:10C1B0008093A10B9093A20BA093A30BB093A40B1D
:10C1C000181619061A061B060CF4889AE0918F0BB4
:10C1D000F091900B4091A50B5091A60B6091A70B8D
:10C1E0007091A80B86819781A085B185840F951FDA
:10C1F000A61FB71F8093A50B9093A60BA093A70B28
:10C20000B093A80B181619061A061B060CF48E9A82
:10C21000E0918F0BF091900B4091A90B5091AA0BDC
:10C220006091AB0B7091AC0B82859385A485B5852D
:10C23000840F951FA61FB71F8093A90B9093AA0B7D
:10C24000A093AB0BB093AC0B181619061A061B067D
:10C2500044F49FB7F89480910B01886080930B01A0
:10C260009FBFE0918F0BF091900B4091AD0B5091DF
:10C27000AE0B6091AF0B7091B00B86859785A0894E
:10C28000B189840F951FA61FB71F8093AD0B9093A4
:10C29000AE0BA093AF0BB093B00B181619061A068D
:10C2A0001B060CF4149A8091A10B9091A20BA09103
:10C2B000A30BB091A40B181619061A061B0684F5D9
:10C2C000E0918F0BF091900B4289538964897589B5
:10C2D000841B950BA60BB70B8093A10B9093A20B1D
:10C2E000A093A30BB093A40B809111024091910BEA
:10C2F0005091920B6091930B7091940B082E000C4F
:10C30000990BAA0BBB0B840F951FA61FB71F809319
:10C31000910B9093920BA093930BB093940B8898EE
:10C320008091A50B9091A60BA091A70BB091A80BA3
:10C33000181619061A061B0684F5E0918F0BF0916A
:10C34000900B4289538964897589841B950BA60BD0
:10C35000B70B8093A50B9093A60BA093A70BB0935C
:10C36000A80B809112024091950B5091960B609111
:10C37000970B7091980B082E000C990BAA0BBB0B16
:10C38000840F951FA61FB71F8093950B9093960B54
:10C39000A093970BB093980B8E988091A90B9091D6
:10C3A000AA0BA091AB0BB091AC0B181619061A068C
:10C3B0001B06BCF5E0918F0BF091900B42895389DD
:10C3C00064897589841B950BA60BB70B8093A90B09
:10C3D0009093AA0BA093AB0BB093AC0B809113027C
:10C3E0004091990B50919A0B60919B0B70919C0B13
:10C3F000082E000C990BAA0BBB0B840F951FA61FD0
:10C40000B71F8093990B90939A0BA0939B0BB093BB
:10C410009C0B9FB7F89480910B01877F80930B0151
:10C420009FBF8091AD0B9091AE0BA091AF0BB091DF
:10C43000B00B181619061A061B0684F5E0918F0B2F
:10C44000F091900B4289538964897589841B950BFF
:10C45000A60BB70B8093AD0B9093AE0BA093AF0BD5
:10C46000B093B00B8091140240919D0B50919E0BA4
:10C4700060919F0B7091A00B082E000C990BAA0BDA
:10C48000BB0B840F951FA61FB71F80939D0B909326
:10C490009E0BA0939F0BB093A00B14988091C30B9D
:10C4A0009091C40BA091C50BB091C60B0196A11D34
:10C4B000B11D8093C30B9093C40BA093C50BB09395
:10C4C000C60B2150E0918F0BF091900B428953895C
:10C4D0006489758984179507A607B70708F451CEB4
:10C4E000BB24B39401C0B12C4091C30B5091C40B39
:10C4F0006091C50B7091C60BE0908F0BF090900B84
:10C50000F70186899789A08DB18D84179507A607B5
:10C51000B70708F4C6C04091B10B5091B20B6091BF
:10C52000B30B7091B40B068D178D20A131A1AA27F2
:10C53000419FB12D529FC001629F900D619F800D60
:10C54000911D429FB00D811D9A1F519FB00D811DFD
:10C550009A1F609FB00D811D9A1F509FB10D8A1FB9
:10C560009A1FB6958A1F9A1F349F800D911D359F83
:10C57000900D112423AD34AD820F931F9093B60B11
:10C580008093B50B47A950AD61AD72ADA0E0B0E0AE
:10C59000481759076A077B0720F45093B60B40935E
:10C5A000B50B8091B50B9091B60B8134BCE99B071C
:10C5B00028F48132EEE49E0748F002C080E49CE952
:10C5C000969587959695879524E007C08131F7E287
:10C5D0009F0730F09695879522E02093BA0B08C00C
:10C5E00021E02093BA0B8032910510F480E290E0B4
:10C5F0008C0100521109011528E01207E8F0E12F23
:10C60000FF27EE0FFF1FEE0FFF1FCF018958944E3B
:10C61000FC01329625913491AA27039FA001029F25
:10C62000410D5A1F06944A1F5A1F1124FC012591DF
:10C630003491241B350B1EC0A801569547954C7F9D
:10C640004958584EFA0125913491FA013296659174
:10C650007491A80147705527649FC001659F900D94
:10C66000749F900D1124B3E096958795BA95E1F7E4
:10C67000281B390B2436310508F052CBFCEDEF2E88
:10C68000F3E0FF2ED7018D917D01882309F443CB80
:10C690000E94008FF7CF8091AF04811146CBC90172
:10C6A0004ACB4091C30B5091C40B6091C50B709164
:10C6B000C60BF701828D938DA48DB58D84179507D8
:10C6C000A607B70708F0EBC00091BB0B1091BC0B9D
:10C6D0002091BD0B3091BE0B09831A832B833C83C1
:10C6E000468D578D60A171A1AA27059FB12D169F78
:10C6F0006001269FD00C259FC00CD11C069FB00D59
:10C70000C11CDA1E159FB00DC11CDA1E249FB00D8E
:10C71000C11CDA1E149FB10DCA1EDA1EB695CA1EC0
:10C72000DA1E709FC00CD11C719FD00C1124809117
:10C73000B50B9091B60BFF96C816D90680F48C19EC
:10C740009D0940815181628173816C01E12CF12C42
:10C75000C416D506E606F70620F4CA0102C0808199
:10C76000918181341CE9910728F481322EE49207EB
:10C7700048F002C080E49CE9969587959695879548
:10C7800024E007C0813137E2930730F09695879512
:10C7900022E02093BA0B08C021E02093BA0B80322C
:10C7A000910510F480E290E08C010052110901150E
:10C7B00048E01407E8F0E12FFF27EE0FFF1FEE0F10
:10C7C000FF1FCF018958944EFC0132962591349178
:10C7D000AA27039FA001029F410D5A1F06944A1FDA
:10C7E0005A1F1124FC0125913491241B350B1EC0C6
:10C7F000C801969587958C7F8958984EFC012591A4
:10C800003491FC01329665917491A80147705527C7
:10C81000649FC001659F900D749F900D112443E0AB
:10C82000969587954A95E1F7281B390B24363105F3
:10C8300088F48CEDE82E83E0F82ED7018D917D01F0
:10C84000882319F00E94008FF8CFC8010E94268C1F
:10C8500024E630E080910B02811104C08091AF0486
:10C86000882339F0C901293BBBE03B0708F068C0C9
:10C8700001C0C901909389008093880089819A81C1
:10C88000AB81BC81820F931FA11DB11D8093BB0B97
:10C890009093BC0BA093BD0BB093BE0B64CA2091C8
:10C8A000B80B3091B90B80910B02811104C08091BB
:10C8B000AF048823F1F0293BEBE03E07D0F0C9013B
:10C8C00068EB7BE00E9426ED883E43E0940708F089
:10C8D00052C08854944FA901481B590B60E070E086
:10C8E0004093BF0B5093C00B6093C10B7093C20B6E
:10C8F0009C0130938900209388008091B70B80932E
:10C90000BA0B31CA0E94B6713ACC68EB7BE00E9448
:10C9100026ED883E03E0900780F48854944FA901E7
:10C92000481B590B60E070E04093BF0B5093C00B65
:10C930006093C10B7093C20BFEC988EB9BE0EFCFF5
:10C9400068EB7BE00E9426ED883E13E0910780F4BF
:10C950008854944FA901481B590B60E070E0409344
:10C96000BF0B5093C00B6093C10B7093C20B82CF6F
:10C9700088EB9BE0EFCF88EB9BE0ADCFCF92DF92CF
:10C98000EF92FF92CF93DF936A017B01FC018491C8
:10C99000EF012196882321F00E94008FFE01F7CF3E
:10C9A0004AE0C701B601DF91CF91FF90EF90DF9091
:10C9B000CF900C94078FCF92DF92EF92FF92CF939C
:10C9C000DF936A017B01FC018491EF0121968823AA
:10C9D00021F00E94008FFE01F7CF42E0C701B601AF
:10C9E000DF91CF91FF90EF90DF90CF900C94878FE5
:10C9F000CF92DF92EF92FF92CF93DF936A017B0198
:10CA0000FC018491EF012196882321F00E94008F80
:10CA1000FE01F7CF42E0C701B601DF91CF91FF9051
:10CA2000EF90DF90CF900C94878F80E090E0A0E2B1
:10CA3000B1E48093010C9093020CA093030CB0938B
:10CA4000040C40E050E0BA018091060C9091070C74
:10CA50000C94CACF80E090E0A0E8BFE38093010C83
:10CA60009093020CA093030CB093040C40E050E0B0
:10CA7000BA018091060C9091070C0C94CACF8DECF2
:10CA80009CECACECBDE38093010C9093020CA09362
:10CA9000030CB093040C40E050E0BA018091060C06
:10CAA0009091070C0C94CACFCF92DF92EF92FF9235
:10CAB000CF93C82F0E94E7506B017C0124EA30E736
:10CAC0004DE75FE36091010C7091020C8091030CC3
:10CAD0009091040C0E943FE687FD05C046E950E0B6
:10CAE00060E070E003C040E050E0BA01C40ED51E23
:10CAF000E61EF71EC0928E06D0928F06E092900638
:10CB0000F0929106C0930F02CF91FF90EF90DF90CB
:10CB1000CF90089580919D0681110C946B4C60918B
:10CB20007606709177068091780690917906611566
:10CB300071058105910571F10E9445E62091010C76
:10CB40003091020C4091030C5091040C0E94A4E619
:10CB50009B01AC016091C8047091C9048091CA0422
:10CB60009091CB040E9462EA6093C8047093C90458
:10CB70008093CA049093CB041092760610927706A5
:10CB8000109278061092790683E090E08DDF81E0C4
:10CB90008093400280914002882349F088EC94E021
:10CBA0000E946354BC018DE092E20C9419D1089567
:10CBB0002F923F924F925F926F927F928F929F92AD
:10CBC000AF92BF92CF92DF92EF92FF920F931F939B
:10CBD000CF93DF9300D000D0CDB7DEB720919D0674
:10CBE0002223D1F026960FB6F894DEBF0FBECDBF3C
:10CBF000DF91CF911F910F91FF90EF90DF90CF9039
:10CC0000BF90AF909F908F907F906F905F904F906C
:10CC10003F902F900C946B4C8B011C0180917606F9
:10CC200090917706A0917806B0917906892B8A2B8E
:10CC30008B2B09F497C00E94AB719801220F331F10
:10CC4000220F331F3E832D83F901E454FB4F4080B4
:10CC500051806280738080912702811115C020E08D
:10CC600030E04AE754E4C301B2010E9461EA4B019B
:10CC70005C0120E030E04AE754E4C301B2010E94C5
:10CC800062EA6B017C0110C0ED81FE81EF50F44F30
:10CC900080809180A280B380ED81FE81E55EFD4FB2
:10CCA000C080D180E280F3808091760690917706F3
:10CCB000A0917806B091790689839A83AB83BC836F
:10CCC000BC01CD010E9445E62091010C3091020C7F
:10CCD0004091030C5091040C0E94A4E69B01AC010E
:10CCE000C301B2010E9462EAAD81BE81A454BB4F70
:10CCF0003D01FD01608371838283938329813A81A1
:10CD00004B815C8157FF0DC0A50194010E943FE655
:10CD100087FF1BC0D3018D929D92AD92BC92139759
:10CD200014C029813A814B815C81232B242B252B34
:10CD300061F0A70196010E9488EC181634F4D30123
:10CD4000CD92DD92ED92FC921397C801ADDE109268
:10CD5000760610927706109278061092790681E096
:10CD60008093400280914002882329F1C801880FF6
:10CD7000991F880F991F84549B4F0E946354BC01D4
:10CD8000C10126960FB6F894DEBF0FBECDBFDF916E
:10CD9000CF911F910F91FF90EF90DF90CF90BF90B8
:10CDA000AF909F908F907F906F905F904F903F904B
:10CDB0002F900C9419D126960FB6F894DEBF0FBEB3
:10CDC000CDBFDF91CF911F910F91FF90EF90DF903A
:10CDD000CF90BF90AF909F908F907F906F905F901B
:10CDE0004F903F902F90089562E070E086E092E2CD
:10CDF000DFCE61E070E08FEF91E2DACE60E070E0CC
:10CE000088EF91E2D5CEAF92BF92CF92DF92EF92B0
:10CE1000FF920F931F93CF93DF9310929B06809105
:10CE2000760690917706A0917806B09179068130C8
:10CE30009048A105B10540F0109276061092770651
:10CE40001092780610927906C09176068091000CB7
:10CE50001816DCF4282F082E000C330B2150310952
:10CE60004C2F0C2E000C550B4217530774F0CFEFCC
:10CE7000C80F8C2F90E0A0E0B0E0809376069093EE
:10CE80007706A0937806B09379061092BA12809133
:10CE9000B912C81714F4C093B9128091B912082EB0
:10CEA000000C990B04962C2F0C2E000C330B8217C0
:10CEB000930724F48CEF8C0F8093B912D091B912A0
:10CEC00010E085EBE82E81E2F82E9FE8C92E91E272
:10CED000D92E2BEDA22E21E2B22ED11117C08091B6
:10CEE0004002882349F081E0C11180E024E043EF53
:10CEF00051E2612F0E94EE5580919D06882309F42E
:10CF00007EC0C1117CC00E946B4C75C0D130D9F479
:10CF100080914002882351F081E0C13009F080E027
:10CF200023E049EE51E2612F0E94EE5580919D066B
:10CF3000882309F464C0C13009F061C08CE090E836
:10CF40000E94825958C0D230D9F48091400288237F
:10CF500051F081E0C23009F080E020E24FED51E273
:10CF6000612F0E94EE5580919D06882309F447C0E9
:10CF7000C23009F044C0B092520CA092510C39C09A
:10CF8000D330E9F480914002882351F081E0C3302E
:10CF900009F080E020E24AEC51E2612F0E94EE5558
:10CFA00080919D06882359F1C33049F5D092520CE7
:10CFB000C092510C0E943C710E94644C1CC0D43041
:10CFC000F1F480914002882351F081E0C43009F0EF
:10CFD00080E020E249EB51E2612F0E94EE55809102
:10CFE0009D06882361F0C43051F4F092520CE09217
:10CFF000510C0E943C718091BA12811180C08091C5
:10D0000088069091890620918C0630918D06232BFD
:10D0100011F4892B31F1D53031F58091400288230C
:10D0200051F081E0C53009F080E020E24CEA51E2A5
:10D03000612F0E94EE5580919D06882309F45DC002
:10D04000C53009F05AC010928B0610928A060E94D1
:10D0500086CE0E94644C8091BA12882309F44DC098
:10D060004EC005E001C006E0D0131EC08091400212
:10D07000882349F081E0CD1380E023E040EA51E2CB
:10D08000612F0E94EE5580919D06882361F0CD139B
:10D090000AC08EE699E60E9482598091BA128111E7
:10D0A0002EC00C2F01C00D2F81E0800FD81749F042
:10D0B0001F5FDF5F153009F010CF0E5F0093000C8B
:10D0C0001EC080914002882349F081E0CD1380E0AA
:10D0D00023E044E951E2612F0E94EE5580919D06C4
:10D0E000882331F3CD13E4CF8AE898E60E94825971
:10D0F0008091BA128823E1F202C006E0D5CFDF9119
:10D10000CF911F910F91FF90EF90DF90CF90BF9044
:10D11000AF9008951F93CF93DF9310929B06809159
:10D12000760690917706A0917806B09179068130C5
:10D130009048A105B10540F010927606109277064E
:10D140001092780610927906C09176068091FF0BB6
:10D150001816DCF4282F082E000C330B215031094F
:10D160004C2F0C2E000C550B4217530774F0CFEFC9
:10D17000C80F8C2F90E0A0E0B0E0809376069093EB
:10D180007706A0937806B09379061092BA12809130
:10D19000B912C81714F4C093B9128091B912082EAD
:10D1A000000C990B04962C2F0C2E000C330B8217BD
:10D1B000930724F48CEF8C0F8093B9121091B9125D
:10D1C000D0E0111117C080914002882349F081E01E
:10D1D000C11180E024E047E851E26D2F0E94EE5536
:10D1E00080919D06882309F46DC0C1116BC00E9417
:10D1F0006B4C64C01130F9F480914002882351F0E7
:10D2000081E0C13009F080E020E24BE751E26D2F70
:10D210000E94EE5580919D06882309F453C0C130C9
:10D2200009F050C04091380C5091390C6091300C8D
:10D230007091310C1CC01230F9F4809140028823A7
:10D2400051F081E0C23009F080E020E24BE651E28B
:10D250006D2F0E94EE5580919D06882399F1C23072
:10D2600089F54091380C5091390C6FEF7FEF809128
:10D27000340C9091350C20C0133021F58091400280
:10D28000882351F081E0C33009F080E020E24BE5D3
:10D2900051E26D2F0E94EE5580919D06882391F0FA
:10D2A000C33081F44091380C5091390C6091300CAE
:10D2B0007091310C80E090E00E943D4E8091BA1256
:10D2C000811108C0DF5F1F5FD53009F07ACF84E09D
:10D2D0008093FF0BDF91CF911F9108951F93CF9300
:10D2E000DF9310929B068091760690917706A0912D
:10D2F0007806B091790681309048A105B10540F0DB
:10D30000109276061092770610927806109279069F
:10D31000C09176068091FE0B1816DCF4282F082E9B
:10D32000000C330B215031094C2F0C2E000C550BE7
:10D330004217530774F0CFEFC80F8C2F90E0A0E096
:10D34000B0E08093760690937706A0937806B0932A
:10D3500079061092BA128091B912C81714F4C093CA
:10D36000B9128091B912082E000C990B04962C2F3B
:10D370000C2E000C330B8217930724F48CEF8C0FC8
:10D380008093B9121091B912D0E0111117C0809199
:10D390004002882349F081E0C11180E024E043E5A8
:10D3A00051E26D2F0E94EE5580919D06882309F46D
:10D3B0006DC0C1116BC00E946B4C64C01130F9F498
:10D3C00080914002882351F081E0C13009F080E073
:10D3D00020E247E451E26D2F0E94EE5580919D06B8
:10D3E000882309F453C0C13009F050C04091360C75
:10D3F0005091370C60912E0C70912F0C1CC0123084
:10D40000F9F480914002882351F081E0C23009F0A4
:10D4100080E020E247E351E26D2F0E94EE558091BB
:10D420009D06882399F1C23089F54091360C5091C0
:10D43000370C6FEF7FEF8091320C9091330C20C04E
:10D44000133021F580914002882351F081E0C330F0
:10D4500009F080E020E247E251E26D2F0E94EE5594
:10D4600080919D06882391F0C33081F44091360C61
:10D470005091370C60912E0C70912F0C80E090E051
:10D480000E943D4E8091BA12811108C0DF5F1F5F7C
:10D49000D53009F07ACF84E08093FE0BDF91CF91F5
:10D4A0001F910895FF920F931F93CF93DF931092D4
:10D4B0009B068091760690917706A0917806B091B0
:10D4C000790681309048A105B10540F010927606AA
:10D4D000109277061092780610927906C09176061F
:10D4E0008091FD0B1816DCF4282F082E000C330B4E
:10D4F000215031094C2F0C2E000C550B42175307AD
:10D5000074F0CFEFC80F8C2F90E0A0E0B0E08093D4
:10D51000760690937706A0937806B09379061092DA
:10D52000BA128091B912C81714F4C093B91280913D
:10D53000B912082E000C990B04962C2F0C2E000CFF
:10D54000330B8217930724F48CEF8C0F8093B9125E
:10D550001091B912D0E0FF24F394111117C08091FB
:10D560004002882349F081E0C11180E024E042E2DA
:10D5700051E26D2F0E94EE5580919D06882309F49B
:10D58000E4C0C111E2C00E946B4CDBC0113021F538
:10D5900080914002882379F089E192E00E949555BC
:10D5A0009C0181E0C13009F080E000E04CE151E2F3
:10D5B0006D2F0E94A4E080919D06882309F4C5C0C8
:10D5C000C13009F0C2C027EE33E04AE050E069E123
:10D5D00072E086E191E2B3C0123071F580914002B1
:10D5E000882379F088E896E00E9495559C0181E0B7
:10D5F000C23009F080E000E04FE051E26D2F0E9460
:10D60000A4E080919D06882309F49FC0C23009F0F0
:10D610009CC0F0929B06109297061092980610926A
:10D62000990610929A0623EB3BE644E051E068E845
:10D6300076E088E091E22FC0133081F580914002BE
:10D64000882379F08CE896E00E9495559C0181E052
:10D65000C33009F080E000E044E051E26D2F0E9409
:10D66000A4E080919D06882309F46FC0C33009F0BF
:10D670006CC0F0929B06109297061092980610923A
:10D68000990610929A0626EB3BE647E850E06CE8D4
:10D6900076E080E091E20E94F3D753C0143061F548
:10D6A00080914002882379F08AE896E00E9495559F
:10D6B0009C0181E0C43009F080E000E046EF50E2D8
:10D6C0006D2F0E94A4E080919D068823F1F1C43063
:10D6D000E1F5F0929B061092970610929806109230
:10D6E000990610929A062FEF30E040E050E06AE889
:10D6F00076E08CEE90E223C0153039F5809140023F
:10D70000882379F087E192E00E9495559C0181E0A1
:10D71000C53009F080E000E047EE50E26D2F0E9436
:10D72000A4E080919D06882381F0C53071F427EE36
:10D7300033E04AE050E067E172E082EE90E20E945E
:10D740004EE08091BA12811108C0DF5F1F5FD530B3
:10D7500009F003CF86E08093FD0BDF91CF911F91FD
:10D760000F91FF90089580E00C9453CE0C9420CE3E
:10D77000EF92FF921F93CF93DF937C017093070C7E
:10D780006093060C10929B06809176069091770626
:10D79000A0917806B091790681309048A105B10535
:10D7A00040F010927606109277061092780610924A
:10D7B0007906C09176068091050C1816DCF4282FA6
:10D7C000082E000C330B215031094C2F0C2E000C6D
:10D7D000550B4217530774F0CFEFC80F8C2F90E012
:10D7E000A0E0B0E08093760690937706A093780649
:10D7F000B09379061092BA128091B912C81714F436
:10D80000C093B9122091B912022E000C330B2C5F79
:10D810003F4F8C2F0C2E000C990B2817390724F43E
:10D820008CEF8C0F8093B9121091B912D0E091E077
:10D8300081E0E816F10459F122E0E216F10409F45E
:10D8400048C0E114F10409F066C0111189C09923A0
:10D85000B1F01C16A4F08091760690917706A09105
:10D860007806B09179060196A11DB11D80937606C8
:10D8700090937706A0937806B0937906CF5F809156
:10D880004002882309F4D7C065E572E265C0111132
:10D8900067C09923B1F01C16A4F080917606909190
:10D8A0007706A0917806B09179060196A11DB11D69
:10D8B0008093760690937706A0937806B0937906C6
:10D8C000CF5F80914002882309F4B5C06EE472E214
:10D8D00043C0111145C09923B1F01C16A4F08091EA
:10D8E000760690917706A0917806B0917906019618
:10D8F000A11DB11D8093760690937706A0937806BC
:10D90000B0937906CF5F80914002882309F493C0D9
:10D9100067E472E221C0111123C09923B1F01C16F3
:10D92000A4F08091760690917706A0917806B09148
:10D9300079060196A11DB11D809376069093770616
:10D94000A0937806B0937906CF5F80914002882338
:10D9500009F471C06EE372E28D2F0E9490D96BC002
:10D960001130C9F480914002882351F081E0C13028
:10D9700009F080E024E044E352E26D2F0E94EE556E
:10D9800080919D06882309F456C0C13009F053C028
:10D990000E946B4C4CC01230B9F480914002882335
:10D9A00051F081E0C23009F080E023E04AE252E227
:10D9B0006D2F0E94EE5580919D068823E1F1C230C3
:10D9C000D1F585E195E631C01330B9F4809140027C
:10D9D000882351F081E0C33009F080E023E041E288
:10D9E00052E26D2F0E94EE5580919D06882319F119
:10D9F000C33009F58AE295E618C01430E1F480914D
:10DA00004002882351F081E0C43009F080E023E037
:10DA100046E152E26D2F0E94EE5580919D068823CB
:10DA200051F0C43041F48FE395E60E948259809111
:10DA3000BA12811108C0DF5F1F5F90E0D53009F096
:10DA4000F7CED093050CDF91CF911F91FF90EF900F
:10DA500008952F923F924F925F926F927F928F9292
:10DA60009F92AF92BF92CF92DF92EF92FF920F936D
:10DA70001F93CF93DF9300D000D0CDB7DEB78C01DA
:10DA80000E94E750F801C680D780E084F184C11479
:10DA9000D104E104F10409F0F6C22485222309F43B
:10DAA00060C332852150248721E0230F22874585DA
:10DAB000241301C01286F80124E0329FE00DF11D0D
:10DAC0001124C684D784E088F188F801C282D38209
:10DAD000E482F582DC01CB018C0D9D1DA11DB11DE1
:10DAE00086839783A087B18784819581892B09F4E8
:10DAF00038C3FFB7FD83F894F80122803380048196
:10DB0000158180910C02853221F08F3F09F0B8C257
:10DB100005C0E1E2FDE024912E83EDC085E2809313
:10DB20000C02E1E2FDE0E491EF3F09F4A9C2E2302A
:10DB300009F474C054F5EE2309F453C0E13009F040
:10DB4000D9C010928000109281008091810088607D
:10DB50008093810080918100816080938100EBE05F
:10DB6000FBE0E491F0E0EE0FFF1FEE54F54F8591DE
:10DB700094919093150C8093140CE1E5FBE0E491F3
:10DB8000E093130C81E08E83B9C0E43009F48EC0B9
:10DB90000CF468C0E53009F0ADC01092200110927D
:10DBA00021018091210188608093210180912101D0
:10DBB000816080932101EBE0FBE0E491F0E0EE0F67
:10DBC000FF1FEE54F54F8591949190930C0C809328
:10DBD0000B0CE1E5FBE0E491E0930A0C25E02E83D9
:10DBE0008DC014BC15BC84B5826084BD85B58160D0
:10DBF00085BDEBE0FBE0E491F0E0EE0FFF1FEE549B
:10DC0000F54F859194919093180C8093170CE1E552
:10DC1000FBE0E491E093160C1E8270C01092B000FD
:10DC20001092B1008091B00082608093B00080912A
:10DC3000B10081608093B100EBE0FBE0E491F0E0A3
:10DC4000EE0FFF1FEE54F54F85919491909370065F
:10DC500080936F06E1E5FBE0E491E093710692E0CA
:10DC60009E834CC010929000109291008091910080
:10DC700088608093910080919100816080939100F1
:10DC8000EBE0FBE0E491F0E0EE0FFF1FEE54F54F08
:10DC9000859194919093120C8093110CE1E5FBE037
:10DCA000E491E093100CE3E0EE8328C01092A00012
:10DCB0001092A1008091A10088608093A1008091C2
:10DCC000A10081608093A100EBE0FBE0E491F0E033
:10DCD000EE0FFF1FEE54F54F8591949190930F0C2A
:10DCE00080930E0CE1E5FBE0E491E0930D0CF4E091
:10DCF000FE8304C0EE838E8187FDC2C12101612CA9
:10DD0000712C61E085E20E94AC4F4801A12CB12C3E
:10DD10008E818D7F09F0BDC060E072E18AE790E0FE
:10DD2000A50194010E9426EA29833A834B835C83F0
:10DD300069017A0191E0C91AD108E108F108EFEF11
:10DD4000CE16D104E104F10409F008F44DC060E4FA
:10DD500072E48FE090E0A50194010E9426EA690137
:10DD60007A01F1E0CF1AD108E108F1082E812230C2
:10DD700001F58FEFC816D104E104F10409F008F4AD
:10DD8000EEC160E970ED83E090E0A50194010E948E
:10DD900026EA69017A0191E0C91AD108E108F1087F
:10DDA000EFEFCE16D104E104F10409F0E0F583E0D1
:10DDB00069C0FFEFCF16D104E104F104B9F0B0F06F
:10DDC00068E478EE81E090E0A50194010E9426EAE3
:10DDD00069017A0181E0C81AD108E108F1089E8141
:10DDE000992309F49AC190C181E001C082E09E812B
:10DDF0009923A1F047C089819A81AB81BC812AE037
:10DE0000B595A795979587952A95D1F76C017D01D2
:10DE1000E1E0CE1AD108E108F10885E095B5987FD8
:10DE2000892B85BDA1C068E478EE81E090E0A50172
:10DE300094010E9426EA69017A01F1E0CF1AD10823
:10DE4000E108F1082FEFC216D104E104F10409F052
:10DE500008F428C164E274EF80E090E0A501940129
:10DE60000E9426EA69017A01E1E0CE1AD108E108B0
:10DE7000F108FFEFCF16D104E104F10411F008F02E
:10DE800013C185E09091B100987F892B8093B100F8
:10DE90006BC060E072E18AE790E0A50194010E9406
:10DEA00026EA69017A01E1E0CE1AD108E108F10819
:10DEB000C114D104F1E0EF06F10488F068E478EED3
:10DEC00081E090E0A50194010E9426EA69017A01AF
:10DED00081E0C81AD108E108F10883E001C081E0BF
:10DEE0009E81913071F490918100987F892B80936D
:10DEF0008100452846284728D9F52FEF3FEFA90193
:10DF000068C0EE81E33071F490919100987F892B85
:10DF10008093910045284628472851F52FEF3FEF81
:10DF2000A90179C0FE81F43071F49091A100987F2D
:10DF3000892B8093A100452846284728C9F42FEF54
:10DF40003FEFA9017AC02E81253071F49091210113
:10DF5000987F892B8093210145284628472841F442
:10DF60002FEF3FEFA9017BC045284628472869F0DD
:10DF70009801220F331FD1010E9452EA28EE33E0AC
:10DF800040E050E00E9404EA03C02FEF3FEFA901F8
:10DF90008E81823081F12CF4882361F08130C9F0C8
:10DFA0006FC09E81943009F448C0ACF1953009F4FB
:10DFB00056C066C0C7BC2093290C30932A0C4093EE
:10DFC0002B0C50932C0C80916E00826080936E001D
:10DFD00057C0D0928900C09288002093250C3093BE
:10DFE000260C4093270C5093280C80916F00826080
:10DFF00080936F0045C0C092B300209372063093A7
:10E000007306409374065093750680917000826089
:10E010008093700035C0D0929900C09298002093F0
:10E02000210C3093220C4093230C5093240C8091AC
:10E03000710082608093710023C0D092A900C092C9
:10E04000A80020931D0C30931E0C40931F0C50937E
:10E05000200C8091720082608093720011C0D09277
:10E060002901C09228012093190C30931A0C409377
:10E070001B0C50931C0C8091730082608093730082
:10E08000ED81EFBF6EC0DC01CB018C199D09AE099B
:10E09000BF09B7FD66C04098F80116821782108646
:10E0A00011865FC084E0EECE62E17AE780E090E026
:10E0B000A50194010E9426EA69017A0181E0C81A4B
:10E0C000D108E108F1089FEFC916D104E104F10479
:10E0D000C9F0C0F089819A81AB81BC815AE0B595C5
:10E0E000A795979587955A95D1F76C017D0121E009
:10E0F000C21AD108E108F1088E81882309F48DCE77
:10E1000087E0C0CE86E073CEEFEFCE16D104E104F7
:10E11000F10409F048F684E06ACE8FEFC816D10406
:10E12000E104F104D1F0C8F062E17AE780E090E028
:10E13000A50194010E9426EA69017A01F1E0CF1A53
:10E14000D108E108F1082FEFC216D104E104F1046F
:10E1500011F008F050CE84E061CE83E05FCE82E023
:10E1600091CE26960FB6F894DEBF0FBECDBFDF91DD
:10E17000CF911F910F91FF90EF90DF90CF90BF90C4
:10E18000AF909F908F907F906F905F904F903F9057
:10E190002F900895EF92FF920F931F93CF93DF93E9
:10E1A0001F92CDB7DEB7082F162FE7E7F7E284916D
:10E1B0007F012FEFE21AF20A882331F099830E943F
:10E1C000008FF7019981F3CFE02FF92F84917F0120
:10E1D0009FEFE91AF90A882321F00E94008FF701C6
:10E1E000F5CF6091611470916214809163149091E5
:10E1F00064140E946D8F8AE00E94008F11110E94AA
:10E20000C8D71092200D10921F0D0F90DF91CF9163
:10E210001F910F91FF90EF90089520916A0430E0D4
:10E22000F901E453FB4F80832F5F3F4F2370332767
:10E2300020936A0480916E068F5F80936E06089526
:10E24000CF93FC0180818B33A1F080916E068430E6
:10E2500080F4C62FBF0180916A0420E6829FC0012E
:10E26000112483519B4F0E94AFED8C2FD6DF81E0AC
:10E2700001C080E0CF910895DF92EF92FF920F935B
:10E280001F93CF93DF93CDB7DEB76E970FB6F89499
:10E29000DEBF0FBECDBF6091510C7091520C611565
:10E2A000710501F14DE150E0CE0101967C010E9423
:10E2B000AFE51E8EF7018F010E191F09D190DD20E9
:10E2C00019F09AE0D912F7CFF701E00FF11F108291
:10E2D00060E0C701B5DF882329F0C7010E942692BC
:10E2E000811109C081E02091510C3091520C232BF7
:10E2F000A1F480E012C0DD2049F00F5F1F4F809134
:10E30000510C9091520C080F191F02C000E010E050
:10E310001093520C0093510CE5CF6E960FB6F89403
:10E32000DEBF0FBECDBFDF91CF911F910F91FF9048
:10E33000EF90DF90089528EC34E044EC54E060EC7A
:10E3400074E08CEB94E00C9497D4FC01659175918A
:10E350008591949108950E94E7506093630C7093A7
:10E36000640C8093650C9093660C08950F931F9333
:10E37000CF93DF93E0918F0BF091900B428153810B
:10E3800064817581141615061606170604F520918A
:10E390008C0B20FF1CC03CB12091090C32953695A6
:10E3A000377041E03427832F81702E7F822B80933A
:10E3B000090C9091080C9170892349F08091EC042C
:10E3C00081608093EC0480E090E00E945A5DE091CF
:10E3D0008F0BF091900B86819781A085B1851816DF
:10E3E00019061A061B0654F580918C0B81FF26C076
:10E3F000809103012091090C422F50E0869591E015
:10E400008927082F017010E022273327201B310BAA
:10E410002427352722703327242735272093090CFA
:10E420008091080C8270282349F08091EC0482606E
:10E430008093EC0481E090E00E945A5DE0918F0BA4
:10E44000F091900B82859385A485B58518161906E1
:10E450001A061B068CF580918C0B82FF2DC08091D3
:10E46000AF04882349F199B18091090C282F30E03D
:10E47000892F86958695869591E089278170C82F8A
:10E4800080E0D82F882799278C1B9D0B8227932704
:10E4900084709927822793278093090C9091080C08
:10E4A0009470892349F08091EC0484608093EC049B
:10E4B00082E090E00E945A5D8091090C8093080CE4
:10E4C000DF91CF911F910F910895CF93DF93E3EBED
:10E4D000F4E28491EF012196882321F00E94008FBD
:10E4E000FE01F7CFEBEAF4E28491EF012196882355
:10E4F00021F00E94008FFE01F7CF659B03C0C0EFA3
:10E50000D3E002C0C5EFD3E08991882319F00E94BF
:10E51000008FFACF8AE00E94008FE3EAF4E2849150
:10E52000EF012196882321F00E94008FFE01F7CF92
:10E530008091030181FF03C0C0EFD3E002C0C5EFAB
:10E54000D3E08991882319F00E94008FFACF8AE0E6
:10E550000E94008FEBE9F4E28491EF012196882379
:10E5600021F00E94008FFE01F7CF4B9B03C0C0EF4C
:10E57000D3E002C0C5EFD3E08991882319F00E944F
:10E58000008FFACF8AE0DF91CF910C94008FAF9289
:10E59000BF92CF92DF92EF92FF920F931F93CF9390
:10E5A000C82F882319F0E5E8F4E20CC0EEE7FCE29E
:10E5B00084918F010F5F1F4F8823A9F30E94008F62
:10E5C000F801F6CF84918F010F5F1F4F882321F050
:10E5D0000E94008FF801F6CF8AE00E94008FC111DF
:10E5E0002CC0EEE7FCE284918F010F5F1F4F882360
:10E5F00021F00E94008FF801F6CFE2E7F4E2849167
:10E600008F010F5F1F4F882321F00E94008FF801B8
:10E61000F6CF8091B812882321F08AE00E94008F03
:10E620003AC0E7E6F4E284918F010F5F1F4F882321
:10E6300091F10E94008FF801F6CF4091890250912C
:10E640008A0260918B0270918C028EE594E20E94A6
:10E65000F8648AE00E94008F8091B812811127C06F
:10E66000CC2319F0E3E5F4E20CC0EEE7FCE2849180
:10E670008F010F5F1F4F8823A9F30E94008FF801BD
:10E68000F6CF84918F010F5F1F4F882381F00E9486
:10E69000008FF801F6CFEEE7FCE284918F010F5F67
:10E6A0001F4F882351F20E94008FF801F6CFC1114D
:10E6B00024C0EEE7FCE284918F010F5F1F4F882397
:10E6C00021F00E94008FF801F6CFE2E4F4E2849199
:10E6D0008F010F5F1F4F882321F00E94008FF801E8
:10E6E000F6CFEEE7FCE284918F010F5F1F4F882386
:10E6F00021F00E94008FF801F6CF4091BD12509199
:10E70000BE126091BF127091C0128AE394E20E941F
:10E71000F8644091C1125091C2126091C31270917D
:10E72000C41287E394E20E94F8644091C5125091AC
:10E73000C6126091C7127091C81284E394E20E94DD
:10E74000F8644091C9125091CA126091CB12709135
:10E75000CC1281E394E20E94F8648AE00E94008F68
:10E76000C11124C0EEE7FCE284918F010F5F1F4FBF
:10E77000882321F00E94008FF801F6CFE3E1F4E254
:10E7800084918F010F5F1F4F882321F00E94008F1B
:10E79000F801F6CFEEE7FCE284918F010F5F1F4F87
:10E7A000882321F00E94008FF801F6CF4091ED12EE
:10E7B0005091EE126091EF127091F0128AE094E2A3
:10E7C0000E94F8644091F1125091F2126091F3129C
:10E7D0007091F41287E094E20E94F8644091F5127F
:10E7E0005091F6126091F7127091F81284E094E261
:10E7F0000E94F8644091F9125091FA126091FB1254
:10E800007091FC1281E094E20E94F8648AE00E9418
:10E81000008FC11124C0EEE7FCE284918F010F5FED
:10E820001F4F882321F00E94008FF801F6CFEFEDF3
:10E83000F3E284918F010F5F1F4F882321F00E9424
:10E84000008FF801F6CFEEE7FCE284918F010F5FB5
:10E850001F4F882321F00E94008FF801F6CF4091CE
:10E86000D5125091D6126091D7127091D81286EDC0
:10E8700093E20E94BE644091D9125091DA126091E5
:10E88000DB127091DC1283ED93E20E94BE64409132
:10E89000DD125091DE126091DF127091E01280ED76
:10E8A00093E20E94BE644091E1125091E2126091A5
:10E8B000E3127091E4128DEC93E20E94BE648AE050
:10E8C0000E94008FC11124C0EEE7FCE284918F0109
:10E8D0000F5F1F4F882321F00E94008FF801F6CFB1
:10E8E000E3E8F3E284918F010F5F1F4F882321F04B
:10E8F0000E94008FF801F6CFEEE7FCE284918F01D1
:10E900000F5F1F4F882321F00E94008FF801F6CF80
:10E9100040910D1350910E1360910F1370911013CD
:10E920008AE793E20E94F8644091D1125091D2128A
:10E930006091D3127091D41287E793E20E94F86439
:10E940004091CD125091CE126091CF127091D012A1
:10E9500084E793E20E94F8648AE00E94008FC1116C
:10E9600024C0EEE7FCE284918F010F5F1F4F8823E4
:10E9700021F00E94008FF801F6CFE0E0F3E28491ED
:10E980008F010F5F1F4F882321F00E94008FF80135
:10E99000F6CFEEE7FCE284918F010F5F1F4F8823D3
:10E9A00021F00E94008FF801F6CF4091E9125091BA
:10E9B000EA126091EB127091EC1287EF92E20E94E2
:10E9C000F8644091E5125091E6126091E71270915F
:10E9D000E81284EF92E20E94F8644091171350917C
:10E9E00018136091191370911A1381EF92E20E942B
:10E9F000BE644091FD125091FE126091FF12709121
:10EA000000138EEE92E20E94F8644091011350913F
:10EA1000021360910313709104138BEE92E20E9433
:10EA2000F86440910513509106136091071370919B
:10EA3000081388EE92E20E94F86440910913509105
:10EA40000A1360910B1370910C1385EE92E20E94F1
:10EA5000F8648AE00E94008FC11124C0EEE7FCE256
:10EA600084918F010F5F1F4F882321F00E94008F38
:10EA7000F801F6CFE7EDF2E284918F010F5F1F4FAF
:10EA8000882321F00E94008FF801F6CFEEE7FCE228
:10EA900084918F010F5F1F4F882321F00E94008F08
:10EAA000F801F6CF4091B0045091B1046091B204E6
:10EAB0007091B3048EEC92E20E94F8644091B40429
:10EAC0005091B5046091B6047091B7048BEC92E25A
:10EAD0000E94F8644091B8045091B9046091BA045E
:10EAE0007091BB0488EC92E20E94F8648AE00E9474
:10EAF000008FCC2379F082E3A82E8CE0B82E9EE222
:10EB0000C92E9CE0D92E26E3E22E2CE0F22E00E066
:10EB100010E024C0EEE7FCE284918F010F5F1F4FED
:10EB2000882321F00E94008FF801F6CFEBEAF2E291
:10EB300084918F010F5F1F4F882321F00E94008F67
:10EB4000F801F6CFEEE7FCE284918F010F5F1F4FD3
:10EB5000882389F20E94008FF801F6CFB80182EA7B
:10EB600092E2B9D0F501619171915F018FE992E272
:10EB7000B2D0F601619171916F018CE992E2ABD054
:10EB8000F701619171917F0189E992E2A4D08AE055
:10EB90000E94008F0130110519F001E010E0DECF76
:10EBA000C11124C0EEE7FCE284918F010F5F1F4F7B
:10EBB000882321F00E94008FF801F6CFEAE8F2E204
:10EBC00084918F010F5F1F4F882321F00E94008FD7
:10EBD000F801F6CFEEE7FCE284918F010F5F1F4F43
:10EBE000882321F00E94008FF801F6CF409128027F
:10EBF0005091290260912A0270912B0281E892E2E1
:10EC00000E94F8642CEA35EC47E25EE36091300242
:10EC10007091310280913202909133020E943EEB5A
:10EC2000AB01BC018EE792E20E94DB642CEA35EC7A
:10EC300047E25EE360912C0270912D0280912E02DA
:10EC400090912F020E94A4E6AB01BC018BE792E2F7
:10EC50000E94DB648AE00E94008FC11124C0EEE7AD
:10EC6000FCE284918F010F5F1F4F882321F00E94E7
:10EC7000008FF801F6CFE5E6F2E284918F010F5F95
:10EC80001F4F882321F00E94008FF801F6CFEEE796
:10EC9000FCE284918F010F5F1F4F882321F00E94B7
:10ECA000008FF801F6CF409111135091121360912B
:10ECB0001313709114138CE592E20E94F8648AE0B9
:10ECC000CF911F910F91FF90EF90DF90CF90BF9069
:10ECD000AF900C94008F0F931F93CF93DF938B0112
:10ECE000FC018491EF012196882321F00E94008F7E
:10ECF000FE01F7CFB801110F880B990BDF91CF916F
:10ED00001F910F910C946D8F0F931F93CF93DF93EF
:10ED10001F921F92CDB7DEB7FC0184918F010F5F68
:10ED20001F4F811102C08B0108C069837A830E9442
:10ED3000008FF80169817A81F0CFF80181918F010C
:10ED4000882319F00E94008FF8CF0F900F90DF9169
:10ED5000CF911F910F910895CF938091960F8823A3
:10ED6000B9F140918E0F50918F0F6091900F70917B
:10ED7000910F2EE83DE08091970F9091980F0E949F
:10ED800070D3C82F811102C0C0E023C04091920F00
:10ED90005091930F6091940F7091950F411551050B
:10EDA0006105710591F02EE83DE08091970F9091FB
:10EDB000980F0E9470D3882339F31092920F10920B
:10EDC000930F1092940F1092950F1092960F01C00E
:10EDD000C1E08C2FCF910895CF92DF92EF92FF92F6
:10EDE000CF936B017C01C42F80918E0F90918F0F78
:10EDF000A091900FB091910F8C159D05AE05BF05A8
:10EE0000C9F0AADF811102C080E018C02EE83DE001
:10EE1000B701A6018091970F9091980F0E94D2D3CD
:10EE2000882391F3C0928E0FD0928F0FE092900FB3
:10EE3000F092910F81E0C1118093960FCF91FF90D6
:10EE4000EF90DF90CF9008954F925F926F927F92F4
:10EE50008F929F92AF92BF92CF92DF92EF92FF92EA
:10EE60000F931F93CF93DF93EC016A017B0128017D
:10EE70003901423051056105710510F480E064C02C
:10EE800089859A85AB85BC850196A11DB11D841726
:10EE90009507A607B70790F38F89803149F48D2C29
:10EEA0009E2CAF2CBB248B899C89AD89BE890FC059
:10EEB000803221F78B889C88AD88BE88DB01CA012F
:10EEC00057E0B695A795979587955A95D1F7880EEF
:10EED000991EAA1EBB1E41E0C501B4017DDF882337
:10EEE00069F29F89903161F4DD24EE24FF249601BC
:10EEF000220F331FF901E257F24F5182408211C0B5
:10EF0000E894C7F8DD24EE24FF249601220F331F76
:10EF1000220F331FF901E257F24F40825182628281
:10EF200073829A89923080F04D815E816F817885FD
:10EF3000840E951EA61EB71E8092920F9092930F7C
:10EF4000A092940FB092950FDF91CF911F910F91E6
:10EF5000FF90EF90DF90CF90BF90AF909F908F90F9
:10EF60007F906F905F904F900895CF92DF92EF92D5
:10EF7000FF920F931F93CF93DF93FC0181859285BE
:10EF8000A385B4850196A11DB11D84179507A60719
:10EF9000B70710F480E061C08789803149F4BB274E
:10EFA000A72F962F852FC388D488E588F6880FC0B1
:10EFB000803281F783899489A589B6896A017B01AA
:10EFC000C7E0F694E794D794C794CA95D1F78C0D0F
:10EFD0009D1DAE1DBF1DE9016A017B018F0140919E
:10EFE0008E0F50918F0F6091900F7091910F841739
:10EFF0009507A607B70799F4F80187898031B1F41E
:10F00000B701A601552766277727440F551FFA0138
:10F01000E257F24F80819181A0E0B0E019C040E05A
:10F02000BC01CD01D9DE8111E7CFB4CFB701A60174
:10F030004F77552766277727440F551F440F551FD5
:10F04000FA01E257F24F80819181A281B381BF70B2
:10F0500088839983AA83BB8381E0DF91CF911F913D
:10F060000F91FF90EF90DF90CF9008954F925F92B5
:10F070006F927F92AF92BF92CF92DF92EF92FF9208
:10F080000F931F93CF93DF9300D01F92CDB7DEB7BE
:10F090008C0149835A836B837C835901C12CD12C09
:10F0A0007601412C82E0582E612C712C49815A81C5
:10F0B0006B817C819E012F5F3F4FC80156DF882303
:10F0C00041F1D301C201F801058404C0880F991FE2
:10F0D000AA1FBB1F0A94D2F7C80ED91EEA1EFB1E38
:10F0E00049815A816B817C818789803139F481E043
:10F0F000483F5F4F6105710538F4D8CF81E0483F44
:10F100005F4F6F4F7F4090F2F501C082D182E28263
:10F11000F3820F900F900F900F90DF91CF911F917E
:10F120000F91FF90EF90DF90CF90BF90AF907F90C6
:10F130006F905F904F900895CF93DF93EC018B8198
:10F14000882331F1898187FF20C061E0CE010E94D0
:10F15000B5D1FC01892BE1F08081853EC9F08B811E
:10F16000823040F489899A89AB89BC89848F958FD4
:10F17000A68FB78F8D899E89AF89B88D938F828F27
:10F18000B58BA48B89818F778983DF91CF91E4CD73
:10F1900081E0888380E0DF91CF9108958F929F92E4
:10F1A000AF92BF92CF92DF92EF92FF920F931F9395
:10F1B000CF93DF93EC018B81811102C080E076C098
:10F1C00009891A892B893C890417150726073707EF
:10F1D000A8F36A017B01823029F4C886D986EA86C1
:10F1E000FB860DC0C114D104E104F10451F41C826A
:10F1F0001D821E821F82188619861A861B8681E050
:10F2000055C088849984AA84BB84E98DFA8D2585AC
:10F2100030E0275F3F4FB501A4014150510961091A
:10F220007109022E04C076956795579547950A9403
:10F23000D2F7D701C6010197A109B10904C0B6955B
:10F24000A795979587952A95D2F784179507A607CE
:10F25000B70720F089288A288B2849F44D895E89D0
:10F260006F89788D4C835D836E837F8304C0841B9C
:10F27000950BA60BB70B4C015D018E010C5F1F4F68
:10F2800081149104A104B10409F4A7CF4C815D81DC
:10F290006E817F819801898D9A8D67DE91E0891A50
:10F2A0009108A108B1088111EBCF88CFDF91CF91F0
:10F2B0001F910F91FF90EF90DF90CF90BF90AF9094
:10F2C0009F908F9008952F923F924F925F926F92EE
:10F2D0007F928F929F92AF92BF92CF92DF92EF92E6
:10F2E000FF920F931F93CF93DF9300D01F92CDB760
:10F2F000DEB78C014B011A01DC0113968C91139738
:10F300008130C1F411968C9181FF14C082FF18C026
:10F31000F801418952896389748980859185A28524
:10F32000B38584179507A607B70751F0C80136DFE4
:10F33000811106C081E0F80180838FEF9FEF2CC11F
:10F34000610185C0D80159968D919C915A97FC0115
:10F35000248121502A013B0139E076946794579427
:10F3600047943A95D1F7722E74207A01F1E0FF228A
:10F37000772009F478C080E092E08E199F09560149
:10F380008C159D0508F45C01D80159962D913C918E
:10F390005A9714968D919D910D90BC91A02D029736
:10F3A000A109B109F901058404C0880F991FAA1F9A
:10F3B000BB1F0A94D2F74685578560897189840FEF
:10F3C000951FA61FB71F9C01AD01270D311D411DC3
:10F3D000511D29013A01A11432E0B30609F089C098
:10F3E00080918E0F90918F0FA091900FB091910FFF
:10F3F00084159505A605B70569F41092960F8FEF51
:10F400009FEFDC0180938E0F90938F0FA093900F4E
:10F41000B093910F9401B301A2018091970F909145
:10F42000980F0E9470D3882309F484CFF801808557
:10F430009185A285B3858A0D9B1DA11DB11D808775
:10F440009187A287B3878A0C9B1CCA18DB08D80156
:10F4500018964D915D916D917C911B97C114D104CB
:10F4600009F070CF7AC0E114F10409F084CF14964A
:10F470004D915D916D917C911797411551056105F5
:10F48000710559F455968D919D910D90BC91A02DCB
:10F490000097A105B10539F520C09E012F5F3F4FB0
:10F4A00064DD882309F446CF89819A81AB81BC81D0
:10F4B000F801218D328DF9012789203139F4883FF7
:10F4C000FFEF9F07A105B10540F40DC0883F2FEF66
:10F4D0009207A2072FE0B20730F0C8010E94D1D1F5
:10F4E000811149CF27CFF80184839583A683B78301
:10F4F00042CFE114F10411F5D80118964D915D91B8
:10F500006D917C911B9751968D919D910D90BC9121
:10F51000A02D481759076A077B0780F01DDC882358
:10F5200009F408CF81E08093960F40928E0F50929D
:10F530008F0F6092900F7092910F07C041E0C3014E
:10F54000B2014ADC882309F4F5CEA501B401C70154
:10F550008257924F0E9474ED69CF51968D919D9183
:10F560000D90BC91A02D84179507A607B70740F40E
:10F57000F801418B528B638B748B8181806881830E
:10F58000D80111968C9183FD02C0C10105C0C8014C
:10F59000D3DD8111FACFCECE0F900F900F900F9048
:10F5A000DF91CF911F910F91FF90EF90DF90CF905F
:10F5B000BF90AF909F908F907F906F905F904F9093
:10F5C0003F902F900895CF93DF931F92CDB7DEB772
:10F5D000698341E050E0BE016F5F7F4F049673DEA8
:10F5E0000F90DF91CF9108952F923F924F925F92AB
:10F5F0006F927F928F929F92AF92BF92CF92DF9243
:10F60000EF92FF920F931F93CF93DF9300D01F923F
:10F61000CDB7DEB79C838B834B015A01DC01139677
:10F620008C91811103C08FEF9FEFE9C0EB81FC81CA
:10F63000818180FFF8CFAB81BC8151960D911D91E6
:10F640002D913C91549718964D915D916D917C91BF
:10F650001B97C501A0E0B0E068017901C41AD50A82
:10F66000E60AF70AC816D906EA06FB0618F4580196
:10F67000A41AB50A75018B819C8104969A838983AB
:10F68000612C92E0792EE114F10409F48AC0AB8177
:10F69000BC8118964D915D916D917C911B976A018B
:10F6A000B1E0DB22EB81FC8123811A012B0189E08F
:10F6B00056944794379427948A95D1F7818D928DEB
:10F6C000223061F4FC01828D938DA48DB58DBC0137
:10F6D000CD01620D731D841D951D49C0DC0114967A
:10F6E0001C9111501221C114D104F9F411111DC043
:10F6F000452B462B472B59F4EB81FC818589968954
:10F70000A789B08D84839583A683B7830EC0AB8110
:10F71000BC8114964D915D916D917C9117972981D3
:10F720003A8123DC882309F47ECFEB81FC81218D93
:10F73000328D84819581A681B7810297A109B10993
:10F74000F901058404C0880F991FAA1FBB1F0A94E2
:10F75000D2F74685578560897189840F951FA61F4A
:10F76000B71FBC01CD01610F711D811D911D93015A
:10F770002C193D0987012E153F0508F48901011553
:10F78000F2E01F0779F520918E0F30918F0F409195
:10F79000900F5091910F621773078407950719F422
:10F7A00021C0C5012CC09401AB01BC018091970F11
:10F7B0009091980F0E94D2D3882309F434CF800E01
:10F7C000911EEB81FC8180859185A285B385800F98
:10F7D000911FA11DB11D80879187A287B387E01A71
:10F7E000F10A51CF40E0F8DA882309F41CCFB601C2
:10F7F0006257724FA801C4010E9474EDE0CF0F90D0
:10F800000F900F900F90DF91CF911F910F91FF906C
:10F81000EF90DF90CF90BF90AF909F908F907F90B0
:10F820006F905F904F903F902F900895DF92EF92EE
:10F83000FF920F931F93CF93DF937C01EB018A011B
:10F840008DE0D82E40E250E0BE01C701CDDE80320F
:10F85000910539F021E0892B09F420E0822F819570
:10F860003EC02881222399F1253E61F32E3251F3C7
:10F870000115110541F13B853F733F3021F54A8D5C
:10F880005B8D452B01F52F713FEF320F3230D8F4ED
:10F8900030E021503109D29EC001D39E900D112439
:10F8A000D801A80FB91FFE0120E0AD01253088F472
:10F8B00031813D932F5F32962D30C1F7288126FF8D
:10F8C00002C0FA0115862B8523FDBCCF08C080E05D
:10F8D00006C02B3010F43481ECCF3681EACFDF91B3
:10F8E000CF911F910F91FF90EF90DF9008954F926D
:10F8F0005F926F927F92AF92BF92CF92DF92EF9220
:10F90000FF920F931F93CF93DF931F92CDB7DEB774
:10F910008C017B015A01D22EDB0159968D919C916D
:10F920005A97F801928F818F40E050E0BA01C701E9
:10F9300035DCC12CF70180859185A285B38541898D
:10F9400052896389748984179507A607B70708F059
:10F9500062C025E0B695A795979587952A95D1F72A
:10F96000F82FFF707F2ED70113968C91823008F408
:10F9700063C041E050E0BE016F5F7F4FC70134DEDE
:10F98000019719F4898190E002C08FEF9FEF0196F3
:10F9900009F452C0F70180859185A285B3854F9601
:10F9A000A11DB11D80879187A287B387F0E27F9E5A
:10F9B000C0011124BC016257724F61157105E1F15C
:10F9C000DB012C91222319F0253ED1F465C1C11031
:10F9D0000EC040918E0F50918F0F6091900F7091DB
:10F9E000910FF8014487558766877787708AFC01F5
:10F9F000E257F24F8081882361F0CC24C3949ACFE0
:10FA00004BE050E0C5010E9467ED892B09F092CFD1
:10FA100015C0CC24C3948D2D8274823469F4CC201B
:10FA200009F489C0D80150967C9061E0C8010E9419
:10FA3000B5D1009709F005C180E031C1D7FCFCCFFA
:10FA4000F0E27F9EA00111249A012257324FD90182
:10FA50001B968C91817121F08D2D827109F067C008
:10FA600080918E0F90918F0FA091900FB091910F78
:10FA7000F80184879587A687B787708AFA01E257CD
:10FA8000F24F4489558960E070E0BA015527442758
:10FA9000D80155964D935D936D937C935897828DC5
:10FAA000938DA0E0B0E0482B592B6A2B7B2BD8011B
:10FAB00055964D935D936D937C935897D9011B9602
:10FAC0008C91887159F4848D958DA68DB78DF80130
:10FAD000818B928BA38BB48B81E00FC0803139F581
:10FAE00098012F5E3F4FD80159968D919C915A975E
:10FAF000BDDA8823E1F084E0F80183838D2D8F70D7
:10FB0000D80111968C931197F801148215821682F0
:10FB1000178218961D921D921D921C921B97D4FE5F
:10FB2000AFC0C8010E948EA88111AAC085CFD8019C
:10FB300013961C9281CFF7018381823009F47CCF28
:10FB400081899289A389B489803E9F4FAF41B105D5
:10FB500008F072CFC7010E94D1D1882309F46CCF7D
:10FB6000FBD8882309F468CFD70159962D913C9191
:10FB70005A9714968D919D910D90BC91A02D02974E
:10FB8000A109B109F901058404C0880F991FAA1FB2
:10FB9000BB1F0A94D2F74684578460887188480E48
:10FBA000591E6A1E7B1E81E08093960F40928E0F35
:10FBB00050928F0F6092900F7092910F80E092E0C0
:10FBC000EEE8FDE0DF019C011D9221503040E1F79D
:10FBD000CC24C394D7015996ED91FC915A97848116
:10FBE000C81698F42EE83DE0B301A2014C0D511D5A
:10FBF000611D711D8091970F9091980F0E9470D395
:10FC0000882309F419CFC394E5CF80E092E0A0E007
:10FC1000B0E0058404C0880F991FAA1FBB1F0A9477
:10FC2000D2F7F7014189528963897489840F951F3E
:10FC3000A61FB71F818B928BA38BB48B8EE89DE0A0
:10FC4000712C20E2DC011D922A95E9F72BE0F501E9
:10FC5000DC0101900D922A95E1F721E238E2FC01E6
:10FC6000318B208B40E058E057874687338B228BBF
:10FC7000318F208F578B468B6FD88111E1CEDCCE30
:10FC8000D5FE08C0F8014189528963897489C80189
:10FC900085DA05C081E003C0C110AFCE9ACE0F90C7
:10FCA000DF91CF911F910F91FF90EF90DF90CF9058
:10FCB000BF90AF907F906F905F904F9008950F939B
:10FCC0001F93CF93DF93FC012381222311F080E067
:10FCD00043C08B01EC01FB018789803131F1803217
:10FCE000B1F783E08B83F801428D538D648D758D60
:10FCF0004D8B5E8B6F8B788F9E012F5E3F4FC801BF
:10FD0000B5D9882321F31A8F098F81E089831C825A
:10FD10001D821E821F82188619861A861B861C86E3
:10FD20001D861E861F86188A17C082E08B831D8A57
:10FD30001E8A1F8A188EFB01808D918DA0E0B0E095
:10FD400025E0880F991FAA1FBB1F2A95D1F7898B21
:10FD50009A8BAB8BBC8BD7CFDF91CF911F910F913B
:10FD60000895CF93DF93EB01FC012381211102C0A1
:10FD700080E028C02250223020F48FE2888319824C
:10FD800020C060E00E94B5D1009791F3FC0190E0A3
:10FD900080E02EE23081303269F0883029F4DE01D3
:10FDA000A90FB11D2C939F5FDE01A90FB11D3081FA
:10FDB0003C939F5F8F5F31968B3061F7C90FD11DE8
:10FDC000188281E0DF91CF910895CF93DF93EC010A
:10FDD000B3D91B82DF91CF9108952F923F924F921A
:10FDE0005F926F927F928F929F92AF92BF92CF92CB
:10FDF000DF92EF92FF920F931F93CF93DF93CDB7D4
:10FE0000DEB7C554D1090FB6F894DEBF0FBECDBF23
:10FE10003C015B018A01322E1C8E1F8E19821C82CE
:10FE2000672B11F410E0A7C0FC0183818111FACF88
:10FE3000FA0180818F3261F4CA018C010196F801C8
:10FE400020812F32D1F3F50183818250823010F46A
:10FE500075010AC0618D728DCE01019630DF882355
:10FE600009F3CE0101967C016E019CE1C90ED11C03
:10FE700026014E01E7E38E0E911CFBE0F80D25965E
:10FE8000FFAF2597CE01019624969FAF8EAF2497A2
:10FE90002696CFAE26972D2C35C080E281932596ED
:10FEA0009FAD25979E13F9CFD80190E027E04A2F08
:10FEB0003B2F8D91811128C08FA9803209F4B2CFD8
:10FEC000842F932F8C01FC01208101962F32D1F3D6
:10FED000222309F44AC021E0A401B701C60107DDCD
:10FEE000882309F49FCFEA14FB0411F0C7016DDFEA
:10FEF000C414D50499F126969FAD2697822D7601DC
:10FF0000C92ED82EF401C9CF8F32B1F28E3219F03A
:10FF1000EDECF4E20AC02A3009F484CF98E02AE03C
:10FF2000C6CF3196381709F47DCF34913111F9CF0E
:10FF3000291708F477CF813208F474CF8F3709F48A
:10FF400071CF31E0390FF401E90FF11D9FE9980FEE
:10FF50009A3108F480528083932FA9CF23969FADC6
:10FF6000239724968FAD2497CACF232DA401B701E0
:10FF7000C301BDDC182FCE0101960E941DB4CE0135
:10FF80004C960E941DB4812FCB5BDF4F0FB6F894C7
:10FF9000DEBF0FBECDBFDF91CF911F910F91FF90BC
:10FFA000EF90DF90CF90BF90AF909F908F907F9019
:10FFB0006F905F904F903F902F9008952CEA35EC12
:10FFC00047E25EE360913C0C70913D0C80913E0CE9
:10FFD00090913F0C0E943EEB60932C0270932D0297
:10FFE00080932E0290932F0208952CEA35EC47E27D
:10FFF0005EE36091400C7091410C8091420C9091B5
:020000021000EC
:10000000430C0E94A4E66093300270933102809307
:1000100032029093330208951F93CF93DF9310928F
:100020009B068091760690917706A0917806B09114
:10003000790681309048A105B10540F0109276060E
:10004000109277061092780610927906C091760683
:1000500080913A0C1816DCF4282F082E000C330B74
:10006000215031094C2F0C2E000C550B4217530711
:1000700074F0CFEFC80F8C2F90E0A0E0B0E0809339
:10008000760690937706A0937806B093790610923F
:10009000BA128091B912C81714F4C093B9128091A2
:1000A000B912082E000C990B04962C2F0C2E000C64
:1000B000330B8217930724F48CEF8C0F8093B912C3
:1000C0001091B912D0E0111117C08091400288231D
:1000D00049F081E0C11180E024E04BEF54E26D2F44
:1000E0000E94EE5580919D06882309F470C0C111CD
:1000F0006EC00E946B4C67C01130C9F48091400201
:10010000882351F081E0C13009F080E023E044EF22
:1001100054E26D2F0E94EE5580919D06882309F4CC
:1001200056C0C13009F053C087E695E84AC0123086
:10013000B9F480914002882351F081E0C23009F087
:1001400080E023E04DEE54E26D2F0E94EE55809149
:100150009D068823E1F1C230D1F58DE695E831C0E6
:100160001330B9F480914002882351F081E0C3300C
:1001700009F080E023E046EE54E26D2F0E94EE5538
:1001800080919D06882319F1C33009F583E795E82E
:1001900018C01430E1F480914002882351F081E0CE
:1001A000C43009F080E023E04DED54E26D2F0E9451
:1001B000EE5580919D06882351F0C43041F489E7C3
:1001C00095E80E9482598091BA12811107C0DF5FC1
:1001D0001F5FD53009F077CFD0933A0CDF91CF91E4
:1001E0001F9108953F924F925F926F927F928F92EC
:1001F0009F92AF92BF92CF92DF92EF92FF920F93B6
:100200001F93CF93DF9310929B0680917606909177
:100210007706A0917806B091790681309048A105C3
:10022000B10540F01092760610927706109278068B
:1002300010927906C09176068091440C1816DCF471
:10024000282F082E000C330B215031094C2F0C2E77
:10025000000C550B4217530774F0CFEFC80F8C2FCB
:1002600090E0A0E0B0E08093760690937706A093AC
:100270007806B09379061092BA128091B912C81715
:1002800014F4C093B9128091B912082E000C990B86
:1002900004962C2F0C2E000C330B8217930724F49A
:1002A0008CEF8C0F8093B9123090B912D0E054E6E5
:1002B000452E512C612C712C6DE9C62E6BEAD62E81
:1002C0007EEDA72E7FE7B72EE5EF8E2EEFE79E2E71
:1002D000311017C080914002882349F081E0C1119C
:1002E00080E024E040EF55E26D2F0E94EE558091B2
:1002F0009D06882309F4A7C1C111A5C10E946B4CBA
:100300009EC181E038122EC080914002882379F08E
:1003100088E896E00E9495559C0181E0C13009F083
:1003200080E000E049EE55E26D2F0E94A4E080914C
:100330009D06882309F487C1C13009F084C1C093A8
:100340009B061092970610929806109299061092AA
:100350009A0623EB3BE644E051E068E876E082EE63
:1003600095E231C092E0391231C080914002882379
:1003700079F08CE896E00E9495559C0181E0C230AE
:1003800009F080E000E04EED55E26D2F0E94A4E000
:1003900080919D06882309F456C1C23009F053C1EB
:1003A00081E080939B061092970610929806109217
:1003B000990610929A0626EB3BE647E850E06CE877
:1003C00076E08AED95E20E94F3D739C1A3E03A12B4
:1003D00031C080914002882379F08AE896E00E943B
:1003E00095559C0181E0C33009F080E000E040EDCC
:1003F00055E26D2F0E94A4E080919D06882309F4A8
:1004000022C1C33009F01FC181E080939B06109286
:100410009706109298061092990610929A062FEF5E
:1004200030E040E050E06AE876E086EC95E20E9439
:100430004EE005C1B4E03B1229C080914002882300
:1004400099F080912D0C811103C025EB35E202C09B
:1004500029EB35E281E0C43009F080E001E04DEBAA
:1004600055E26D2F0E94A4E080919D06882309F437
:10047000EAC0C43009F0E7C090912D0C81E08927D3
:1004800080932D0C83E080934002D9C025E0321286
:100490003AC080914002882311F181E08F9384E07B
:1004A0008F931F921F928CE392E09F938F93A7EA02
:1004B000B5E2BF93AF93AEEAB5E2BF93AF93DF93DC
:1004C00081E0C53009F080E08F930E9414E18DB780
:1004D0009EB70C960FB6F8949EBF0FBE8DBF80914D
:1004E0009D06882309F4AFC0C53009F0ACC0E12CEB
:1004F000F12C02E813E420E030E0A9016CE372E0A3
:1005000080EA95E23CC096E039123CC080914002FE
:10051000882311F181E08F9384E08F931F921F92C3
:1005200088E392E09F938F93A2E9B5E2BF93AF93E4
:10053000A9E9B5E2BF93AF93DF9381E0C63009F03C
:1005400080E08F930E9414E18DB79EB70C960FB692
:10055000F8949EBF0FBE8DBF80919D06882309F43D
:1005600072C0C63009F06FC0E12CF12C02E813E430
:1005700020E030E0A90168E372E08BE895E20E9498
:10058000D8DF5DC097E039125EC0809140028823B9
:1005900079F084E392E00E94AB549C0181E0C73083
:1005A00009F080E000E043E855E26D2F0E94A4E0EE
:1005B00080919D06882309F446C0C73009F043C0E6
:1005C0000E94444C83E080934002ABE7B5E2B093D5
:1005D0008506A093840684E392E09093830680933B
:1005E000820610927E0610927F061092800610926C
:1005F000810640927A0650927B0660927C06709249
:100600007D0620E030E048EC52E4609134027091C5
:10061000350280913602909137020E94A4E60E9432
:10062000ABEB609376067093770680937806909391
:100630007906A4EABDEAB0930E02A0930D02809160
:10064000BA1281110DC12CEA35EC47E25EE36091EC
:1006500030027091310280913202909133020E94F7
:100660003EEB6093400C7093410C8093420C90934E
:10067000430C2CEA35EC47E25EE360912C0270916A
:100680002D0280912E0290912F020E94A4E6609389
:100690003C0C70933D0C80933E0C90933F0CB8E063
:1006A0003B1231C080914002882379F088E292E0C9
:1006B0000E9498529C0181E0C83009F080E000E07F
:1006C00045E755E26D2F0E94A4E080919D068823A6
:1006D00009F4BEC0C83009F0BBC0E12C18E1F12E0E
:1006E0000CE116E420E030E040E85FE368E272E00D
:1006F0008FE695E20E9459DF86EA9BEA90930E020C
:1007000080930D02A1C029E0321233C080914002D3
:10071000882379F080E49CE00E9498529C0181E05B
:10072000C93009F080E000E049E655E26D2F0E94F3
:10073000A4E080919D06882309F48AC0C93009F09D
:1007400087C0E12C18E1F12E0CE116E42AE037ED28
:1007500043E25CE360E47CE083E695E20E9459DFDB
:10076000D0920E02C0920D02909287068092860669
:100770006BC08AE0381233C080914002882379F040
:100780008CE39CE00E9498529C0181E0CA3009F001
:1007900080E000E04DE555E26D2F0E94A4E08091DD
:1007A0009D06882309F454C0CA3009F051C0E12CD9
:1007B00018E1F12E0CE116E420E030E040E85FE3C0
:1007C0006CE37CE087E595E20E9459DFD0920E024F
:1007D000C0920D02B0928706A092860635C09BE0BB
:1007E000391217C080914002882351F081E0CB304C
:1007F00009F080E023E046E455E26D2F0E94EE55BB
:1008000080919D06882321F1CB3011F582EC9CEB81
:1008100019C0ACE03A121CC080914002882351F00C
:1008200081E0CC3009F080E023E045E355E26D2F14
:100830000E94EE5580919D06882351F0CC3041F402
:100840008FEB9CEB0E9482598091BA12811108C0F3
:10085000DF5F3394D53009F03BCD8DE08093440CBD
:10086000DF91CF911F910F91FF90EF90DF90CF908C
:10087000BF90AF909F908F907F906F905F904F90C0
:100880003F9008958F929F92AF92BF92CF92DF9246
:10089000FF920F931F93CF93DF9300D000D0CDB77B
:1008A000DEB710929B068091760690917706A09114
:1008B0007806B091790681309048A105B10540F0E5
:1008C00010927606109277061092780610927906AA
:1008D0001091760680913B0C1816DCF4282F082E18
:1008E000000C330B21503109412F012E000C550B08
:1008F0004217530774F01FEF180F812F90E0A0E00C
:10090000B0E08093760690937706A0937806B09334
:1009100079061092BA128091B912181714F4109334
:10092000B9128091B912082E000C990B0496212F50
:10093000012E000C330B8217930724F48CEF810FE8
:100940008093B912F090B91200E083E9A82E82E0FA
:10095000B82E94E6C92ED12C2AEB822E22E0922EBC
:10096000F11017C080914002882349F081E01111F5
:1009700080E024E040E355E2602F0E94EE55809134
:100980009D06882309F48AC0111188C00E946B4C0F
:1009900081C081E0F81219C080914002882351F093
:1009A00081E0113009F080E023E044E255E2602F5D
:1009B0000E94EE5580919D06882309F46FC0113086
:1009C00009F06CC082EF90E81BC022E0F2121BC05D
:1009D00080914002882351F081E0123009F080E0DC
:1009E00023E04DE155E2602F0E94EE5580919D0677
:1009F000882309F453C0123009F050C088E797EB00
:100A00000E94825947C083E0F81217C080914002CB
:100A1000882351F081E0133009F080E023E044E1C5
:100A200055E2602F0E94EE5580919D068823B1F11A
:100A30001330A1F584EA90EBE3CF24E0F2122EC04C
:100A400080914002882351F081E0143009F080E069
:100A500020E243E055E2602F0E94EE5580919D0612
:100A60008823E1F01430D1F40E9482B2BE82AD82BC
:100A7000DA82C982BE016B5F7F4FCE0101963DD6FF
:100A80009C828B82DA82C982BE016D5F7F4FCE016C
:100A9000019633D68091BA12811107C00F5FF3948B
:100AA000053009F05DCF00933B0C26960FB6F89405
:100AB000DEBF0FBECDBFDF91CF911F910F91FF9091
:100AC000DF90CF90BF90AF909F908F9008956EEF82
:100AD00076E680E090E00C94B86B69EF76E681E012
:100AE00090E00C94B86B64EF76E682E090E00C94B2
:100AF000B86B6AE875E683E090E00C94B86BAF924F
:100B0000BF92CF92DF92EF92FF920F931F93CF93FA
:100B1000DF9310929B064091760650917706609184
:100B2000780670917906413050486105710540F0B2
:100B30001092760610927706109278061092790637
:100B4000C09176069091450C1916DCF4292F092ED8
:100B5000000C330B215031094C2F0C2E000C550B7F
:100B60004217530774F0CFEFC90F4C2F50E060E0ED
:100B700070E0409376065093770660937806709302
:100B800079061092BA129091B912C91714F4C09351
:100B9000B9122091B912022E000C330B2C5F3F4F7B
:100BA0004C2F0C2E000C550B2417350724F49CEF0A
:100BB0009C0F9093B9121091B912D0E0282F30E019
:100BC000220F331FC901825D934F6C01C9018E5CF6
:100BD000934F5C01C9018A5C934F7C01111117C0CE
:100BE00080914002882349F081E0C11180E024E037
:100BF00042E256E26D2F0E94EE5580919D068823B9
:100C000009F472C0C11170C00E946B4C69C01130F0
:100C100011F580914002882371F0C7010E9495551B
:100C20009C0181E0C13009F080E000E048E156E23B
:100C30006D2F0E94A4E080919D06882309F454C082
:100C4000C13009F051C02FEF30E040E050E0B70173
:100C50008EE096E243C0123001F580914002882375
:100C600071F0C5010E9495559C0181E0C23009F0E8
:100C700080E000E047E056E26D2F0E94A4E0809102
:100C80009D06882389F1C23079F524E031E045E002
:100C900050E0B50180E096E221C0133029F5809143
:100CA0004002882371F0C6010E9495559C0181E0A5
:100CB000C33009F080E000E04CEF55E26D2F0E9458
:100CC000A4E080919D06882379F0C33069F427E879
:100CD00030E045E050E0B60188EF95E20E944EE03A
:100CE0008091BA12811108C0DF5F1F5FD53009F013
:100CF00075CF84E08093450CDF91CF911F910F91C8
:100D0000FF90EF90DF90CF90BF90AF900895EF925B
:100D1000FF920F931F93CF93DF93CDB7DEB76F97FB
:100D20000FB6F894DEBF0FBECDBF7B0109E710E11F
:100D30002BE730E1F8013183208322E030E030936B
:100D4000B3122093B2129093B5128093B41240E084
:100D500050E0BA018FE790E10E94CE78F8018081DF
:100D600091812BE1FC013496DE01159601900D92E4
:100D70002A95E1F7FC01828193819C838B838EE22B
:100D800093E09A838983A701BE016F5F7F4F8FEE47
:100D900093E00E9420A9CE0101960E9423B46F9691
:100DA0000FB6F894DEBF0FBECDBFDF91CF911F917C
:100DB0000F91FF90EF90089510922D108091FB11EC
:100DC000882319F088EF91E100C80895E0919B0F06
:100DD000F0919C0F0190F081E02D682F8BE99FE04E
:100DE0001994CF93DF938091D80F811107C081E0D0
:100DF0008093D80F8FE99FE00E9472B5C091A10F38
:100E0000D091A20FE091D00FF091D10F82E019950F
:100E1000E091D00FF091D10F81E0199520E030E002
:100E200044E1BE018FE99FE00E94F0B422ED3FE073
:100E300047E1BE018FE99FE00E94F0B4E091D00F3E
:100E4000F091D10F80E0DF91CF9119946F927F9252
:100E50008F929F92BF92CF92DF92EF92FF920F9369
:100E60001F93CF93DF93CDB7DEB7AD970FB6F8944E
:100E7000DEBF0FBECDBF20912E10222309F4D2C1B8
:100E8000B62E7C018091FB11882309F49AC044237B
:100E900009F4A0C180911312882311F1E7E7F7E26A
:100EA00084918F010F5F1F4F882319F0A9D7F80194
:100EB000F7CFE4E3F7E284918F010F5F1F4F8823A0
:100EC00019F09ED7F801F7CF61E070E080E090E084
:100ED0000E946D8F8AE094D78BE297E20E94559230
:100EE0008FE280931812D12C21E009E112E19FE1F9
:100EF000C92E8091D011D816B8F4CD9CC001112410
:100F0000B80182569F4E2DA70E94B17EC8012DA523
:100F10008C010196F8013081332321F02D3811F036
:100F20002F5FF6CFD394E5CF27FD08C0B80188EF37
:100F300091E10E94B17EEEE7FCE203C0F80110826D
:100F4000FACF84918F010F5F1F4F882319F058D774
:100F5000F801F7CFB70182E197E20E9484766091B1
:100F60001312FDE86F9FB0011124685E7D4E87E08B
:100F700097E20E9484764091A9125091AA12609142
:100F8000AB127091AC1281E097E20E94BE648AE0DD
:100F900037D78091131294E0899FF0011124EC5E01
:100FA000FD4E4091A9125091AA126091AB1270911E
:100FB000AC1240835183628373838F5F80931312DB
:100FC0000CC01092131282E0D82E06C1B70184EF34
:100FD00096E20E9484768AE013D7EEDECE01019677
:100FE0006C010E9413B48AE590E190937A1080938B
:100FF0007910F70180818F3209F05CC087010F5FA3
:101000001F4F09F45DC06FE270E0C8010E949BEDC4
:101010003C01009709F455C00817190708F051C0A2
:101020004C01801A910AA401B801CE0180960E9459
:10103000C4EDE0E2F0E0EC0FFD1FE80DF91D1082B9
:10104000CE0180964C018C01F80181918F0188239B
:1010500011F0D6D6F9CF8AE0D3D66091791070918D
:101060007A106115710511F06C5F7F4F21E0AE01C0
:10107000405E5F4FCE0105960E94ED7E811114C047
:10108000E0EEF6E284918F010F5F1F4F882319F085
:10109000B7D6F801F7CFF40181914F01882311F001
:1010A000AFD6F9CF8EE282C0D0927A10C09279107A
:1010B0008301A5CF8BE790E190937A10809379100C
:1010C00087019091791080917A10692F782FBB2039
:1010D00009F457C06115710511F06C5F7F4F21E075
:1010E000A80188EF91E10E94ED7E882309F445C0B4
:1010F0008091091290910A12A0910B12B0910C12DA
:101100008093A5129093A612A093A712B093A81251
:10111000B80182ED96E20E9484764091A51250912A
:10112000A6126091A7127091A8128AEC96E20E9412
:10113000BE648AE065D61092A9121092AA1210928B
:10114000AB121092AC12EBEBF6E284917F019FEFB1
:10115000E91AF90A882319F053D6F701F6CFB80136
:1011600080E090E0D4DD80913D10882319F08DE37C
:1011700090E101C0C80160E027C0B80187EA96E2AB
:1011800010C06115710511F06C5F7F4F26E5A80155
:1011900088EF91E10E94ED7E81110AC0B80183E9D8
:1011A00096E20E9484768EE22BD68AE029D60EC083
:1011B00081E080932B10B70181E896E20E9484764B
:1011C0008AE01ED660E0C8010E949D56C6010E94BA
:1011D00023B428C0DD24D394EEE7FCE284918F0190
:1011E0000F5F1F4F882319F00BD6F801F7CFECEFF4
:1011F000F6E284918F010F5F1F4F882319F000D60C
:10120000F801F7CFE1E0DE1619F00FEF13E002C0AE
:1012100005E014E0F80181918F01882309F4D6CE0E
:10122000EFD5F8CFAD960FB6F894DEBF0FBECDBFA9
:10123000DF91CF911F910F91FF90EF90DF90CF90B2
:10124000BF909F908F907F906F900895CF92DF9284
:10125000EF92FF920F931F93CF93DF93CDB7DEB73B
:10126000EDB6FEB6DC010D900020E9F79D01281BCC
:10127000390B2C5F3F4F4DB75EB7421B530B0FB678
:10128000F8945EBF0FBE4DBF0DB71EB70F5F1F4F67
:101290009F938F938AE796E29F938F931F930F9369
:1012A0000E94D8E5680154E0C50ED11C0F900F9044
:1012B0000F900F900F900F90F6018081882349F0D6
:1012C000082E000C990B0E945FEDF60181936F01CF
:1012D000F3CF60E0C8010E942071882319F0C80193
:1012E0000E94269286E796E29093520C8093510CCE
:1012F0000E943C710FB6F894FEBE0FBEEDBEDF91AA
:10130000CF911F910F91FF90EF90DF90CF900895B4
:10131000AF92BF92CF92DF92EF92FF920F931F9303
:10132000CF93DF93CDB7DEB7AA970FB6F894DEBFA1
:101330000FBECDBF809159108F93809158108F931D
:101340008DE696E29F938F937E0181E2E80EF11C79
:10135000FF92EF920E94D8E50F900F900F900F90A0
:101360000F900F9010E0F70101900020E9F73197FE
:10137000EE19FF091E1784F46701C10ED11C17FD79
:10138000DA94F6018081082E000C990B0E945FED23
:10139000F60180831F5FE7CF40E050E0BA018EE5A1
:1013A00090E10E94CE7800E0CE0101966C01809120
:1013B0006110823028F4011114C08FEF9FEF16C026
:1013C0008091661090916710A0916810B09169109B
:1013D0008F719927AA27BB27892B8A2B8B2B59F72B
:1013E0001AC08091581090915910019690935910FD
:1013F00080935810AA960FB6F894DEBF0FBECDBFEB
:10140000DF91CF911F910F91FF90EF90DF90CF90E0
:10141000BF90AF90089540E050E0B6018EE590E1B6
:101420000E94167C18163CF6F60101900020E9F7A0
:1014300031971E2F1C19115068F05601A10EB11CD6
:1014400017FDBA94F501808190E00E945FEDF501EF
:101450008083F1CF8A858E3709F4A9CF45E050E02B
:10146000B701C6010E94B6ED892B09F0A0CFC701D4
:10147000EDDE01E09CCFCF92DF92EF92FF921F93BF
:10148000CF93DF9310922E1080916110882321F06A
:101490008EE590E10E94E57E1092D5111092D21156
:1014A00085E38093D1110E94E750EB01A89561E09C
:1014B0008091D1110E94AC4F81ED91E10E94D6D272
:1014C0002398229A219A209A289A85E08093D31112
:1014D00082E58CBD1DBC1AE08FEF0E94DBD211505B
:1014E000D9F720E030E0A90160E081ED91E10E94B0
:1014F00001D3182F8093D411813049F00E94E75016
:101500006C1B7D0B613D774060F381E054C02AEA9B
:1015100031E040E050E068E081ED91E10E9401D3CC
:1015200082FF03C01093D5110EC014E00E94E0D2D8
:101530008093D4111150D1F78A3A11F082E03BC068
:1015400082E08093D5118091D511823021F0C12C99
:10155000D12C760105C0C12CD12CE12C80E4F82ED1
:1015600020E030E0A90167E381ED91E10E9401D321
:10157000A701960169E281ED91E10E9401D3809378
:10158000D411882349F00E94E7506C1B7D0B613D0C
:10159000774030F38AE00FC08091D511823011F589
:1015A00020E030E0A9016AE381ED91E10E9401D3DE
:1015B000882351F088E08093D21181ED91E10E945F
:1015C000D6D2EEE7FCE21AC00E94E0D2807C803CDA
:1015D00019F483E08093D5110E94E0D20E94E0D2FA
:1015E0000E94E0D281ED91E10E94D6D21092D311F7
:1015F00081E00E94C0A681112EC013C08491EF012A
:101600002196882319F0FCD3FE01F8CFEFE5F6E22E
:101610008491EF012196882309F450C0F1D3FE0193
:10162000F7CF80E00E94C0A6811115C0E7E7F7E27E
:101630008491EF012196882319F0E2D3FE01F8CFBF
:10164000EBE4F6E28491EF012196882309F436C099
:10165000D7D3FE01F7CF66ED71E18EE590E10E94F0
:101660005F7E811114C0E7E7F7E28491EF012196D4
:10167000882319F0C5D3FE01F8CFEAE3F6E284919E
:10168000EF0121968823D1F0BBD3FE01F8CF81E092
:1016900080932E10EEE7FCE28491EF0121968823DF
:1016A00019F0AED3FE01F8CFEEE2F6E28491EF013D
:1016B0002196882319F0A4D3FE01F8CF8BE1EEE543
:1016C000F0E1AFE7B0E101900D928A95E1F78091EA
:1016D0005C1090915D1090937E1080937D108AE550
:1016E00090E190937A1080937910DF91CF911F91C0
:1016F000FF90EF90DF90CF9008950F931F93CF93BB
:10170000DF938C01EB0190910B1020910C10921340
:1017100007C08FEF9FE00E94296D0E94065CF3CF07
:10172000F801A081B1814881598180910A1034E08B
:10173000839FF0011124ED5FFF4EB387A287558789
:1017400044879F5F90930B108F5F821719F08093EF
:101750000A1002C010920A10DF91CF911F910F91D1
:101760000895CF93DF93CDB7DEB78091500C8111F0
:1017700010C09E01275F3F4F4F81588562E470E0A3
:1017800086E492E00E9407E60E946FA883E08093BF
:101790004002DF91CF91089580911D1090911E100D
:1017A00081309105B9F1029759F40E9439A86093EC
:1017B0001F1070932010809321109093221018C056
:1017C00010922310109224101092251010922610BF
:1017D00010922710109228101092291010922A109F
:1017E00010921F10109220101092211010922210AF
:1017F00081E090E090931E1080931D100E94E750AE
:1018000060932310709324108093251090932610DA
:1018100081E0089580E0089580911D1090911E1040
:10182000019791F482E090E090931E1080931D1038
:101830000E94E7506093271070932810809329101E
:1018400090932A1081E0089580E00895BC0180E023
:1018500090E04AE0DCD28DE0D3D28AE0D1C28F9210
:101860009F92AF92BF92CF92DF92EF92FF92CF936F
:1018700020E030E04AE754E4FC016081718182811C
:1018800093810E94A4E60E94A6EB6B017C01611586
:1018900071058105910561F097FF0AC0F094E0940D
:1018A000D094C094C11CD11CE11CF11C8DE201C07C
:1018B00080E28093490CC701B60128EE33E040E096
:1018C00050E00E9426EA8AE0882E912CA12CB12CAF
:1018D000CA01B901A50194010E9426EA605D6093E6
:1018E0004A0C8EE280934B0CC701B60124E630E02F
:1018F00040E050E00E9426EACA01B901A501940126
:101900000E9426EA605D60934C0CC701B601A501F8
:1019100094010E9426EAC62FCA01B901A5019401CB
:101920000E9426EA605D60934D0CC05DC0934E0C32
:1019300089E49CE0CF91FF90EF90DF90CF90BF9033
:10194000AF909F908F900895FF920F931F93CF9326
:10195000DF931F92CDB7DEB7982F862F692F49836B
:101960000E94EDCF9091D30F8091470C4981891748
:1019700038F19091D50F8091460C981708F180911D
:101980003D108823D1F0109252100DE310E1442352
:1019900019F082E00E94E6D085E1F82EF8018191ED
:1019A0008F01882321F00E94CFD0F81AF7CFFF20B3
:1019B00039F080E20BDAFA94FACF00E310E1E7CFD6
:1019C0000F90DF91CF911F910F91FF900895CF92CB
:1019D000DF92EF92FF92C0908902D0908A02E0904D
:1019E0008B02F0908C028091B812882321F120E0C4
:1019F00030E0A901C701B6010E943FE68823D9F073
:101A000020E030E040E05FE3C701B6010E94A4E6B9
:101A10009B01AC010E94A4E62BED3FE049E450E4B9
:101A20000E94A4E69B01AC0160E070E080E89FE3C7
:101A30000E943EEB04C060E070E080E89FE36093AA
:101A40009502709396028093970290939802FF906C
:101A5000EF90DF90CF9008952F923F924F925F9238
:101A60006F927F928F929F92AF92BF92CF92DF92AE
:101A7000EF92FF920F931F93CF93DF93CDB7DEB713
:101A800068970FB6F894DEBF0FBECDBF1C015B0197
:101A90008A01DC01D7966D917D918D919C91DA97A9
:101AA0000E9443E66B017C01F50120813181428176
:101AB00053810E94A4E60E9428EB0E94ABEB698749
:101AC0007A878B879C87D8012D913D914D915C91B0
:101AD000C701B6010E94A4E60E9428EB0E94ABEB6E
:101AE0006D877E878F87988B29853A854B855C85A6
:101AF000283731054105510540F488E790E0A0E022
:101B0000B0E089879A87AB87BC872D853E854F8556
:101B10005889283731054105510540F488E790E0A0
:101B2000A0E0B0E08D879E87AF87B88B91012D5BD9
:101B30003F4FD9018D919D910D90BC91A02D8D832A
:101B40009E83AF83B887BC01CD010E9445E66983BF
:101B50007A838B839C8369857A858B859C850E949B
:101B600043E6698B7A8B8B8B9C8B20E030E0A9015C
:101B700069817A818B819C810E943FE6882339F1BB
:101B8000A7019601C701B6010E94A4E64B015C01C2
:101B900029893A894B895C89CA01B9010E94A4E666
:101BA0009B01AC01C501B4010E9461EA4B015C01DB
:101BB00029813A814B815C81CA01B9010E9462EAA4
:101BC0009B01AC01C501B4010E943EEB03C060E083
:101BD00070E0CB010E9428EB0E94A6EB2B013C0198
:101BE0006D817E818F8198859095809570956195A6
:101BF0007F4F8F4F9F4F0E9445E64B015C016D85E3
:101C00007E858F8598890E9443E66D837E838F83CE
:101C1000988720E030E0A901C501B4010E943FE6A9
:101C2000882349F12D813E814F815885CA01B90130
:101C30000E94A4E66D8B7E8B8F8B988FA7019601F7
:101C4000C701B6010E94A4E69B01AC016D897E89A3
:101C50008F89988D0E9461EA6B017C01A501940136
:101C6000C501B4010E9462EA9B01AC01C701B60143
:101C70000E943EEB03C060E070E0CB010E94D7EB16
:101C8000F10182889388A488B58875016401C4181D
:101C9000D508E608F7080E94A6EBC61AD70AE80A94
:101CA000F90AF7FE6BC020E030E0A90169817A8172
:101CB0008B819C810E943FE6882309F447C02981DB
:101CC0003A814B815C81CA01B9010E9462EA6B01D1
:101CD0007C01C501B4010E9443E69B01AC01C70130
:101CE000B6010E94A4E66B017C0129893A894B89DF
:101CF0005C89CA01B9010E94A4E69B01AC01C7013D
:101D0000B6010E9461EA6B017C012D813E814F8109
:101D10005885CA01B9010E94A4E69B01AC01C70124
:101D2000B6010E9462EA6B017C0120E030E040E8ED
:101D300050E469817A818B819C810E94A4E69B0199
:101D4000AC01C701B6010E943EEB03C060E070E049
:101D5000CB010E9428EB0E94A6EB2B013C0197FFD0
:101D600003C0412C512C3201481459046A047B04ED
:101D700010F024013501C12CD12C76018FB7F894D5
:101D8000D1019C9193FD22C0F101468A578A608E51
:101D9000718EC40CD51CE61CF71C5A96CD92DD92B0
:101DA000ED92FC925D9729853A854B855C85DB96A3
:101DB0002D933D934D935C93DE97FF962D853E8545
:101DC0004F85588920833183428353838FBF689620
:101DD0000FB6F894DEBF0FBECDBFDF91CF911F913C
:101DE0000F91FF90EF90DF90CF90BF90AF909F90BA
:101DF0008F907F906F905F904F903F902F900895BD
:101E00009091C00095FFFCCF8093C60008958F92FB
:101E10009F92AF92BF92EF92FF921F93CF93DF9367
:101E2000CDB7DEB7A0970FB6F894DEBF0FBECDBF1B
:101E3000611571058105910579F110E0842E912CD1
:101E4000A12CB12CEE24E394F12CEC0EFD1EE10E3E
:101E5000F11C17FDFA94A50194010E9404EAF70110
:101E60006083B901CA011F5F611571058105910584
:101E700049F7115010F1E1E0F0E0EC0FFD1FE10F28
:101E8000F11D17FDFA9580818A3010F097E301C0AB
:101E900090E3890FB5DFEDCF80E3A0960FB6F894FD
:101EA000DEBF0FBECDBFDF91CF911F91FF90EF90AE
:101EB000BF90AF909F908F90A3CFA0960FB6F8944D
:101EC000DEBF0FBECDBFDF91CF911F91FF90EF908E
:101ED000BF90AF909F908F900895CF92DF92EF9236
:101EE000FF926B017C0197FF0AC08DE289DFF094BD
:101EF000E094D094C094C11CD11CE11CF11C4AE0B8
:101F0000C701B601FF90EF90DF90CF9080CF8F9206
:101F10009F92AF92BF92CF92DF92EF92FF92CF93B8
:101F20006B017C01B42E20E030E0A9010E943FE665
:101F300087FF06C08DE264DFF7FAF094F7F8F094BB
:101F4000C0E060E070E080E09FE3CB1541F02DEC55
:101F50003CEC4CEC5DE30E94A4E6CF5FF6CF9B0126
:101F6000AC01C701B6010E9462EA6B017C010E94CC
:101F7000ABEB4B015C014AE04ADFCC2379F1C501B0
:101F8000B4010E9443E69B01AC01C701B6010E9467
:101F900061EA6B017C018EE233DF20E030E040E259
:101FA00051E4C701B6010E94A4E64B015C010E9406
:101FB000A6EB6B01770FEE08FF08C701B6018DDFB6
:101FC000C701B6010E9445E69B01AC01C501B40101
:101FD0000E9461EA6B017C01C150F9F6CF91FF903C
:101FE000EF90DF90CF90BF90AF909F908F9008952B
:101FF0008FB7F8949091140D2091130D291759F073
:10200000E92FF0E0ED56F34F208130E09F5F9F779E
:102010009093140D02C02FEF3FEF8FBFC9010895B9
:102020001F920F920FB60F9211240BB60F922F939F
:102030003F938F939F93EF93FF932091C6009FB799
:10204000F894E091130D81E08E0F8F773091140D8D
:10205000831731F0F0E0ED56F34F20838093130D9A
:102060009FBFFF91EF919F918F913F912F910F9083
:102070000BBE0F900FBE0F901F901895CF92DF925E
:10208000EF92FF92CF93DF93EC01C090F10BD090D1
:10209000F20BE090F30BF090F40BA701960168812E
:1020A00079818A819B810E943FE687FF04C0C882B4
:1020B000D982EA82FB82C090F50BD090F60BE090BB
:1020C000F70BF090F80BA70196016C817D818E8152
:1020D0009F810E943FE687FF04C0CC82DD82EE82B2
:1020E000FF82C090F90BD090FA0BE090FB0BF090C0
:1020F000FC0BA7019601688579858A859B850E94DE
:102100003FE687FF04C0C886D986EA86FB86C09072
:102110001B02D0901C02E0901D02F0901E02A7014D
:102120009601688179818A819B810E9488EC1816CA
:1021300024F4C882D982EA82FB82C0901F02D09028
:102140002002E0902102F0902202A70196016C810A
:102150007D818E819F810E9488EC181624F4CC82A8
:10216000DD82EE82FF82C0902302D0902402E090B4
:102170002502F0902602A7019601688579858A8557
:102180009B850E9488EC181624F4C886D986EA86B6
:10219000FB86DF91CF91FF90EF90DF90CF90089575
:1021A0004F925F926F927F928F929F92AF92BF9267
:1021B000CF92DF92EF92FF920F931F93CF93DF9313
:1021C00000D000D0CDB7DEB77C01FC01E354F74D61
:1021D000149182E0E816F10421F481E07CD68111AB
:1021E0001EC16701CC0CDD1CCC0CDD1CC6018F545C
:1021F000974D0E94A5714B015C01612F110F770B68
:10220000880B990B0E9445E62B013C0120E030E051
:1022100040EC5FE3C501B4010E94A4E6A301920172
:102220000E94A4E6AB01BC0100E010E09801C701E8
:1022300064D492E0E916F10479F48DEA98E20E9400
:10224000A57120E030E040EA50E40E943FE687FDBF
:1022500009C08DEA98E203C0C6018B55974D0E94D4
:10226000A57104C060E070E080EA90E49B01AC01DD
:10227000C301B2010E94A4E64B015C0120E030E002
:10228000A9010E943FE6882309F456C000E010E04F
:102290009801B501A4017058C7012FD486E0E4E18C
:1022A000F3E0DE01119601900D928A95E1F7F701B6
:1022B000EE0FFF1F81E090E08C0F9D1FE80FF91FCC
:1022C0008081918118161906C4F0EEE7FCE2849132
:1022D0008F010F5F1F4F882319F092DDF801F7CFB0
:1022E000E3E8F8E284918F010F5F1F4F882319F014
:1022F00087DDF801F7CF8AE090E0BC01990F880BE9
:10230000990B0E9445E69B01AC01F601E65EFC4F8D
:1023100060817181828193810E943EEB2B013C019F
:10232000A5019401C501B4010E9462EAAB01BC01A0
:1023300093018201C701E1D381E0F701E959FB4F25
:102340008083F701E455FB4F8083F601E958F34F92
:102350001082118212821382C701A4D7C601895844
:10236000974D0E94A571860104541B4FF601E55953
:10237000F34F20813181428153810E9462EAF8014A
:102380006083718382839383F2E0EF16F104D1F4CA
:102390002091111330911213409113135091141383
:1023A0006091C4047091C5048091C6049091C704E3
:1023B0000E9461EA6093C4047093C5048093C604CC
:1023C0009093C7040E949B71F601ED57F34FD6011D
:1023D000A454BB4F8D919D910D90BC91A02D8083F5
:1023E0009183A283B38382E0E816F104C1F480E014
:1023F00026960FB6F894DEBF0FBECDBFDF91CF910A
:102400001F910F91FF90EF90DF90CF90BF90AF9012
:102410009F908F907F906F905F904F905CC52696B5
:102420000FB6F894DEBF0FBECDBFDF91CF911F91E5
:102430000F91FF90EF90DF90CF90BF90AF909F9063
:102440008F907F906F905F904F9008950F931F93A0
:10245000CF93DF938C01EEE7FCE28491EF012196AC
:10246000882319F0CDDCFE01F8CFB8018AE698E2A6
:102470000E94847682E2C4DC8AE0C2DC81E0DF91E3
:10248000CF911F910F9108955F9AECEAF4E01082CA
:102490008A9A11829FB7F894A8E0B1E08C9181608C
:1024A0008C939FBF1282129A08958C01E7E7F7E29E
:1024B0008491EF012196882319F0A2DCFE01F8CF68
:1024C000EAE4F8E28491EF012196882319F098DC80
:1024D000FE01F8CF0E9486CED7DF0E94665961E0E8
:1024E000C8010E9488560E94644C0E94F18684E0D4
:1024F0000E941CD08091A00F869586951092D60FD1
:102500008093D70F86E492E00E9407D18091A00FBC
:1025100086958695880F1092D60F8093D70F8BE300
:1025200098E20E94FAD08091A00F86958695982F08
:10253000990F890F1092D60F8093D70F8EE298E2F1
:102540000E94FAD00E9435A68111D1CF2FEF8BE4E3
:102550009DE1215080409040E1F700C00000F894D8
:102560002FEF84E39CE0215080409040E1F700C0D1
:1025700000000E9486CEA895FECF4F925F926F9288
:102580007F928F929F92AF92BF92CF92DF92EF9203
:10259000FF920F931F93CF93DF930E94AE560E943A
:1025A000E7506B017C0110914102112309F45FC0D7
:1025B00080915F0C9091600C009709F458C0409195
:1025C000150D5091160D6091170D7091180D460163
:1025D0005701841A950AA60AB70AB7FC5AC0833075
:1025E0009105F9F034F401970CF441C0EEE7FCE2F8
:1025F00006C0049709F03BC0EEE7FCE226C08491D8
:10260000EF012196882319F0FBDBFE01F8CFE0EB08
:10261000F7E28491EF012196882349F1F1DBFE0175
:10262000F8CFEEE7FCE28491EF012196882319F0C0
:10263000E7DBFE01F8CFE9E9F7E28491EF012196AB
:102640008823A9F0DDDBFE01F8CF8491EF0121960C
:10265000882319F0D5DBFE01F8CFE1E8F7E2849199
:10266000EF012196882319F0CBDBFE01F8CF212F53
:1026700030E0A8EEB3E00E9452EAC60ED71EE81E74
:10268000F91EC092150DD092160DE092170DF09222
:10269000180D80916E06843008F4BBD70E94E75075
:1026A000C090670CD090680CE090690CF0906A0CB8
:1026B000C114D104E104F10459F10091630C1091AB
:1026C000640C2091650C3091660C0C0D1D1D2E1DA7
:1026D0003F1D5B016C01A01AB10AC20AD30AD7FCE4
:1026E00017C0E7E7F7E28491EF012196882319F0FC
:1026F00087DBFE01F8CF6091610C7091620C84EF72
:1027000097E20E9484768AE07BDB8BEE97E255C0ED
:10271000C0904202D0904302E0904402F090450203
:10272000C114D104E104F104D9F00091630C1091BB
:10273000640C2091650C3091660C0C0D1D1D2E1D36
:102740003F1DDC01CB01801B910BA20BB30BB7FD2E
:1027500007C09091FD0F8091FE0F981709F460C19A
:1027600080911D0D90911E0D909902C0019604C09C
:10277000181619062CF4019790931E0D80931D0DC9
:1027800080911D0D90911E0D8E3E9240BCF0E7E7AA
:10279000F7E28491EF012196882319F031DBFE01E5
:1027A000F8CFEBECF7E28491EF012196882319F042
:1027B00027DBFE01F8CF82EC97E277DE60918A0694
:1027C0009091FD0F8091FE0F981791F0E091FE0F10
:1027D0008DE4E89FF0011124ED5FF84F6081809156
:1027E000FE0F9091FD0F891719F08F5F8F70F9CF51
:1027F00070E089E00E94E84F80912D0C882309F455
:10280000F9C000913C0210913D02D0913E02C0916E
:102810003F0260918806709189066E5F7F4F072E98
:10282000000C880B990B0E9445E698014D2F5C2FF8
:102830000E943FE687FDDEC0F090FE0F912CA12C98
:10284000B12CE12C8DE4882E8091FD0FF81609F44F
:102850005BC08F2D90E0889EF001899EF00D1124C1
:10286000E454F94F4281538164817581452B462B95
:10287000472B81F44681578160857185452B462B16
:10288000472B41F44285538564857585452B462B3E
:10289000472BA9F1889E9001899E300D1124F901E2
:1028A000E454F94F6F0166857785808991890E948C
:1028B00045E62B013C01F60162897389848995897B
:1028C0000E9443E69B01AC01C301B2010E943EEBB2
:1028D000F60123A134A145A156A10E94A4E63B0123
:1028E0006C019B01AC01692D7A2D8B2D9E2D0E94D0
:1028F0003FE687FF04C0962CA72CBC2CED2C81E072
:102900008F0D8F70F82EA0CF2091340230913502B8
:102910004091360250913702692D7A2D8B2D9E2DD4
:102920000E94A4E69B01AC01B8018D2F9C2F0E9450
:1029300062EA6B017C0198014D2F5C2F0E943FE6FB
:1029400087FD14C00091380210913902D0913A02EB
:10295000C0913B0298014D2F5C2FB601C7010E9428
:1029600088EC18161CF08601DE2DCF2DC090190DB5
:10297000D0901A0DE0901B0DF0901C0DA701960150
:10298000B8018D2F9C2F0E943FE687FF1CC020E0DE
:1029900037ED43EA5CE3B8018D2F9C2F0E94A4E63B
:1029A0004B015C0128E431EE4AE75FE3C701B60161
:1029B0000E94A4E69B01AC01C501B4010E9462EA39
:1029C0008B01D82FC92FC801AD2FBC2F8093190DB3
:1029D00090931A0DA0931B0DB0931C0DB8018D2F71
:1029E0009C2F0E94A6EB709389066093880680E076
:1029F0000E9453CE0E94065C8FEF9FE0DF91CF9143
:102A00001F910F91FF90EF90DF90CF90BF90AF900C
:102A10009F908F907F906F905F904F900C94296D56
:102A20005F9A1092AC048A9A1092AD049FB7F89402
:102A3000809108018160809308019FBF1092AE04CD
:102A4000129A8ECECF93DF9380E090E00E947D5D5E
:102A5000C3E5DCE0688379838A839B8381E090E02F
:102A60000E947D5D6C837D838E839F8382E090E0F6
:102A70000E947D5D688779878A879B87DF91CF91E8
:102A80000895CF93DF930E94AB71E0916D06F0E063
:102A9000E453FB4F8081882371F0EEE7F7E28491E5
:102AA000EF012196882319F0ABD9FE01F8CF8AE017
:102AB000DF91CF91A5C9DF91CF910895CF92EF9289
:102AC000FF920F931F93E0900002F090010200919B
:102AD000020210910302C090560428EC34E044EC4A
:102AE00054E060EC74E08CEB94E00E943BBD1F91DD
:102AF0000F91FF90EF90CF900895AF92BF92CF9239
:102B0000DF92EF92FF920F931F93CF93DF9300D04A
:102B10001F92CDB7DEB779015C01AA0CBB1CAA0CD1
:102B2000BB1CC50184549B4F6C01FC0110821182B7
:102B30001282138249835A836B837C830E949B7128
:102B400049815A816B817C81F60140835183628384
:102B50007383C090560420E030E0A901B801C7019A
:102B60000E943FE6811108C0F501E65EFC4F30810E
:102B700021819281838104C0302F212F9E2D8F2DA2
:102B8000E32EF22E092F182F28EC34E044EC54E009
:102B900060EC74E08CEB94E00E943BBD0E949B5D76
:102BA0001092EC040F900F900F900F90DF91CF9147
:102BB0001F910F91FF90EF90DF90CF90BF90AF905B
:102BC000089580918A0D90918B0DA0918C0DB091FC
:102BD0008D0D8093000290930102A0930202B093A6
:102BE00003028091880D9091890D90931A02809331
:102BF00019020C94AB718091000290910102A09196
:102C00000202B091030280938A0D90938B0DA093E2
:102C10008C0DB0938D0D8091190290911A029093B2
:102C2000890D8093880D84E690E090931A0280933A
:102C300019020C94AB714F925F926F927F928F92B8
:102C40009F92AF92BF92CF92DF92EF92FF920F933B
:102C50001F93CF93DF935C014B01EA018901409000
:102C600000025090010260900202709003022881DD
:102C700039814A815B816091C4047091C50480915F
:102C8000C6049091C7040E943FE687FF29C0F8015F
:102C9000C080D180E280F38020E030E0A901C7014C
:102CA000B6010E943FE6811106C0C12CD12C20E85C
:102CB000E22E20E4F22EC0920002D0920102E092B5
:102CC0000202F092030288819981AA81BB818093DC
:102CD000C4049093C504A093C604B093C704EEDE69
:102CE000F801C080D180E280F38020E030E0A901CB
:102CF000C701B6010E943FE6811107C095E5C92EC4
:102D0000DC2C95E0E92E93E4F92EC0920002D092DB
:102D10000102E0920202F0920302F50180819181AA
:102D2000A281B3818093BC049093BD04A093BE04A0
:102D3000B093BF04F40180819181A281B38180931B
:102D4000C0049093C104A093C204B093C304B6DE40
:102D5000288139814A815B816091C4047091C504E6
:102D60008091C6049091C7040E9488EC18164CF517
:102D7000F801C080D180E280F38020E030E0A9013A
:102D8000C701B6010E943FE6811106C0C12CD12CBB
:102D900080E8E82E80E4F82EC0920002D092010272
:102DA000E0920202F092030288819981AA81BB819C
:102DB0008093C4049093C504A093C604B093C70441
:102DC0007DDE0E949B5D4092000250920102609263
:102DD000020270920302DF91CF911F910F91FF9039
:102DE000EF90DF90CF90BF90AF909F908F907F90AB
:102DF0006F905F904F9008959B01AC0160EC74E080
:102E00008CEB94E018CF8F929F92AF92BF92CF92AB
:102E1000DF92EF92FF92CF93DF93CDB7DEB7289783
:102E20000FB6F894DEBF0FBECDBF2091730C30916A
:102E3000740C4091750C5091760C0E9462EA6B0103
:102E40007C0169837A838B839C838090111390909B
:102E50001213A0901313B090141320E030E0A901D6
:102E6000C501B4010E943FE687FF0AC0A501940195
:102E7000C701B6010E9461EA69837A838B839C83D0
:102E80002091C4043091C5044091C6045091C704F8
:102E900069817A818B819C810E9488EC181654F498
:102EA0001D821E821F821886BE016B5F7F4FCE017E
:102EB0000196A2DF28960FB6F894DEBF0FBECDBFF5
:102EC000DF91CF91FF90EF90DF90CF90BF90AF90C8
:102ED0009F908F9008951F93CF93DF93CDB7DEB768
:102EE0002C970FB6F894DEBF0FBECDBF9091AF0404
:102EF000981779F1182F60E070E080E291E483DFA9
:102F00008091BC049091BD04A091BE04B091BF0417
:102F100089879A87AB87BC878091C0049091C10450
:102F2000A091C204B091C3048D839E83AF83B88700
:102F300019821A821B821C829E012F5F3F4F44EC34
:102F400054E0BE016B5F7F4FCE01099674DE109393
:102F5000AF0480E02C960FB6F894DEBF0FBECDBF55
:102F6000DF91CF911F9108952F923F924F925F92E0
:102F70006F927F928F929F92AF92BF92CF92DF9289
:102F8000EF92FF920F93CF93DF93CDB7DEB76497A5
:102F90000FB6F894DEBF0FBECDBF2B013C01490137
:102FA0005A0117018091000290910102A091020242
:102FB000B0910302898B9A8BAB8BBC8B60E070E085
:102FC00080EA90E420DF85E595E5A5E0B3E4809311
:102FD000000290930102A0930202B09303021986AB
:102FE0001A861B861C8620E030E040E251E4C501D1
:102FF000B4010E9461EA6D837E838F83988720E00D
:1030000030E040E251E4C301B2010E9461EA698309
:103010007A838B839C839E01275F3F4F44EC54E06F
:10302000BE016B5F7F4FCE01019605DE81E053DF6D
:10303000882339F0C12CD12C80ECE82E8FE7F82EB4
:10304000F4C00E94AB7120E030E040EA50E46091AF
:10305000730C7091740C8091750C9091760C0E9499
:1030600062EA6B017C0169877A878B879C878091F4
:10307000111390911213A0911313B09114138D8713
:103080009E87AF87B88B20E030E0A901BC01CD015D
:103090000E943FE687FF0CC02D853E854F855889ED
:1030A000C701B6010E9461EA69877A878B879C878E
:1030B0002091C4043091C5044091C6045091C704C6
:1030C00069857A858B859C850E943FE687FF0EC0C7
:1030D00080E090E0A0E8B0E489839A83AB83BC836E
:1030E000BE016F5F7F4FCE01099686DE80E090E0E3
:1030F000A0E0B0E48D839E83AF83B88720E030E00A
:103100004BE953E46091730C7091740C8091750CD1
:103110009091760C0E9461EA69837A838B839C8309
:10312000BE016B5F7F4FCE01019666DE1092EC040C
:1031300089DC80915B0C90915C0CA0915D0CB0914E
:103140005E0C8093C4049093C504A093C604B0930E
:10315000C7040E949B71209111133091121340916A
:103160001313509114136091C4047091C50480919D
:10317000C6049091C7040E9462EA6B017C010111B0
:1031800006C060E070E080EA90E43DDE04C080E0CC
:10319000A2DE81114FCF93E0291631040CF439C01F
:1031A000EDE5FAE284911F01AFEF2A1A3A0A88236B
:1031B00021F00E94008FF101F5CF43E0C301B2017D
:1031C0000E94878FE8E5FAE284913F01BFEF6B1A16
:1031D0007B0A882321F00E94008FF301F5CF43E0A2
:1031E000C501B4010E94878FE3E5FAE284915F0193
:1031F0009FEFA91AB90A882321F00E94008FF501D8
:10320000F5CF43E0C701B6010E94878F8AE00E9494
:10321000008F89899A89AB89BC8980930002909339
:103220000102A0930202B0930302C701B6016496A3
:103230000FB6F894DEBF0FBECDBFDF91CF910F91D7
:10324000FF90EF90DF90CF90BF90AF909F908F90C6
:103250007F906F905F904F903F902F90089580E106
:10326000E3E8FCE0ACEBB4E001900D928A95E1F765
:103270000895CF92EF92FF920F931F93C090560440
:103280007B018C012FE83CE04BE85CE067E87CE0E8
:1032900083E89CE00E943BBD1F910F91FF90EF904F
:1032A000CF900895CF92DF92EF92FF920F931F93EA
:1032B000CF93DF93EC01CC0FDD1FCC0FDD1FFE01A0
:1032C000E055FB4F20E030E0A901608171818281EF
:1032D00093810E9462EAFE01E958F34F2081318117
:1032E000428153810E9462EA6B017C01FE01E55933
:1032F000F34F6083718382839383CE01895B954D05
:103300000E94A5718E010F50144FA70196010E94D3
:1033100062EAF8016083718382839383CE01855CC6
:10332000954D0E94A571C55EDD4FA70196010E94D3
:1033300062EA688379838A839B83DF91CF911F91AF
:103340000F91FF90EF90DF90CF900895682F880F36
:10335000770B80915C0490915D040E949BED9C0131
:10336000909353048093520481E0232B09F480E06E
:10337000089580915204909153044AE050E060E037
:1033800070E001960E9433E397FD1EC080915204C5
:10339000909153044AE050E060E070E001960E9492
:1033A00033E36F3F71058105910509F07CF480914D
:1033B0005204909153044AE050E060E070E00196BE
:1033C0000E9433E3862F089580E008958FEF0895DB
:1033D000EF92FF921F93CF93DF937C0184E5B6DFDA
:1033E000182F882339F1C5DF8823F9F0EEE7FCE2D6
:1033F0008491EF012196882321F00E94008FFE0125
:10340000F7CF8DE40E94008FB701FF0C880B990B5A
:103410000E946D8FAEDF682F70E088E29AE20E9412
:103420006B768AE00E94008F09C0A3DF8093550469
:1034300010E004C08091560480935504812FDF91E1
:10344000CF911F91FF90EF900895E0915204F09179
:103450005304818121E030E0803239F42F5F3F4F07
:10346000DF01A20FB31F8C91F7CF8D3211F08B3299
:1034700031F42F5F3F4FDF01A20FB31F8C918E32CB
:1034800019F4E20FF31F818180538A3030F471DF29
:1034900091E0811103C090E001C091E0892F08956F
:1034A00080915204909153044AE050E060E070E053
:1034B00001960E9433E3CB010895809152049091CC
:1034C00053044AE050E060E070E001960C945BE445
:1034D0000F931F93CF93DF93C0915204D091530465
:1034E00065E470E0CE010E949BED8C01CE01019657
:1034F0000115110541F460E070E0DF91CF911F915B
:103500000F910C94CDE1F801108260E070E00E9410
:10351000CDE125E4F8012083DF91CF911F910F9138
:103520000895BF92CF92DF92EF92FF920F931F9375
:10353000CF93DF9383E8E82E8CE0F82E0CEB14E0B9
:1035400097E5C92E94E0D92EC0EBD2E0BC2E84E0E2
:10355000B80E8991FBDE8823D1F0BADFF601208115
:10356000211104C020915B04222331F0F801208155
:1035700031814281538103C020E030E0A9010E94E3
:1035800062EAF70160837183828393830AC0F80142
:1035900080819181A281B381F70180839183A2838D
:1035A000B383F4E0EF0EF11C0C5F1F4F8FEFC81ACE
:1035B000D80ABC12CECF86E4C9DE8823B9F088DFF2
:1035C00020E030E0A9010E9488EC18167CF480DF2E
:1035D00020E030E040E752E40E943EEB60930002BE
:1035E000709301028093020290930302DF91CF91C6
:1035F0001F910F91FF90EF90DF90CF90BF900895B3
:1036000067DF20E030E04AE754E40E94A4E60C942F
:10361000ABEB2F923F924F925F926F927F928F927D
:103620009F92AF92BF92CF92DF92EF92FF920F9351
:103630001F93CF93DF931F92CDB7DEB70E943C71EB
:10364000811180C280916E06843058F42FB7F894AF
:103650008091130D9091140D2FBF891B8F7709F066
:1036600047C180912D10882309F46CC280916E06A9
:10367000811102C01092870DEE24E3944091A912AB
:103680005091AA126091AB127091AC128091A51268
:103690009091A612A091A712B091A81248175907AD
:1036A0006A077B0708F4E12C00E010E0992493946A
:1036B00080E6882E99EFC92E99E2D92E25EFA22E09
:1036C00029E2B22E3DE8732E80916E06843008F018
:1036D00039C2E11037C28091870D811133C28091C8
:1036E000001290910112A0910212B09103128093E6
:1036F000A9129093AA12A093AB12B093AC1241E01E
:1037000050E0BE016F5F7F4F88EF91E10E94F47A35
:10371000019719F4898190E002C08FEF9FEFF82E96
:10372000EE24E3942090A9123090AA124090AB129C
:103730005090AC124091A5125091A6126091A71220
:103740007091A8122416350646065706C8F4E12CD7
:103750008F3FEFEF9E0709F47CC0FAE08F1709F462
:1037600097C02DE0821709F493C083E2F81619F090
:103770009AE3F912A3C08091860D81119FC083C086
:10378000E4E1FAE284912F012FEF421A520A8823D2
:1037900021F00E94008FF201F5CF0E949B5D88EF1F
:1037A00091E10E94E57E80911312882359F18150A6
:1037B00080931312789EC001112441E061E0885E7D
:1037C0009D4E0E942687E091131284E0E89FF0014D
:1037D0001124EC5EFD4E40815181628173814093E2
:1037E000A9125093AA126093AB127093AC1288EF97
:1037F00091E10E94CE7880912E108823D1F0909292
:103800002D1017C010922D10D092520CC092510C56
:103810000E943C710E9420A80E9439A86D33710556
:103820008105910530F0B092520CA092510C0E948B
:103830003C711092B11280912E10882319F00E94D1
:10384000888921C00E943B8A80912E108111F7CF78
:103850001AC0E7E7F7E284912F019FEF491A590A4E
:10386000882321F00E94008FF201F5CFE5E0FAE213
:1038700084912F012FEF421A520A882321F00E94CF
:10388000008FF201F5CF83E2F81202C09092870D0B
:103890001092860D0115110509F416CF80916A0466
:1038A000889E000D111D1124F801E351FB4F108279
:1038B00080E00E940D7100E010E006CF0F35110589
:1038C00008F002CF9BE3F91202C09092860D80911E
:1038D000860D8111F9CE80916A04F801889EE00D71
:1038E000F11D1124E351FB4FF0820F5F1F4FECCE0F
